:020000040000FA
:1000000092EF01F01200FFFF10EF04F01200FFFF6B
:1000100000000901C80E926F66806650010B06E071
:100020000901925103E009019207F7D7120000007D
:100030000901C80E926F66846650040B06E0090140
:10004000925103E009019207F7D71200D9CFE6FFDA
:10005000E1CFD9FF3F0E6816676A666AFE0EDB5075
:100060006712FD0EDB506812678AE552E7CFD9FFB1
:100070001200D9CFE6FFE1CFD9FFFE0EDB506A6E4A
:1000800067AE02D0FF0E30D00F0E671408080CE0E8
:100090000F0E67140B0808E06850040B03E168506A
:1000A000010B1FE0000E20D00F0E6714080804E0BB
:1000B0000F0E67140B0818E10901C80E926F685003
:1000C000010B04E0925102E09207F9D76850040B4B
:1000D00001E0010E496E1F0E66144910F7E166AC8F
:1000E00002D0FE0E01D0000EE552E7CFD9FF12007C
:1000F000D9CFE6FFE1CFD9FF0000FE0EDBCFE6FF50
:10010000B8DFE552006E005003E091DF005000D0F0
:10011000E552E7CFD9FF120000007ADF700EE66EDD
:10012000E7DFE552000901E028D0800EE66EE0DF4F
:10013000E552000901E021D0E66ADADFE552000964
:1001400001E01BD0400EE66ED3DFE552000901E06E
:1001500014D0016A1E0E015C0FE20150EA6A000F22
:10016000E96E060EEA22EF50E66EC2DFE5520009A4
:1001700001E003D0012AEED75ADF12000000016A25
:100180001E0E015C09E20150EA6A000FE96E060EDC
:10019000EA22EF68012AF4D712000000016A1E0E5D
:1001A000015C09E20150EA6A000FE96E060EEA22DC
:1001B000EF6A012AF4D712000000EFDFE66A080EAA
:1001C000E66E44DFE552E552090E696E21DF700EDE
:1001D000E66E8EDFE552000901E01CD0800EE66E6F
:1001E00087DFE552000901E015D0C80EE66E80DF1A
:1001F000E552000901E00ED0E66A7ADFE552000917
:1002000001E008D0E00EE66E73DFE552000901E080
:1002100001D00DDF12000000CFDF0601050E026FD6
:100220000601340E036F0601460E146F0601050E1B
:10023000176F0601040E186F0601640E196F060190
:10024000010E1A6F0601670E1B6F0601020E1C6F6E
:100250000601600E1D6F60DF1200000037D836D82F
:100260008D8A8D8C84848C80120009018E6B09012B
:100270008A07000E8B5B09018D5109018C5D04E03A
:1002800084948C908D9A8D9C8E2FFED709018D5170
:1002900009018C5D06E009018CB18C8009018CB3E9
:1002A00084848E2FFED78CC98DF9120000000900BE
:1002B000F5CF89F90900F5CF88F9090188510901BD
:1002C00086270901895109018723120000000901CD
:1002D000886B896B0901540E885D3D0E895905E2D2
:1002E0000901882B000E8923F5D7120000000901AF
:1002F000886B896B0901220E885D060E895905E21B
:100300000901882B000E8923F5D7120000008250C6
:10031000010B03E08250020B02E1010E02D0000E3D
:1003200000D01200C16A0F01DF0E256F0F01F70E1A
:10033000246F0F01E00E236F3A0EC06EEF0E896E30
:100340008A6A8B6A9A0E8C6E100E8D6E8E6A8F6A18
:10035000010E906E200E916EEF0E926E070E936E50
:10036000930E946E600E956E030E966E7D0E976ED4
:10037000060E986EFE0E996ECF0E9A6E8A8AC79EF2
:10038000C698C78CF00EC616C680C68A240EAC6E00
:10039000190EAF6E900EAB6EF29EA698636AFE0EBB
:1003A000626E010E616E7F9E7F9C7F84550E7E6E15
:1003B000AA0E7E6E7F82F28EFFDEAEDE4EDF090178
:1003C000916BA4DF000904E10A0E0901915D09E2C5
:1003D000640E0901915D05E279DF78DF0901912B57
:1003E000F0D77F9409019151630802E218EF02F0FF
:1003F0000901866B876BF66A080EF76EF86A56DF9E
:10040000000009018851891102E102EF04F04EDF7A
:10041000800EF61805E1FD0EF71802E1010EF8183E
:1004200001E0F5D709018651871102E102EF04F0DE
:1004300001D81200F0DE09018C6B09018BA703D0F3
:100440000901010E8C6F11DF9EAA17D0AECF8FF974
:10045000490E09018F5D0AE14B0EAD6E47DF580E64
:10046000AD6E44DF320EAD6E41DF02D08FC9ADFFFD
:10047000440E09018F5D01E101D0DDD709018A6BCE
:100480008B6B0901020E8C6F09018AA902D0090148
:100490008C6BEBDE2FD8020EF85C05E1420EAD6EE0
:1004A000F86A0ED8FF000CD8410EAD6EEAD71200E4
:1004B0000000550E7E6EAA0E7E6E7F820000120036
:1004C000940E7F6EF5DF000EE96E090EEA6E0A00EB
:1004D0000901100E846F0901080E856FEE50F56E4C
:1004E0000F00852FFBD7840E7F6EE2DF842FF3D7BA
:1004F0007F94120000000901906B0901846B0901CF
:100500008451496E4A6AD8904A5004E6840E495C88
:10051000000E4A5814E29EAAFED7AECF8FF9090109
:100520008451EA6A000FE96E090EEA228FC9EFFFD3
:1005300009018F51090190270901842BE0D7090196
:1005400090510BE1030E0901825D07E280C9F6FFBD
:1005500081C9F7FF82C9F8FF03D04E0EAD6ECBD72D
:100560001200FFFFFFFFFFFFFFFFFFFFFFFFFFFF87
:10057000FFFFFFFFFFFFFFFFFFFFFFFFFFFFFFFF8B
:10058000FFFFFFFFFFFFFFFFFFFFFFFFFFFFFFFF7B
:10059000FFFFFFFFFFFFFFFFFFFFFFFFFFFFFFFF6B
:1005A000FFFFFFFFFFFFFFFFFFFFFFFFFFFFFFFF5B
:1008000000001200280EE66E61ECE5F0E552FFEF05
:10081000E4F01200FFFFFFFFFFFFFFFFFFFFFFFFFE
:1008200091EF1FF01200FFFFFFFFFFFFFFFFFFFF31
:100830000000B9ECB6F0990E496E9C0E4A6E010E9E
:1008400015EFC1F0B9ECB6F0000E496E9D0E4A6E80
:10085000010E15EFC1F0B9ECB6F0E50E4B6E9D0E32
:100860004C6E010E4D6EFE0EDBCF4EF050ECB8F02C
:10087000F3ECC4F0B5EFB6F0B9ECB6F06E0E496E1D
:100880009B0E4A6E010E15EFC1F0B9ECB6F0590E91
:10089000496E9B0E4A6E010E15EFC1F0B9ECB6F031
:1008A000C30E496E8E0E4A6E010E15EFC1F02BEC91
:1008B000C1F0050DBAECB7F00A0E49260A0E4A221D
:1008C000FD0EDB504924E96E000E4A20EA6EEF501F
:1008D000B5EFB6F02EC1E6FFBEDFE5521200350ED1
:1008E0000124E66EB8DFE5521200B9ECB6F0EC0E6A
:1008F000496E8F0E4A6E010E15EFC1F09EC1C4F114
:100900009FC1C5F1A0C1C6F1A1C1C7F1A2C1C8F183
:1009100012000A0E8EECC1F03D501200640E8EECF7
:10092000C1F03D501200E80E496E030E4A6E85EC90
:10093000B8F00BEFC6F0010155513C0DF3CF16F2A4
:10094000F4CF17F21200640E496E4A6A37C23DF0C6
:1009500038C23EF00BECC6F0006E1200E66A45ECC1
:1009600022F0E5521200010E6FEFB7F0020E6FEFAA
:10097000B7F087C2E6FF63EFC4F0E66A63EFC4F046
:1009800001018AB73B0C300CAFECBDF019E3E5EC8C
:10099000C2F002E6CAECBFF013E2AFECBDF010E328
:1009A000E5ECC2F002E6CAECBFF00AE2AFECBDF043
:1009B00007E3E5ECC2F002E6CAECBFF001E2010C8D
:1009C000000C909000000000000000000701D06BB8
:1009D0000101D2A304D00701D0830701D081010116
:1009E000D2A504D00701D0870701D085D0C7E6FF84
:1009F00095EC53F0E55200000000000000008E82EC
:100A0000040EE66E61ECE5F0E5528E92040EE66EA1
:100A100061ECE5F0E552000000000000000090806D
:100A200012002150100B08E0640E02010B5D04E37C
:100A3000EEECB8F001E02198120079ECC0F0010171
:100A4000AC6BB59F1200010156A1010CD70E6CECE6
:100A5000C6F0F00802E2EF0E006E00501E0803E23E
:100A6000F00E005C01E3000C010CA70EE66EB30E65
:100A7000E66E010E14ECB7F07CECC0F006E1EEEC93
:100A8000BCF003E001011E0EAC6F66C100F08BEC00
:100A9000BBF00A0E665D02E2200E1A6F1200A00E75
:100AA000E66EB30EE66E010E14ECB7F068C100F00E
:100AB00000500AE00101030E016F8BECBBF00A0E3F
:100AC000685D02E2200E1A6F120001014851120007
:100AD000800E071406E02050010B03E102012151B2
:100AE00001E0000C010C0201010E3A6F7E0E00ECD9
:100AF000B8F001011E0EAC6F120027EC33F071EC60
:100B000029F0A8EF14F02BECC1F004080FE0CFECB3
:100B1000B7F00EE0FE0EDB500A0808E0FE0EDB50D8
:100B20000D0804E0FE0EDB50090802E1010E01D0C1
:100B3000000EB5EFB6F007019351D880925502E24E
:100B400092C793F792079051902BEA6A000FE96ED3
:100B50000C0EEA22EF501200D9CFE6FFE1CFD9FF09
:100B6000FE0EDB50D80805E1300EF36EFE0EF3CF1B
:100B7000DBFF060EAB1405E0AB98000000000000A0
:100B8000AB88200EF36EFE0EDBCFF4FFF350F45C67
:100B900004E3FE0EDB507E0807E2FE0EDBCFE6FF2D
:100BA000B2DFE552000944E00401F051496E4A6A9F
:100BB000D8904A5004E6FF0E495C000E4A5838E2CD
:100BC000FE0EDB503B0804E0FE0EDB507C0802E129
:100BD0000401F92BFE0EDB50210804E0FE0EDB5071
:100BE00040080AE13B0E0401FE5D04E07C0E0401B6
:100BF000FE5D02E10401F92BFE0EDBCFFEF40401E1
:100C0000F151EA6A000FE96E0B0EEA22FE0EDBCF0D
:100C1000EFFF0401F12B0401F02B0401F05108E176
:100C20000401FE6BFEC4F9F4FEC4F1F4FEC4F2F458
:100C3000E552E7CFD9FF1200ACA212000401F8512F
:100C400004ECC2F0006E0050E66E5BECBBF000C03E
:100C5000EFFF3B0E005C03E07C0E005C01E129909D
:100C60000401F82B1200B9ECB6F0ACA2FED72FECC1
:100C7000C1F05BECBBF0FE0EDBCFEFFFB5EFB6F0E3
:100C8000F2EC0EF0010EE66E11EC0FF0E5528494DA
:100C90008C908D9A8D9CF29E0000F66A080EF76E7D
:100CA000F86A940E7F6E550E7E6EAA0E7E6E7F825F
:100CB000000000EC00F012000401F007F251EA6AB3
:100CC000000FE96E0B0EEA22EF50006EF22B1200BD
:100CD000ABECBAF00AE11F50020B07E102018951A7
:100CE000020B04E18951010B01E1000C010CE6EC5F
:100CF000C0F02050200B1FE08250010B03E1825016
:100D0000020B03E02F50400B16E030ECBEF02F9C9E
:100D100038ECBEF08CECCFF09CECCFF0980EE66E89
:100D2000B30EE66E010E4CECC3F00101E79988ECBE
:100D300087F03DEC0FF0E552B5EFB6F0E6ECC0F011
:100D4000DF6A780E4C6E910E4D6E010E4E6EFD0EEA
:100D5000DBCF4FF0506A516A090E416E426A436A16
:100D60004FC03CF050C03DF051C03EF0E9ECE0F027
:100D700039C04FF03AC050F03BC051F0BEECBCF06F
:100D8000DFCF52F0536A546AAFECBAF00800F5CFE7
:100D900000F0F5500DE0090EDF5C0AE2FE0EDB50BC
:100DA00003E1D8ECD5F002D0FBECD5F0DF2AC9D7AF
:100DB000E552B5EFB6F02750200B06E005011051C3
:100DC000020119112D1101E1000C010C81EC1DF043
:100DD000CFECBFF02D6B3751381102E0209449DA87
:100DE0000AEF5CF00701BA51010B07E08AECB8F09A
:100DF00004E0050ED45D01E0000C010C0101269D0C
:100E0000010E0D6E26BF0D681200030E6FECB7F0D9
:100E1000258E12006A0E28EFB7F06B0E28EFB7F0A0
:100E200001018E51010B08E093EC0DF0000904E084
:100E300001013B51800B01E0000C010C040E6FEC32
:100E4000B7F001013C0EAC6F12000101AC510EE194
:100E50002DAC09D06E0EE66E950EE66E010EA7EC77
:100E6000B8F0E55201D0EADF258E2D8C1200258ED8
:100E7000050E6FEFB7F019ECB9F000010E6EE66ADF
:100E800083ECC2F00F6E120087C1E6FFA80E22ECC1
:100E9000B7F093C100F0330E0201875D07E10A0E3F
:100EA00001019503F350FE0BE842006E0050E66E20
:100EB000A90E22EFB7F0B9ECB6F0FE0EDB509BECBA
:100EC000B7F0EF500BE1FE0EDFECB7F007E34DECAF
:100ED000BDF09BECB7F0100EEF6EEFD7B5EFB6F0AC
:100EE000B9ECB6F0FE0EDB501FECB9F0EF50300855
:100EF0000BE1FE0EDFECB7F007E34DECBDF01FECAD
:100F0000B9F0200EEF6EEED7B5EFB6F0830E096E96
:100F1000FA0E8EECB8F000500E6E0EC00FF00E6A96
:100F2000FB0E70ECC6F00050C6EFB8F03AC18BF281
:100F3000120001013A51130804E2010E3A6F2BA688
:100F40003A6B1EEFAAF02BECC1F0020802E1B6C723
:100F5000B5F7FE0EDB0402E1B5C7B6F7B5EFB6F0A4
:100F60008CECC3F040EFBEF042C1ABF242C1AAF23A
:100F70008CECC3F0EF50400B03E00201020EAA6FAD
:100F80000101D551C9ECB7F0EF50400B03E002016D
:100F9000020EAB6F1200E6ECC0F02850010B11E11D
:100FA000F8ECC4F010E14A500EE11750010B03E0D9
:100FB000220E155C06E01F50100B05E0290E155C93
:100FC00002E1000E01D0010EDF6E2C50800B03E118
:100FD0002C50400B02E0010EDF6E2890DF50E552EE
:100FE000B5EFB6F01A9C238A12000101E38B11C5FC
:100FF00012F50501106B279A1200B2ECBCF01EE04E
:101000000901E6511BE0E8ECC2F0E6C9E6FFDCECC2
:101010000EF0E5520901E75105E0E7C9E6FFDCEC17
:101020000EF0E5520901E76BE7C9E6F901013699CF
:101030000450010B01E036890AEF07F0010136AFD9
:1010400005D004A002D01A8812001A8A1200B9EC46
:10105000B6F0B2ECBCF00CE0FE0EDB5009E0C5DFF0
:101060004FECC3F00901E6AF02D001013689D2DEB0
:10107000B5EFB6F0B9ECB6F0B2ECBCF011E0FE0E94
:10108000DB500EE0FD0EDB500BE0AFDF4FECC3F0AA
:10109000F5ECBEF0FE0EDBAE02D001013689BADE01
:1010A000B5EFB6F0B9ECB6F0010136AD12D0E8EC10
:1010B000C2F04FECC3F0FD0EDB5002E0F5ECBEF0E9
:1010C00001013699FE0EDBBE3689DB5008E0A2DE58
:1010D00006D0FE0EDBAE02D01A8801D01A8AB5EF18
:1010E000B6F0CBECC5F0DBCFFBF60201D65101E147
:1010F00005D80201190ED66FB5EFB6F002ECC1F0BB
:10110000010EFBC6DBFFB2ECBCF062E02050200B0E
:101110005FE00601FB51FC5D5BE067DF7BDE010108
:101120003689890E82ECB7F00101E3A50BD0530E8E
:1011300082ECB7F0570E82ECB7F0520E82ECB7F0AB
:101140000101E395640EEFECC1F068ECC4F0DF50F0
:10115000300805E2DFCFE6FFDCEC0EF0E552640E6E
:10116000C8ECBCF03AC0DBFF63ECB7F068ECC4F04D
:101170000101E7A503D0520E82ECB7F0DF50300832
:1011800008E30601FB51630804E30101E751040B86
:1011900008E0300EDF5C02E1540E01D0DF5082EC3B
:1011A000B7F00101E7A303D0520E82ECB7F063EC75
:1011B000B7F0010EDBCF3EF080ECC0F0300FDF6EF9
:1011C000300EDF5C02E1540E01D0DF5082ECB7F04C
:1011D000FBC6FCF6020EE15C02E2E16AE552E16E5A
:1011E000B5EFB6F0690E28EFB7F0060E87ECC2F047
:1011F000280EDDECB6F0F2EF08F0010136BFF5DFA6
:1012000012000601980ED880B0553A0EB15509E289
:101210000E50B05D0101D86F0F500601B1590101A8
:1012200008D0B0510E240101D86F0601B1510F2032
:101230000101D96F1200190E3D6E3E6A0EC042F0D8
:101240000FC043F0CBECE0F03BC037F23CC038F2CB
:10125000180E426E436A37C23DF038C23EF015ECBC
:10126000E5F03DC037F23EC038F21200EB0E28EF39
:10127000B7F00101E693199A139276EC15F0F6DFB8
:101280000201376B386B19942CEF0BF088EC96F059
:101290000A0EDDECB6F0E30E4BECB8F0006E005039
:1012A000F5E11200B9ECB6F0F1DFEC0E90ECC3F012
:1012B00091EC69F000C709F0FC0E016E0FC000F060
:1012C0000BEC34F0012A0EC000F00BEC34F0096A8C
:1012D000B5EFB6F0660E28ECB7F019801200670E75
:1012E00028ECB7F019901200E6ECC0F009EC1CF005
:1012F000DF6EBEECBEF007E019A00ED0F0DFDF50CD
:101300000BE1006A07D019B007D0E4DFDF5004E139
:10131000010E006EC3EC6AF0E552B5EFB6F06BEC6F
:10132000B7F003E03450400B04E001015751040BC7
:1013300001E1000C010CE6ECC0F001018AA10AD029
:1013400009EC1CF0DF6EDF0403E0020EDF5C02E15B
:10135000010E01D0000EE552B5EFB6F0ECDF00094A
:1013600005E109EC1CF0040801E0000C010CF6DFBB
:10137000000905E109EC1CF0050801E0000C010C76
:10138000E6ECC0F01E50010B0EE0B9ECB9F00BE03A
:101390006BECB7F003E0F2ECBCF005E11950020B86
:1013A00002E1000E01D0010EDF6EDF5002E09BEC87
:1013B00004F0DF50E552B5EFB6F0E6ECC0F01D509A
:1013C000040B1AE01D50080B17E01E50010B14E02F
:1013D000B9ECB9F011E0050110510EE12050040BF9
:1013E0000BE12050010B08E16BECB7F003E0F2ECED
:1013F000BCF002E1000E01D0010EDF6EDF5002E012
:101400009BEC04F0DF50E552B5EFB6F0840E55ECDE
:10141000BBF0010136AD02D06FEFC4F036BF258EB0
:10142000120002ECC1F0C20EDE6E010EDD6E09ECA0
:101430001CF0010804E009EC1CF002080BE1F40EBA
:10144000DE6E010EDD6E0101345104E0260EDE6E0B
:10145000020EDD6E01C2E6FF00C2E6FF740ED3ECA1
:10146000B6F0020EE15C02E2E16AE552E16EB5EF30
:10147000B6F01D9CB4ECBDF0D0DCDF0E55ECBBF03B
:10148000258E12002BECC1F00A0DF3CF5AF3F4CFE6
:101490005BF3000E03015A27030E5B23B5EFB6F092
:1014A0006B0E005C05E20201AA510101245F1200EB
:1014B000E5ECC2F004E6990E495C000E4A5804E2DD
:1014C0000201AA510101242712001200280E010175
:1014D000D8806855040DF328016E0150E66EAA0EFF
:1014E00022EFB7F0B9ECB6F02AA40AD095ECB8F028
:1014F0003BEC22F0B7ECC5F00101500EAC6F2A9422
:10150000B5EFB6F0149E0A01DA51800B03E1ABECA3
:10151000BAF001E1148E12000101D451080DA7ECBC
:10152000B9F0010ED8904B364C36E806FBE102507C
:10153000080D4B50F324496E4C50F4204950016E75
:1015400012000A01DA8FDEDF02018051D3ECB7F01E
:101550001CE249509608000E4A5417E202687F05C3
:1015600001E1026A030E7F5D02E1010E026EFF0ED1
:10157000025C16E0670E096ECFDF080EE66ED40E31
:10158000E66E0A0E54ECC3F00BD091EC6AF01EAC80
:1015900003D00201098902D00201068B05014785AB
:1015A00002017F6B0101B58F500EAC6F2496318C18
:1015B00012000201996999C289F799C288F799C204
:1015C00087F799C286F799C285F707018E698F69F7
:1015D0008C698D698CC78AF78DC78BF71200040E52
:1015E0000101805D03E18150100B07E0050E805D75
:1015F00003E18150100B01E1000C010C1200E6EC3C
:10160000C0F00101A85103E19E51200821E2DF6AE8
:10161000090EDF5C10E2DF509FECB8F0EF50040BD6
:1016200008E0100EDF24E66E53EC28F0E5520009C6
:1016300002E1DF2AEDD7090EDF5C0AE2100EDF2699
:101640002986DFCFE6FF12EC28F0E552DF5001D00B
:10165000000EE552B5EFB6F01F86B4ECBDF0B599BB
:10166000B59B2582238A1200D9CFE6FFE1CFD9FFAF
:10167000030EE126010EC7CFDBFF020EC6CFDBFF54
:10168000C00EC7128C9600000000FE0EDBCFE6FFF6
:1016900095EC53F0E5520000C950DF6E00008C86D7
:1016A000030EE66E8AECE5F0E552010EDB50C76EE4
:1016B000020EDB50C66EDF5000D0496E030EE15CB7
:1016C00002E2E16AE552E16E4950E552E7CFD9FF07
:1016D0001200A2EC53F0F00EC616C680C68A1200A5
:1016E000800EE66EE66A010EE66E1EECE4F0B7ECE4
:1016F000C5F069EF0BF01282128006010191020120
:101700001E0E306F120012901FA2128012921FB292
:10171000128212002AECC2F0C9ECB7F0EF50E84098
:10172000E8403F0BDF6E000EDF94DF96DF98DF9A14
:10173000DF9CDF9E0A0E006EFE0EDB500DE1DF50D7
:1017400002E1010E006EDF0402E1020E006E020EE5
:10175000DF5C30E1050E2DD0FE0EDB50030804E106
:10176000DF5002E1010E006EFE0EDB5004080EE1B8
:10177000DF0402E1320E006E020EDF5C02E15A0E5F
:10178000006E030EDF5C02E1640E006EFE0EDB04F1
:1017900004E0FE0EDB5002080DE1DF5002E1010E15
:1017A000006EDF0402E1050E006E030EDF5C02E155
:1017B000190E006EE552B5EFB6F0ECECC3F0C4C103
:1017C00000F0000406E10101C551460802E2020EE4
:1017D000006E030E005C06E10101C551280802E21B
:1017E000040E006ED5CA03F0C6ECBEF005E037511A
:1017F000080B02E0040E036E880E4A6E8D0E4B6ECF
:10180000010E4C6E0050A9ECB7F0035091ECBBF008
:10181000EF504924016EBF0E4A6E8D0E4B6E010EC5
:101820004C6E0050A9ECB7F0035097ECBBF0EF50B2
:101830004924026E8BECC5F0E66A7D0EC0ECB8F070
:10184000ECECC3F0280E026E016EC6ECBEF00EE0AA
:101850003751080B0BE01CCA01F021CA02F00150FD
:1018600002E0025003E1280E026E016E8BECC5F01F
:101870007C0ED3ECB6F0ECEFC3F0129A1FB2128AD2
:1018800042DFD4ECBFF0FCEC5FF01F50020B06E02F
:101890000101D551D45D02E01A8C12001AAC02D0BD
:1018A000F2EC07F01200080E0B5C04E33CECC2F013
:1018B00001E1000C010C095004E00701010EFDECF0
:1018C000C4F0096AC4EC04F0000907E0750EE66E86
:1018D000280EE66E010E01ECC5F01200C4EC04F017
:1018E000000909E07E0E096E0C0EE66EB60EE66E7D
:1018F000020E01ECC5F0096A1200CBECC5F0DBCF9B
:1019000048F105ECC5F0E66AF6ECBCF0CFECBFF0B0
:101910001398B5EFB6F00101485112E0060EEFEC56
:10192000C1F048C13EF0EFECC3F0006E005001E1A1
:10193000002A00500101485F48C15BF2DAEFB8F0BD
:1019400083EFBAF00701585106E1080E4BECB8F0EE
:101950000501261501E1000C010C2C9E2C9C71EC5C
:1019600029F0CFEF87F0B9ECB6F0D8ECBFF007E183
:101970002B50010B04E101018A51200B09E140C207
:1019800043F23FC242F23EC241F2FCECBEF009D04B
:10199000FE0EDB5006E043C240F242C23FF241C2BB
:1019A0003EF204802BA002D004902B90A6EC39F0DC
:1019B0000101320EAC6FB5EFB6F025B41200189AE3
:1019C00017B8188A12000301916B926B936B946B9A
:1019D00091C38DF392C38EF393C38FF394C390F3AB
:1019E000030E016EFF0E015C32E0056A030E026E0B
:1019F000FF0E025C22E00250EA6A890FE96E030ED4
:101A0000EA22EF504B6E4C6A0150EA6A850FE96E8C
:101A1000030EEA22EF50DFECB9F009ECBDF0EF5015
:101A2000C6ECB8F00550C6ECB8F009ECBDF00EC03D
:101A3000EFFF0FC005F00206DBD70150EA6A8D0FF9
:101A4000E96E030EEA2205C0EFFF0106CBD71200B4
:101A50002BECC1F0006E00AE04D0006C01010E0E44
:101A6000116F0101040EDDECBFF012510AE111C14A
:101A700012F1100E116F135104E112C113F1100E87
:101A8000126F130E156FB5EFB6F08AECB8F003E1E4
:101A9000030E0A5C01E0000C010C8AECB8F005E1D1
:101AA000020E0A5C03E00A0401E0000C010C8AEC5F
:101AB000B8F003E1020E0A5C01E0000C010C8AECB4
:101AC000B8F007E10A5005E1CF51040B01E0020C28
:101AD000010C000C8AECB8F005E1020E0A5C03E090
:101AE0000A0401E0000C010C0601EC5106E08AEC4E
:101AF000B8F003E10A50000801E3000C010C8AEC85
:101B0000B8F004E10A0403E00A5001E0000C010C03
:101B10008AECB8F006E1020E0A5C04E0030E0A5CEF
:101B200001E0000C010C6BECB7F003E011ECBEF02F
:101B300001E1000C010C0101D45104E10A01DA5168
:101B4000040B01E1000C010C0101D45104E10A0174
:101B5000DA51080B01E1000C010CFAECBCF009E0D1
:101B60000301B851F3ECC3F0DFECB8F0210ED3EC75
:101B7000B6F01200FAECBCF002E0ADEF0DF0E66A50
:101B8000E66A210ED3EFB6F08AECB8F010E1D0513E
:101B9000040B05E00A040CE0020E0A5C09E0CF51D8
:101BA000040B05E00A5004E0030E0A5C01E0000C9F
:101BB000010C0101D45103E1D051400B04E1E4DFF9
:101BC000000901E1000C010CFEECBCF001E0030C8B
:101BD00084ECC0F001E0080C88ECC0F001E11B0CC3
:101BE000D45109E0030ED45D05E10A5004E0030E70
:101BF0000A5C01E0030C010CFEECBCF001E00A0CF5
:101C000084ECC0F001E0380C88ECC0F001E1640C19
:101C1000D45101E0500C380CEFDFE66ED5DFE66EF4
:101C2000D60EE66E0A0E07EFB7F038EC3AF0190E52
:101C300001240A01D880D75503E2190E0124D76F79
:101C4000190ED8800154D75D04E2190ED8800154D2
:101C5000D76FD46B33889DEFBBF0FEECBCF004E192
:101C600084ECC0F001E1000C010CEF0E896E8A6A71
:101C70008B6A9A0E8C6E100E8D6E8E6A8F6A010EB4
:101C8000906E200E916EEF0E926E070E936E930E75
:101C9000946E600E956E030E966E7D0E976E060E18
:101CA000986EFE0E996ECF0E9A6E12001F98258ABE
:101CB0000101B59B02011A511FE0020E685D03E1AC
:101CC000CAECBEF019E00701BA9BBA9B32BCBA8BD2
:101CD000B0EC07F00601EA05EB6F020EEA5D01E2E7
:101CE000EB6BEBC600F00101D45102E0EDC600F051
:101CF0000050E66E11ECC2F002011A6B2582120050
:101D0000C08EA70EB6ECB9F0C3CF0EF0C4CF0FF063
:101D1000A70EB6ECB9F0C3500E26C4500F220EC069
:101D20004DF00FC04EF0D8904E324D320EC04FF0F5
:101D30000FC050F0D89050324F32D89050324F32BE
:101D40004D504F244B6E4E5050204C6E0EC051F0F3
:101D50000FC052F0040ED89052325132E804FBE129
:101D600051504B5C496E52504C584A6E0EC053F065
:101D70000FC054F0060ED89054325332E804FBE101
:101D8000495053240E6E4A5054200F6E0EC0D1F2AB
:101D90000FC0D2F2C09E1200D1C20EF0D2C20FF01C
:101DA000E66AF8EC21F0E5520101200E166F1C6F77
:101DB000188F410E1B6F1200B9ECB6F005011151DE
:101DC000EA6A000FE96E080E94ECC3F0112B115172
:101DD00074ECB7F002E6E2ECBFF001E3116B102BFC
:101DE000B5EFB6F0C4EC04F0000910E035ECB9F042
:101DF000020E0101395D02E1010E396F5CDD1CEC60
:101E000040F06CDD27EC40F088EF6EF07E0E096E3E
:101E1000040EE66EBE0EE66E020EE66E080EF1EFE2
:101E2000C5F0B9ECB6F030ECBEF069EC13F08A986E
:101E30008A86AEEC20F00101766B140EE66EF0ECB3
:101E4000B0F0E552FE0EDB500CE06FEC09F0F2EC66
:101E500008F024ECB2F099ECB2F072ECD6F0BCECE5
:101E6000D4F00601506B7FEC36F00601516B010196
:101E7000B96BEF0E926EB5EFB6F0F29E95ECE5F011
:101E8000F26AF06AB96A9D6A000EA66EA16E9E6E35
:101E90008D8C8D8A8C908484070E936E00000000D8
:101EA00000008A9A0000000000000000270E936ED8
:101EB0004E0E996E000000000000030000000000BC
:101EC00000000000FF001200E6ECC0F020AA3BD0AA
:101ED000E7ECBFF006E3F6ECC3F035E2B9ECBDF099
:101EE00032E21B50080B2FE1E7ECBFF006E3F6EC03
:101EF000C3F029E2B9ECBDF026E2E7ECBFF006E35F
:101F0000F6ECC3F020E2B9ECBDF01DE20050DF6E4C
:101F1000DF50D3ECB7F013E2B9ECBDF010E2DF50C4
:101F2000ECECBFF004E6B40E4B5C000E4C5807E23C
:101F3000900EE66EB30EE66E010E03ECBFF0E66A9D
:101F400070DFE5529ADFE552B5EFB6F0B9ECB6F0C6
:101F50009CECCFF095ECB8F050ECB7F08EECD3F0F1
:101F6000E7ECB9F0E7ECB9F0E7ECB9F0FA0ECFEC3A
:101F7000C2F0FA0ECFECC2F0B5EFB6F0C3CF0EF060
:101F8000C4CF0FF0CEECBEF0CEECBEF0460E0F028A
:101F9000F3CF0FF00E02F3CF0EF0F4500F260F50D8
:101FA000496E4A6A9F0E5AECC3F0006E00508008DA
:101FB00001E2006A0201FC0ED880D155080ED2550C
:101FC00002E2040E0FD0080ED880D155070ED2556C
:101FD00002E2030E07D0140ED880D155050ED2555B
:101FE00003E2020E002607D0200ED880D155030E42
:101FF000D25501E2002A0050800801E2006A080E72
:10200000D880D155070ED25502E2030E07D0140E28
:10201000D880D155050ED25503E2020E00261200DB
:10202000200ED880D155030ED25501E2002A1200AD
:1020300002ECC1F0C08EAB0EB6ECB9F0C3CF49F0E4
:10204000C4CF4AF0C0ECBBF0C0ECBBF049C0DEFF2F
:102050004AC0DDFF93DF00508AECC2F00701A527DC
:102060004A50A623A5C749F0A6C74AF08CECC0F099
:102070000DECB7F049500701A55F4A50A65BC09E22
:1020800043ECB9F002E2E16AE552E16EB5EFB6F079
:102090002BECC1F002E1C00E01D0B00E016E0101C7
:1020A0000D5101264EEC34F0FE0EDB5013E00F0E06
:1020B000005C03E3005030080DE2230E006E0901BE
:1020C000EB5108E0020E0101395D04E00901EB511A
:1020D0007DECC1F00050B5EFB6F0E6ECC0F0D9EC05
:1020E0000AF00701AD6BD4C1DFFFD5CA00F08EEC5A
:1020F000C5F0DF5003ECC4F0AD5160ECC3F0D40E7A
:10210000E66E0A0EE66E51ECBAF0149C0101D45151
:1021100003E0030ED45D06E1030E0A01D45D07E17E
:10212000148C05D0020E0A01D45D01E1148CDAA3EF
:1021300004D0D8CAB2F7D9CAB3F790EC15F08CEC3A
:10214000C3F0EFCFBAF70701BA9F0101D45103E002
:10215000030ED45D02E10701BA8F0FEC1BF03AECDD
:10216000B9F0A3ECD3F0B9EC20F0B4EC07F0E552F1
:10217000B5EFB6F0CBECBBF0CDECC1F031EFBCF07D
:102180008CECC3F040ECBEF0ABECBAF00FE00A010F
:10219000DAA306D0B2C7D8FAB3C7D9FA90EC15F0D3
:1021A000E9DF010138ECBCF0ADC7EFFF1200E6EC4F
:1021B000C0F0DF6A080EDF5C04E274ECC4F0DF2AD2
:1021C000F9D7E552B5EFB6F0E6ECC0F0DF6A080EDD
:1021D000DF5C0CE2E6ECB7F0EFCF49F0FE0EDB502F
:1021E000495C02E1010E03D0DF2AF1D7000EE5526F
:1021F000B5EFB6F0B9ECB6F018BE08D02FECC1F0D0
:1022000075EC04F0E5527F0B66ECB7F0B5EFB6F075
:10221000B9ECB6F018BE15D029A003D01CEC06F01E
:10222000FBD767ECBBF00DE067ECBBF066ECB7F0FA
:10223000D950FC0F99ECC3F0EE2A000EEE22EE22EC
:10224000F0D7B5EFB6F0B9ECB6F018BE23D029A0A0
:1022500003D01CEC06F0FBD7D3ECB8F0BEECBDF01D
:10226000D5ECC1F0BEECBDF009ECC5F015ECBEF04C
:10227000D5ECC1F015ECBEF009ECC5F08CECC0F06B
:10228000D5ECC1F08CECC0F009ECC5F0300E49245F
:1022900066ECB7F0B5EFB6F0B9ECB6F018BE0FD0FB
:1022A0001EAE0DD08B0EE66EB30EE66E010E1DEC6B
:1022B000B7F095ECB8F0ACDFE552E552E552B5EF7A
:1022C000B6F0E6ECC0F00201D32B1EAE19D0B40E6E
:1022D000E66EC00EE66E010EEDECB7F02FECC1F02D
:1022E00089DFE552FE0EDB28E66E84DFE552FE0E46
:1022F000DB50020FE66E7EDFE5523B0E66ECB7F078
:102300002FECC1F061DFE552000915E1DF6A080E2C
:10231000DF5C11E2E6ECB7F0EF50FF080AE1E6EC13
:10232000B7F0FE0EDBCFEFFF58ECBAF024C7EFFF9B
:1023300002D0DF2AECD707012469E552B5EFB6F0E9
:10234000E6ECC0F0DF6A080EDF5C0FE2E6ECB7F007
:10235000EF50FF0808E058ECBAF0EF50016EE6ECE1
:10236000B7F0EF5005D0DF2AEED70201D36BFF0E96
:10237000E552B5EFB6F002ECC1F0DF6A080EDF5CA3
:102380000FE2E6ECB7F0010EEFCFDBFFDB50FF080A
:1023900005E074ECC4F0010EDB5005D0DF2AEED767
:1023A0000201D36B000ED2ECBEF002E2E16AE5520C
:1023B000E16E4950B5EFB6F0E6ECC0F03250100BCC
:1023C00004E1020E0701585D02E1DF6A03D00BEC65
:1023D000C4F0309ADF50E552B5EFB6F002ECC1F030
:1023E0003250100B04E1020E0701585D03E1DE6A72
:1023F000DD6A08D00BECC4F0E66A83ECC2F072EC44
:10240000BCF0309A43ECB9F002E2E16AE552E16EC9
:10241000B5EFB6F0E6ECC0F007015C6B5D6B2DA884
:1024200002D0010E2ED0080E4BECB8F0DF6E070183
:102430005C2B000E5D23ECECC3F0200EDF1406E0F5
:102440000701B00E5C5D040E5D59EDE307015C51C0
:102450005E5D5D515F5904E25CC75EF75DC75FF783
:10246000B00E5C5D040E5D590BE301018B5105E17B
:102470005AC724F7330E15ECB8F02D88000E01D0A2
:10248000010EE552B5EFB6F0B9ECB6F007ECBFF0CF
:10249000B5EFB6F056ECC2F003E2D6ECBEF004D0D5
:1024A000FE0EDB50F60F410FB5EFB6F0020E006ED8
:1024B000020178B9008E35C101F00150280802E20E
:1024C000280E016E0050E66E060E0102F350E66E15
:1024D000780ED3ECB6F011EC1CF0016A0101355115
:1024E000280807E27C0EF1ECBFF003E2280E355D10
:1024F000016E0150E66E3A0E22EFB7F0E6ECC0F046
:1025000009EC1CF0DF6E0F0EE66EDF5007E0030EE5
:10251000DF5C04E001018A51020B02E1000E01D0F0
:10252000010E000905E00A0E01017A03F35001D003
:10253000000EE66E7E0ED3ECB6F0E552B5EFB6F0C7
:1025400064C178F211ECBEF002E165C178F21200CC
:1025500011ECBEF003E178C265F102D078C264F1FB
:10256000EFDF56EF12F08DC20EF08EC20FF07BEC53
:10257000C4F05E0ED3ECB6F08FC20EF090C20FF036
:102580007BECC4F05F0ED3ECB6F092C2E6FF91C2D2
:10259000E6FFE66A7B0EC0EFB8F00601B46BB56BE0
:1025A000020E35ECBBF00601B42B000EB523B4517E
:1025B000B65DB551B75904E2B4C6B6F6B5C6B7F6BE
:1025C000D00ED880B455070EB5550BE201018B51E2
:1025D00005E15AC724F7360E15ECB8F02D88318680
:1025E000010C84B0DDD7000CE6ECC0F0FE0EDBCFB2
:1025F0005AF72D50100B03E13150100B02E1000E81
:1026000020D031A604D00A0E35ECBBF001D0C5DFD6
:102610002FECC1F034EC0BF0E552DF6EE66A34ECDF
:102620000BF0E55201013851100B0AE03050200B3D
:1026300007E1E7A102D02E0E01D0210E9FECC1F0E0
:10264000DF50E552B5EFB6F026ECC1F00101E7919D
:10265000B5EFB6F026ECC1F0FC0E58ECB7F0010176
:10266000E791B5EFB6F026ECC1F081ECC4F00101C2
:10267000E791B5EFB6F026ECC1F081ECC4F0FA0EAC
:1026800058ECB7F0F90E58ECB7F00101E791B5EF4F
:10269000B6F0FEECC5F0D8C1E6FF83ECC2F0D9C1BC
:1026A000E6FF83ECC2F00EC0E6FF83ECC2F00FC081
:1026B000E6FF83ECC2F00101E791B5EFB6F01D0E25
:1026C00090EFC3F01E0E90EFC3F0D9CFE6FFB5EF49
:1026D000B6F02AB203D0600E28ECB7F02A821200BE
:1026E0002AA203D0610E28ECB7F02A9212002AB277
:1026F00003D0600E28ECB7F02A8212002AA203D081
:10270000610E28ECB7F02A921200B9ECB6F031B2A3
:1027100006D0620E28ECB7F0FE0EDBCF1BF2B5EF51
:10272000B6F0B9ECB6F0B00E28ECB7F0FE0EDBCF89
:102730001CF2B5EFB6F0B9ECB6F007018451320DDA
:10274000F6ECBFF090ECC0F012E1FE0EDB500FE1B2
:102750000101D45104E129510A0DF6ECBFF0B6ECA9
:10276000BCF005E00101E80ED86F030ED96FB5EF9C
:10277000B6F0E6ECC0F0D6CA83F707011E0E846FF0
:102780000101D45105E13CECBAF03EC084F710D011
:10279000030ED45D0DE1030E0A5C03E10701140E84
:1027A00006D021ECBAF004E065ECC3F00701846FB9
:1027B000D7CA00F00701BAAF10D0190E006E0A0197
:1027C000D75D06E2DAECBEF09EECC3F0005E05D009
:1027D000190ED75D9EECC3F00026190E005C05E3D0
:1027E000190E005C0701842705D0190ED88000540B
:1027F0000701845F080E006E21A20FD00101D451A1
:1028000002E1020E18D0D40506E0020ED45D03E00A
:10281000040ED45D11E1010E0ED00101D45102E18C
:10282000080E09D0D40506E0020ED45D03E0040EC4
:10283000D45D02E1070E006E07018351FE0BE842F2
:102840000024056EDF6A0550845D13E2DF2A8351A0
:10285000FE0BE8428425016E01500024FE0BE84285
:10286000846F0050015C02E20050016E0050015C78
:10287000836F88ECC0F004E2DFCFE6FF5CDFE55257
:1028800094ECC0F05EE00701BA51800B27E0DF5006
:1028900025E1E3DA3AECBBF00A01D751190808E266
:1028A000190ED75D8AECC2F00101D8274A50D9230E
:1028B00090ECC0F008E2DAECBEF08AECC2F0010164
:1028C000D85F4A50D95B01010A0ED903F3CFD9F181
:1028D000D803F3CFD8F1F450D92704D0DFCFE6FFE7
:1028E0002ADFE55207018351320DBFECB7F08AECC5
:1028F000B8F001E1D98F200E006E07018651005C0F
:1029000010E18A510101D8190CE107018B51010135
:10291000D91907E107018C510E1802E18D510F18EA
:102920000DE000C086F7D8C18AF7D9C18BF70EC079
:102930008CF70FC08DF7005013ECC4F06BDDADECDD
:102940000DF0DDEC0BF08FEC45F0E552B5EFB6F095
:1029500019ECBAF0005001E1120094ECC0F066E00E
:102960000101DC0ED86F050ED96FF00E0E6E0A0E47
:102970000F6E030E005C01E1D98F000403E0020E2C
:10298000005C46E19BEC09F0000915E0010189516A
:10299000640DBFECB7F03AECBBF0010E0F0B05E095
:1029A000D890D933D833E806FBE1640E0101D8276B
:1029B000000ED9232DD0010134512AE03451080DE5
:1029C000F3CFD6F1F4CFD7F15C0ED627000ED72384
:1029D000D6C149F0D7C14AF0F00ED88049560A0E48
:1029E0004A56010E0F0B04E0C0ECBBF0E806FCE118
:1029F00049500101D625D86F4A50D721D96FD6C189
:102A00000EF0D7C10FF0F00ED8800E560A0E0F56FA
:102A1000040ED45D08E1340ED86F080ED96FA00EF5
:102A20000E6E0F0E0F6E300E13ECC4F00AEF12F0A4
:102A3000320EE66E730E22EFB7F0640E28EFB7F099
:102A400002ECC1F06BECB7F01CE0CFECB7F019E191
:102A50000701585116E119ECBEF013E1195111E1CB
:102A600001013B51800B03E1050ED45D0AE1080E24
:102A70004BECB8F0DF6E01013BAF03D0010EDF1469
:102A800001D0000ED2ECBEF002E2E16AE552E16E46
:102A90004950B5EFB6F001013B51800B06E06BECFD
:102AA000B7F003E0CFECB7F001E0000C010C53C12C
:102AB000E6FFF1DF000903E001016E5101D0000ED5
:102AC000E66E340ED3ECB6F06FC1E6FF350E22EFA2
:102AD000B7F0650E28EFB7F02050400B06E001017B
:102AE000E551040B02E1E58501D81200E6ECC0F0E7
:102AF00054C1DFFF11ECBEF002E158C1DFFF1DEC55
:102B0000BEF004E02150020B01E1DF6A080EDF0293
:102B1000F350E66E750E22ECB7F0E552B5EFB6F065
:102B20000701B2510C0803E3B3510C0805E2B26B84
:102B30000C0EB36F0A01DA931200016A0D0E015CEC
:102B400007E073ECBBF002E001501200012AF6D757
:102B5000000C0C0E016E015007E073ECBBF002E0BC
:102B6000015012000106F7D7000C0701B06BB16BE2
:102B7000D7DFB2C701F00701B351D880015409E390
:102B80006FEC04F0F3500701B013F450B113012AB5
:102B9000F2D71200016AFEECBCF00BE0ECECC1F0E5
:102BA00006E249500508000E4A5401E2012A420E8D
:102BB0000DD084ECC0F014E0ECECC1F006E249501A
:102BC0001408000E4A5401E2012A440E0124E66E64
:102BD0002BEC04F0E552F3CFB0F7F4CFB1F71200CD
:102BE000ECECC1F014E249504608000E4A540FE2E2
:102BF0000701F40EB06FB169ABECBAF001E1AFD0F0
:102C00000701B26B0C0EB36F0A01DA83A8D0006A19
:102C1000D751D3ECB7F006E249500D08000E4A54E4
:102C200001E2002AD751D3ECB7F006E2495013086D
:102C3000000E4A5401E2002AD751180801E2002A86
:102C4000D751190801E2002AD751D3ECB7F006E2B8
:102C500049501F08000E4A5401E2002AD751D3EC14
:102C6000B7F006E249502508000E4A5401E2002A56
:102C70000101D45103E0030ED45D1CE1ECECC1F082
:102C800006E249500508000E4A5401E2012A74EC9C
:102C9000C6F006E249500A08000E4A5401E2012A31
:102CA00074ECC6F022E249501308000E4A541DE2AB
:102CB000012A1BD0ECECC1F006E249501E08000EC0
:102CC0004A5401E2012A74ECC6F006E24950280891
:102CD000000E4A5401E2012A74ECC6F006E24950A3
:102CE0003208000E4A5401E2012A260E4C6E9C0E58
:102CF0004D6E010E4E6E00504F6E506A516A030EBB
:102D0000D8904F3650365136E806FAE1BEECBCF0AA
:102D10000150526E536A546AD89052365336543624
:102D2000AFECBAF00900F5CFB0F70A00F5CFB1F774
:102D3000FAECBCF005E00701B085B189B09DB19B0C
:102D4000030E0A01D45D02E0D45109E1F6DE070169
:102D5000B26FFFDE0701B36F0A01DA83E1DE0A0119
:102D6000D40514E10701B305056E0A0EB35D01E257
:102D70000506E3DE0701B26F0550D880B25502E2C6
:102D800005C0B2F7F2DE0A01DA831200020ED45D4A
:102D900012E10701B229056EB251020801E2052ACB
:102DA000D8DE0701B36F0550B35D02E205C0B3F78B
:102DB000DCDE0A01DA8312001E0E006E0101D4511E
:102DC00004E13CECBAF03E500AD0B6ECBCF002E0B4
:102DD000140E05D021ECBAF003E065ECC3F0006EF0
:102DE0000A01D651FE0BE842056E1200050E00ECFA
:102DF000B8F0050E0A01D803F350006E0101012B53
:102E00008BECBBF01B8F1200080E00ECB8F00A012F
:102E1000D951F3ECC3F01AECC4F01B8F1200C4ECD0
:102E2000BBF021ECBEF03B51200B06E1EEECBCF018
:102E300003E001011E0EAC6FB6EC5AF086ECBAF05E
:102E4000300E0101195D02E1200E196F1B8F016B1D
:102E50002A0E006E23886BEF21F00101D45102E1AC
:102E600029510BD0030ED45D11E1030E0A5C02E17F
:102E7000640E03D00A5004E1960E0E6E0F6A120023
:102E8000240E2E251AECB8F00E6E0F6A120094DF95
:102E90000701BAAF13D00050F3ECC3F0DEDF0A0134
:102EA000D751190804E2190ED75DC6ECB8F0190E17
:102EB000D75D18E2DAECBEF00CEFBFF00A01D75193
:102EC000190803E2190ED75D0026190ED75D03E23B
:102ED000DAECBEF0005E0050F3ECC3F0190ED75DE3
:102EE00001E1BBDF1200570E00ECB8F07CECC0F043
:102EF00006E1EEECBCF003E001011E0EAC6FC7DF93
:102F0000FAECBCF00BE00101410E166F500E176F8A
:102F10000301B8510F6AE8307F0B0E6E1AECC4F053
:102F2000FAECBCF009E00101460E186F2951E824C3
:102F30000301B85D07E103D090ECC0F003E10101AB
:102F40002A0E196F01011B8F12000A01D45102E1F0
:102F500066DF0AD0D40502E149DF06D0020ED45D57
:102F600002E152DF01D0BFDF21ECBEF03B51200B6C
:102F700006E1EEECBCF003E001011E0EAC6F1200A6
:102F8000B9ECB6F0070EE126E4EC0DF00A01D65DCF
:102F900004E2E4EC0DF00A01D66FFCEC0DF00A013E
:102FA000D880D65504E2FCEC0DF00A01D66F2DEC6A
:102FB0000EF0000903E00A01190ED76FFDDE90EC58
:102FC000C0F004E3190ED75D002603D0DAECBEF0A2
:102FD00005260550005C03E30550005E0AD0006A38
:102FE000D40507E1DC51D75D04E2DCCAD7FADDCABB
:102FF000D6FA00C0D8FAE0DE0550002690ECC0F00A
:1030000004E3190ED75D002609D0DAECBEF0056E98
:103010000550D880005402E20550005EF6ECC3F083
:103020000BE249505408000E4A5406E2540E006E5A
:10303000DCCAD7FADDCAD6FA00C0D9FA00C0C1F797
:10304000190ED75D03E3190ED75D03D0190ED88092
:10305000D7550701AE6FAF6BBAAF02D00A0E01D0E1
:10306000320EAF03F3CFAFF7AE03F3CFAEF7F450AA
:10307000AF27FE0EDB5004E02050800B01E165DF3E
:103080003450040B0DE10A01DA51020B09E0FEECA9
:10309000BCF006E184ECC0F003E1FAECBCF003E024
:1030A00079DD349401D061DD0701070EAC6FDF508C
:1030B0000A01D55D05E0D5CADFFFA3ECD3F0248A71
:1030C0001EAC03D00201098902D00201068B050162
:1030D000478527EC33F0070EE15C02E2E16AE55236
:1030E000E16EB5EFB6F0006A800E066E056E055013
:1030F0000502F350015CF4500258D8B008D000C06B
:1031000005F006420650051206BE09D0F0D705C0EC
:1031100000F006420650051206BE01D0E8D700D0E6
:103120001200B9ECB6F02A8448C102F009ECB8F0FC
:103130003DE05A0E025E010EE66E48EC10F0E552DC
:10314000016E02504B0817E24B0E025C036E060E36
:103150004A6E4AC043F001C03EF06FECE5F03EC05D
:1031600049F049C043F003C03EF06FECE5F03EC0CB
:1031700003F00350015E0F0E015C02E20F0E016EC0
:103180000150300802E2300E016E01C0BDF702505E
:103190000A0DBFECB7F001508EECC1F03D50026E4D
:1031A00023B604D00250E8240201D96FFBECBFF033
:1031B0000701BC6FFE0EDB50020801E18BD0BCC7DB
:1031C00001F00101E6A502D0040E016E01504B6E24
:1031D0004C6A0250DFECB9F0030ED8900E360F3671
:1031E000E806FBE111ECBFF00A0E4F6E4FC043F052
:1031F0000BC23EF0EFECC3F04D6E4E6A00504B6ECA
:103200004C6A800E3D6E3E6A46ECC6F01DECC6F080
:103210004BECC6F04DC042F04EC043F05FECBAF04C
:10322000036AF7DA016E1C50040B2FE0010403E07F
:10323000020E015C2AE13450400B27E1FE0EDB5008
:1032400024E001C202F0025020E0025074ECB7F01A
:1032500002E600ECC0F019E20250FE0BE842D88012
:10326000005413E20250E824005C0FE2FE0EDB047F
:1032700006E10C0E02010027000E012305D00C0E02
:103280000201005F000E015B032A03500EE1880E6D
:10329000D8800E54130E0F5404E2880E0E6E130ED7
:1032A0000F6E0EC000F20FC001F22450020B06E1B7
:1032B0002250400B03E03150800B0AE0036A006AA1
:1032C00031AE06D0000E0201026F036B006F016B7E
:1032D00011EC0AF0B5EFB6F0B9ECB6F0DFECB8F0EF
:1032E0002FECC1F02AEC13F0B7ECC5F0B5EFB6F057
:1032F000B9ECB6F06AECC3F0770EC3ECBDF0FE0E8D
:10330000DB5003E0100EC3ECBDF0B5EFB6F019ECE6
:10331000BAF0050E005C09E0DEECBEF006E19BECC5
:1033200009F0000902E1000E01D0010E000902E0DF
:10333000000E03D001013451E824E66E3C0E22EF6A
:10334000B7F0E5DF0201A85103E00101345106E0C6
:103350000201A85105E10101345102E0A8EC14F08A
:103360002A8412002AECC2F003E00101285101D0A6
:10337000000EDF6E21B202D0DF9EDF46DFCFE6FF18
:10338000760E22ECB7F0D890DF32D890DF32DF50E3
:1033900005E1FE0EDB5002E0010EDF6EDFCFE6FF3F
:1033A000790E22ECB7F0E552B5EFB6F0B9ECB6F015
:1033B000016A080E015C16E2FE0EDB50012405ECEA
:1033C000C0F0026E100E025C040DF350006E8AEC29
:1033D000B8F001E1006ABFECC5F0005028ECB7F08E
:1033E000012AE7D7140EDDECB6F0B5EFB6F094EC99
:1033F000C0F00CE0220E28ECB7F00101D45102E13C
:10340000180E01D0080EE66ED1DFE5520AEF12F079
:1034100094ECC0F00DE0310E28ECB7F0B7EC09F0F9
:10342000000902E0100E01D0000EE66EBFDFE5528B
:103430000AEF12F098ECC0F002E1F7EF19F008EF94
:103440001AF0020199510101625D18E062C199F21E
:103450006251020B05E1D051200B02E1000E01D0B8
:10346000010E000902E0000E01D0380EE66E0F0ECC
:10347000E66EC80EE66EA10EC0ECB8F01200D5ECF8
:10348000B9F0820E28ECB7F02A9269EC13F0E66AE4
:10349000720E22ECB7F03C0EE66E710E22ECB7F025
:1034A000B9EC13F069EC15F066EC0AF044EC07F0A7
:1034B000B6D85BECC2F0E66A130E22ECB7F001015D
:1034C00062855C95BEDFDDEC45F0E668B30E22EC6C
:1034D000B7F03DD88FEC45F0FEEC46F00DEC07F070
:1034E000B3EC12F0A0EC12F056EC12F076EC15F002
:1034F0008FDFDAECB8F00BDF7EEC12F057EC15F052
:10350000010EE66EF5DEE552D5ECB9F00601B26BC0
:10351000090EB36F6CDF01015F51200B02E0640EF6
:1035200001D0320EE66E1F0E22ECB7F0010EE66EF1
:103530000F0E22EFB7F01200046A01015FAF04D052
:1035400011BC048011BE04823CB904841200010144
:1035500012983B51100B01E012883B51100B0FE009
:103560002150020B0CE01E50200B09E0050ED45D2B
:1035700006E0040ED45D03E0030E006E06D031C1F8
:1035800000F0DEECBEF001E0006A0050E66EA60E30
:1035900022EFB7F0016A0701BAB302D04BC101F0C4
:1035A0004CC102F0BA51020B09E00101D45104E10F
:1035B0000601EA51010802E34DC102F00F0E0101BC
:1035C000D8804155E66E8BECC5F07DC1E6FF47C162
:1035D000E6FFA00EE66E3BEC13F00DECC5F070C1FB
:1035E000E6FF6E0E22ECB7F00701BAB10FD0010171
:1035F000D2AD03D0D29D8FEC45F01450100B06E0F5
:103600001450200B03E11498FEEC46F00701BA5168
:10361000010B02E0AE0E01D0AD0E28EFB7F0CAEFFD
:103620001AF0E6ECC0F019ECBAF0000403E0020E68
:10363000005C09E1E66A3350040B02E0030E01D09E
:10364000000EE66E2BD0005005E1010EE66E50DE56
:10365000E55222D0030E005C1FE1CFECB7F01CE076
:10366000020E0A5C03E153ECBDF00FD00AECC0F08F
:10367000DFECB8F03E0ED3ECB6F0DF6A010196AB9A
:10368000DF2ADFCFE6FF020EE66E140ED3ECB6F0B3
:103690000501040E266F05D0E66AE66A140ED3EC27
:1036A000B6F0E552B5EFB6F0E6ECC0F002012F6BD4
:1036B0000601BF6BBFC6BEF6329E0101D45124E1A4
:1036C0000601EA51010803E31350010B17E0016AF8
:1036D000EA05EB6F020EEA5D03E302011A5102E014
:1036E0000601EB6BEBC6E6FF11ECC2F0E66A030ED7
:1036F000E66E120ED3ECB6F0328E04D05BECC2F064
:103700000601EB6B8CDF5BD0030ED45D56E1629952
:103710001350010B06E1FEECBCF003E19CECC0F0A1
:1037200048E021ECBAF00AE02D0EDF6E010E016ECA
:10373000026A13A015D002012F6F12D0B6ECBCF0B4
:103740000DE0020E016E026A1F0EDF6E010196BBD4
:1037500007D0010E026E3F0EDF6E02D0016A026AD0
:103760008BECC5F0120ED3ECB6F0EDC6E6FF11EC13
:10377000C2F0328EFEECBCF002E00101628907016A
:10378000200E4F6F3F0EDF5C02E1100E4F6F640E94
:10379000DF5C02E10A0E4F6F4B0EDF5C02E10D0EA3
:1037A0004F6F2D0EDF5C02E1160E4F6F4C6B506BAE
:1037B00002D05BECC2F045DE02D05BECC2F0B5ECAF
:1037C00032F0E552B5EFB6F0BF0E6CECC6F0E84053
:1037D000E8403F0B005C02010B6F060E00C0E7FFE4
:1037E000070B04E0E742E79EE806FCE1E750020130
:1037F0000B5F0B07640E0B5D09E22150100B06E115
:103800000101395103E1218805ECC5F00BC200F03C
:1038100012001FB203D00101D45112000101D55191
:10382000120002ECC1F02D50100B01E0010EDE6E13
:10383000DD6A2D980C0E28ECB7F019ECB9F00E6E7D
:103840000F6AFF0E0E1804E10F5002E10E680F68B8
:10385000DF502D98E8B02D88020EE15C02E2E16AAB
:10386000E552E16EB5EFB6F03F6B406B416B426BDA
:10387000400E436FD8903A373937383737373637B5
:103880003537343733374237413740373F373E518A
:10389000425D3D5141593C5140593B513F5909E32B
:1038A0003E51425F3D51415B3C51405B3B513F5B70
:1038B0003A2B432FE0D712000101D09711BED087D9
:1038C000D19911BCD189120059ECBDF001010490CD
:1038D000D051080B01E004800492D151100B01E09B
:1038E0000482119E04B0118E119C04B2118C070148
:1038F000089F04A007D00101D0510701089F020BC7
:1039000001E0088F089D04B2088D66ECB2F09CEFD0
:103910001AF0E6ECC0F087ECC4F0200EF9ECC3F02E
:103920000050026E0F0EF9ECC3F001012B51005C48
:103930001FE1250E025C1CE1050E2CECC3F08AECA5
:10394000B8F013E2010EE66E0A0EDF24F5ECC5F0C6
:103950002BECB7F00F0E01010617D451065D05E000
:10396000288206C1D4F14AECB9F0096A010E02D0EE
:10397000096A000EE552B5EFB6F0B9ECB6F01EAC30
:1039800003D00201098102D00201068305014781AB
:1039900047872B8C2C8A47ECB8F0EE50ED1013E0E3
:1039A0000101442B640E445D03E2B3DF00091DE115
:1039B00001014407FF0E445D03E0ABDF0009F8E1BD
:1039C0000101442B12D001014407FF0E445D03E0C6
:1039D000A0DF00090AE10101442B640E445D03E20B
:1039E00098DF0009F8E101014407B5EFB6F0B9EC42
:1039F000B6F02C0E496E970E4A6E010E24ECC6F0FE
:103A00007F0B006EFE0EDB50040806E1FD0EDB505E
:103A1000310802E2020E006EA0ECC0F006E1FD0EDD
:103A2000DB50310802E2040E006EB5EFB6F0040E72
:103A30000101435D01E3436B395102E0190E04D0EB
:103A4000160E43251AECB8F0006E0050E66EE66ADA
:103A50003C0EE66EF5ECE2F007EFC1F021900201BA
:103A6000320E246F295102E0140E246FC80E366FF7
:103A70001DAC2998DD5102E00DEC07F01D50400B04
:103A800003E02A50800B02E169EC13F00201098780
:103A90000985098309817A6B0901EB6B1200B9EC86
:103AA000B6F0FE0EDB500EE029A006D0FE0EDB5075
:103AB000030B02E11CEC06F0280E35ECBBF0FE0E09
:103AC000DB06EFD7B5EFB6F011C512F50501106BA7
:103AD000279C0101E491120027BA09D013C549F1CE
:103AE00014C529F1249223BC2482ADEC5BF0278A13
:103AF000010136990DEC07F00201216B239A259202
:103B0000120012ECC5F0E0DF2750200B05E0CFECEF
:103B1000B7F002E0080E076EDFDF2F98120027AA29
:103B200002D00101E88B0750220A01E19ED1030A6D
:103B300001E17FD1010A01E1EFD03F0A39E0010A3A
:103B400001E0ADD1278C49C113F529C114F5239C9F
:103B500024B2238C27BA15D0010136AD11D0E7B7B6
:103B600006D03651070B050DF3500A0F496F640E4E
:103B7000296F36B902D0430E296F98EC5BF001D063
:103B8000C0DF9CECC0F007E0200E06014A5D03E0B8
:103B9000200EACECB9F01D901F0E076E02012D51E6
:103BA00001E17ED12750200B01E17AD1076A23D1B0
:103BB0000501105101E188D0CFECB7F016E0275095
:103BC000200B13E00501235107E1020E265D0DE1F4
:103BD000A2EC0CF0000909E102012D5101E12D2BAD
:103BE000080E076E1F0E086E120005011007125115
:103BF000EA6A000FE96E080EEA22EFCF02F7122BF5
:103C0000125174ECB7F002E6E2ECBFF001E3126B84
:103C1000CFECB7F00BE02750200B08E002C7E6FF1F
:103C200062EC35F0E552200E076E12003C0E0701E3
:103C3000025D04E12482238C229C32D13E0E025D7F
:103C400006E12492239C1EBC2BD1228C29D1740E18
:103C5000025D01E125D10601EA510AE02750200B5F
:103C600007E0298A02C7E6FF57EC65F0E552299A7A
:103C7000800E0701025D0FE2180E496E9B0E4A6E20
:103C8000010E4B6E200E025DBDECB9F0BEECB6F03D
:103C90000800F5CF02F7800E025D03E10201040E79
:103CA000526F07010251800805E2800E025DFD0F90
:103CB0000201526F800E0701025D01E3B4D0025190
:103CC00001E1EED0200ECFD027AAE9D0C8ECBDF09C
:103CD00007E007010251800803E3200EACECB9F0C5
:103CE00010DFCFECB7F005E0279C080E076E100E32
:103CF000086E2750200B01E1D3D00201555101E19C
:103D0000CFD0189A55BF188A196B010EE66E7F0E38
:103D1000551548ECBEF0C4D01750800B06E0275074
:103D2000200B09E10B0E155C06E01D50040B03E0AF
:103D30001D50080B58E12750200B09E01750800B4D
:103D400006E025ECBEF003E00B0E155C1CE10AEC6E
:103D50005CF0D7DE209427AAA3D0CFECB7F003E025
:103D60000201010E2D6FCFECBFF00601EA5101E117
:103D700097D007010251800801E292D02F88200ECF
:103D8000ACECB9F08DD0230E155C10E1010EE66E9F
:103D9000B3EC0CF0E5521EAC03D00201098702D04F
:103DA000020106810501478D179E7AD091EC87F0BC
:103DB000000914E02750200B11E00C50006E020E99
:103DC00081ECBCF00C50026E00500C6E0250E66E9E
:103DD000EDEC69F0E5520201196B62D027AA60D0C0
:103DE000F2EC89F05DD0CFECB7F008E02750200B63
:103DF00005E0080E076E1F0E086E52D0FE0E07017A
:103E000002150EE0228E010E016F02A102D0030EF8
:103E1000016F02910243210E076E0501200E07D0AB
:103E20000201020E526F220E076E05011F0E156F62
:103E300037D00701015112E001072380C3EC5BF08A
:103E4000076A1DA006D0020E076E27BA02D03FEC0B
:103E5000BBF0210E086E1D80229E22D00201010EB1
:103E6000526F228E220E076E1BD00201525114E0B7
:103E700023905207C3EC5BF0030E076E1DB007D012
:103E8000070E076E27BA03D0006AC3EC6AF0220E51
:103E9000086E229E1D9004D015C507F001D031DEBA
:103EA0000101E89B1200020171510101D8804855BF
:103EB00002E271C248F12B5109080EE2100E2B5D8F
:103EC0009FECB8F0060E77ECC6F0016E0150D8807A
:103ED000485502E201C048F1395117E102010B5186
:103EE00074ECB7F002E600ECC0F006E201014851C4
:103EF000640802E2640E486F640E02010B5D05E285
:103F0000A4ECC0F002E2320E486F2150100B05E025
:103F1000A4ECC0F002E2320E486F01015F9399EF0A
:103F2000B2F0DACFE4FFE2CFDAFFE9CFE4FFEACF85
:103F3000E4FFE652FC0EB36EF30EB26E02011107FF
:103F40000201115105E10201320E116F01012181BF
:103F50000101E7A92CD00601FD07000EFE5B06015A
:103F6000FD51FE1124E1F29EF26AF06AB96A9D6A7F
:103F7000000EA66EA16E9E6E8D8C8D8A8C908494A0
:103F8000070E936E0000000000008A9A00000000F7
:103F900000000000270E936E4E0E996E0000000088
:103FA000000003000000000000000000FF001E8071
:103FB0001D861D8481B20BD001014FA302D01E903B
:103FC00006D001014FA102D01D9601D01D9481B4ED
:103FD0000BD001014FA302D01E9006D001014FA1CA
:103FE00002D01D9401D01D9687B60BD001014FABB6
:103FF00002D01E9006D001014FA902D01D9601D01B
:104000001D9481B00BD001014FAB02D01E9006D0A1
:1040100001014FA902D01D9401D01D960201120783
:104020000201125137E10201050E126F0101B05178
:1040300016E00101B007020102015151020B05E037
:104040001D50040B02E10201518102010201515194
:10405000080B05E01D50080B02E10201518501012A
:10406000B15106E0FF0E0101B15D02E00101B12B8B
:104070001FAE04D00601DE2B000EDF2307014E51D8
:1040800009E007014E0707014E5104E14FC74EF703
:10409000010121830101AF5102E00101AF070101DC
:1040A000269701012695010126A102D0010126854E
:1040B000010126A302D001012687010126930101F7
:1040C000269188A202D00101268188A002D0010198
:1040D00026830F0E010126150101236F01012351D3
:1040E000EA6AC50FE96E060EEA22EFCF22F1010E51
:1040F0000101221515E01F50080B05E00101010127
:104100003B51010B0DE12050200B0AE0010122AFD1
:1041100003D00101240702D00101242B24B03382F3
:104120009EAA11D00701922B07019151912BEA6AA7
:10413000000FE96E0C0EEA22AECFEFFF070192519D
:1041400002E190C791F7A19207014407E552E5CF3C
:10415000EAFFE5CFE9FFE5CFDAFF110001013BAB54
:1041600007D03B9B238A0601425102E0426B436B1E
:1041700012000701BAB103D0119A119812001198D8
:10418000BAA31188119ABAB3118A12000B0E00EC6F
:10419000B8F0258E12006BECB7F003E0CFECB7F06F
:1041A00006E01394010156A30ED013840CD013948F
:1041B00002013D5107E10101E651800B03E13B5152
:1041C000040B01E01384139613A413861398135061
:1041D000040B04E109ECB8F001E013881200ECC113
:1041E000E9FFEDC1EAFFEECF49F0EECF4AF0EECFA6
:1041F0004BF0EECF4CF0EFCF4DF0EAC1E9FFEBC151
:10420000EAFF49C0EEFF4AC0EEFF4BC0EEFF4CC0D4
:10421000EEFF4DC0EEFF1200B9ECB6F0B9ECBAF00B
:10422000FB0EDBCFECF1FC0EDBCFEDF10101A30EB9
:10423000EA6F010EEB6FD3DF9CEC2CF0D8A002D01C
:10424000010E01D0000EB5EFB6F002ECC1F0005047
:10425000E66E2BECE5F0E552140EE66E8AECE5F026
:10426000E5529FECE5F09AECE5F00009FCE1C45062
:10427000006E0050F80812E2C20410E0050EC25CA5
:104280000DE0090EC25C0AE00D0EC25C07E0110EE3
:10429000C25C04E0390EC25C01E00006020EE15C83
:1042A00002E2E16AE552E16EB5EFB6F0E6ECC0F08D
:1042B0000050DF6EEE0E496E8E0E4A6E010E8EECD1
:1042C000C2F00150006E009ED8ECD5F001AEF2D7DE
:1042D000E552B5EFB6F0E6ECC0F00050DF6E2350CB
:1042E000100B1DE10050E66E75EC04F0E552800BFA
:1042F00016E0180EDF5C08E10101200E166F500E6B
:10430000176F410E186F07D00101450E166F520E40
:10431000186F18C117F1200E196F040E016F2A884B
:1043200023A808D0EA0E496E900E4A6E010E8EEC5C
:10433000C2F007D0DFCFE6FF75EC04F0E552016E66
:10434000DF2A2AA802D0019E2A980150006E009E02
:10435000FBECD5F001AEE4D72398E552B5EFB6F00B
:1043600056ECC2F003E2D6ECBEF004D0FE0EDB50F9
:10437000410FF60F006ED8ECD5F0B5EFB6F056EC65
:10438000C2F003E2D6ECBEF004D0FE0EDB50410FCB
:10439000F60F006EFBECD5F0B5EFB6F017ECC5F0FC
:1043A000DFDFE5527CECBCF0DBDFE552B5EFB6F0C9
:1043B00017ECC5F0E4DFE5527CECBCF0E0DFE55241
:1043C000B5EFB6F0B9ECB6F017ECBFF0020E010194
:1043D00000274DECD5F0DF50006E050E0101005FA7
:1043E0004DECD5F0030E0101005FE552B5EFB6F0DC
:1043F000B9ECB6F017ECBFF0FE0EDB50020F010176
:10440000016F6AECD5F0DF50006EFE0EDBCF01F1DC
:104410006AECD5F0E552B5EFB6F000C059F28CEC7D
:10442000CFF0FF0E005C01E041DF0101B589120011
:1044300000C05AF29CECCFF0FF0E005C01E04BDFB5
:104440000101B58B12008CECCFF0FF0E005C01E097
:104450002DDF0101B58D640EAC6F249612009CEC2B
:10446000CFF0FF0E005C01E036DF0101B58F640E76
:10447000AC6F24961200B9ECB6F0C4ECBBF095EC2E
:10448000B8F050ECB7F0B5EFB6F0B9ECB6F0C4EC5C
:10449000BBF02FECC1F0010EE66E9EEC06F0E5528B
:1044A000E552B5EFB6F0B9ECB6F004EC65F00101F9
:1044B000190EAE6FFC0EDBCFB2F1FD0EDBCFB3F108
:1044C000FE0EDBCFB4F1B5EFB6F0830E096EE00E51
:1044D00070ECC6F0800E005C08E204EC65F00101AF
:1044E000190EAE6F0201E00EA96F1200CBECC5F001
:1044F000DBCF4AF0800E4A1407E0D3ECB8F0496CE9
:104500004A1E000E4A2202D0D3ECB8F0F3ECC4F0FD
:10451000B5EFB6F0B9ECB6F012A60FD0060150B563
:1045200003D0010150ECBEF0288ABCBF289AFE0ED1
:10453000DB5001E0287AB6EC39F0B5EFB6F0CBEC01
:10454000C5F0DBAE08D0DB50FF0DFE0EF3CFDBFF76
:1045500012ECBDF007D012ECBDF0DB50FF0DFE0EEB
:10456000F3CFDBFFDB50B5EFB6F0E6ECC0F00701B0
:10457000585101E05DD11D50400B01E059D132503E
:10458000040B01E154D10101D45104E18450020B28
:1045900001E14DD10B0E4BECB8F00601BC6F21ECE4
:1045A000BAF001E0A5D0140E0601E76EBC19E8AE22
:1045B00002D0BC3503D0E750D880BC5502E2140EBF
:1045C000BC6FEC0EE76EBC19E8AE02D0E73402D047
:1045D000E750BC5D02E2EC0EBC6FBE51E76EBC1949
:1045E000E8AE02D0BC3503D0E750D880BC5502E21B
:1045F000BE2B0BD0BE51E76EBC19E8AE02D0E7343B
:1046000002D0E750BC5D03E2BE07BEC6BCF6200E7A
:10461000496E4A6AC1C63DF0C2C63EF01EECBFF00C
:104620003DC0C0F6C0C649F04A6A49BE4A68495012
:104630000601C15F4A50C25BBCC649F04A6A49BE26
:104640004A684950C1274A50C223C0C6E6FF77DFF7
:10465000E552016E010EE66E0E0E012425ECB9F056
:1046600002011A5101E1E3D01BAA05D0BCC6E6FF46
:104670001CEC6BF0E5523FECB9F02AE01250080B4D
:1046800003E1040E1A1528E03CECC2F001E0010E33
:10469000496ED45103E1D051400B07E0D45103E0FF
:1046A000CF51040B02E0000E01D0010E491809E0C1
:1046B00012A602D0E66A09D00601BC5101012427E6
:1046C0000BD012A605D0010EE66E24DFE55204D011
:1046D0000601BC510101245F0601BC5101E0A7D0D5
:1046E00002011A51320801E3A2D0320E1A6F9FD094
:1046F0001B0EE66EEEEC11F0E552F3CFBCF6F4CFF4
:10470000BDF6026A016A0601BC51E76EBD19E8AE4A
:1047100002D0BD3503D0E750D880BD5505E2BC516D
:10472000BD5DD5ECBBF0026E0601BD51E76EBC1954
:10473000E8AE02D0BC3503D0E750D880BC5505E2C6
:10474000BD51BC5DD5ECBBF0016E0601BF51D880F8
:10475000025402E202C0BFF6BE51D880015402E208
:1047600001C0BEF6000EE76EBF19E8AE02D0BF353D
:1047700003D0E750D880BF5505E2010EE66E0D0E5E
:1047800025ECB9F0010E0601E76EBF19E8AE02D0C4
:10479000BF3503D0E750D880BF5505E2010EE66E65
:1047A0000C0E25ECB9F0020E0601E76EBF19E8AE5B
:1047B00002D0BF3503D0E750D880BF5505E2010EC7
:1047C000E66E0B0E25ECB9F0000E0601E76EBE1981
:1047D000E8AE02D0BE3503D0E750D880BE5505E222
:1047E000010EE66E0F0E25ECB9F0010E0601E76E24
:1047F000BE19E8AE02D0BE3503D0E750D880BE5512
:1048000005E2010EE66E100E25ECB9F0020E06016F
:10481000E76EBE19E8AE02D0BE3503D0E750D880AF
:10482000BE5505E2010EE66E110E25ECB9F032948C
:10483000E552B5EFB6F002ECC1F0FC0EDB506AE1D8
:1048400002012A5167E10490FE0EDB50140804E2D5
:10485000140E42ECBBF00480FE0EDBCF49F0565143
:10486000D880495403E2FE0EDBCF56F201012A51F3
:10487000100B03E0050ED45D05E10450010B02E0CE
:10488000FE0EDB2A010E67C1DBFF050ED45D02E1DF
:10489000010EDB6A010EDB50280803E2DE52280E0F
:1048A000DD6E050EC8ECBCF03EC0DBFFDF6A150E06
:1048B000DF5C22E2006AFE0EDB5004E0FE0EDB50FD
:1048C000DF5C13E301012A51100B07E0050ED45DF4
:1048D00004E002015651DF5C08E001016751040861
:1048E00006E2010EDB50DF5C02E1010E006E0050BB
:1048F00017ECBBF0DF2ADBD71350010B69E0020194
:10490000215166E10101D45103E0030ED45D60E161
:1049100032845ED0FC0EDB0430E102012A5106E055
:10492000FD0EDB5003E12250400B55E1A0ECC0F03E
:1049300003E2080E42ECBBF0FD0EDB500C0805E272
:104940000C0EF36EFD0EF3CFDBFFC6ECBAF0150EC6
:10495000DF5C3EE2FE0EDB5004E0FE0EDB50DF5C6F
:1049600007E3090EDF5C07E3FD0EDB50DF5C03E2CB
:10497000010E17ECBBF0DF2AEAD7FC0EDB50020871
:1049800027E1A0ECC0F003E2080E42ECBBF0FD0E04
:10499000DB500C0805E20B0EF36EFD0EF3CFDBFFD0
:1049A000C6ECBAF0150EDF5C13E2FE0EDB5004E03D
:1049B000FE0EDB50DF5C07E3090EDF5C07E3FD0E54
:1049C000DB50DF5C03E2010E17ECBBF0DF2AEAD715
:1049D000FE0EDBCF0AF2020EE15C02E2E16AE55272
:1049E000E16EB5EFB6F00101D5511EECBBF0B4ECB1
:1049F000C2F00150080D4950F3240A01DF6F4A50FC
:104A0000F420E06F12000101C951C45D0CE1CA51EC
:104A1000C55D09E1CB51C65D06E1CC51C75D03E13F
:104A2000CD51C85D01E0000C010C0101D551D45DF0
:104A300001E0000CD4510BE1D051400B01E0010E1C
:104A4000496EDD51400B01E0010E495C2DE0030E83
:104A5000D45D23E1DC51F2ECB7F00A5C1EE121ECFD
:104A6000BAF00CE00101D051040B01E0010E4A6ED6
:104A7000DD51040B01E0010E4A5C16E021ECBAF0B6
:104A80000CE10101CF51040B01E0010E4B6EDC5132
:104A9000040B01E0010E4B5C07E00101D45103E07F
:104AA000030ED45D01E1000C010CADDF000903E051
:104AB000BCDF000901E1000C010CF7DF00092EE06A
:104AC000ABECBAF001E1010CD5511EECBBF08EEC61
:104AD000C5F08DECC4F0015060ECC3F0D451100D62
:104AE000F3CF4FF0F4CF50F02A0E4F260A0E50228B
:104AF0000701AD51080D4F50F3244D6E5050F42076
:104B00004E6E4DC0E6FF4EC0E6FFA7ECE1F0516EE1
:104B1000060EE15E5150000901E1010C000C1AB2D1
:104B200002D0DDECBBF0D4C1D5F134AA17D001011D
:104B300038A306D0DE93D1B3DE83DE95D1B5DE8512
:104B4000DD9DD0BDDD8DDD95D0B5DD85DC95CFB5A6
:104B5000DC8592ECC5F018ECC2F01AD00101D551F9
:104B600003E1DD9DD0BDDD8D030ED55D11E192EC3D
:104B7000C5F018ECC2F021ECBAF006E00101DD95B9
:104B8000D0A506D0DD8504D00101DC95CFB5DC854C
:104B900034AA0DD0500EE66EE66A2A0EE66E0A0EB4
:104BA000E66E7A0EE66E0A0EC1ECB9F00ED0050E76
:104BB000D45D0BE0100EE66EE66AD451100DCDEC1C
:104BC000C1F08DECC4F093ECC4F0050E0101D55D8D
:104BD00008E0D551EA6ACF0FE96E0A0EEA22ADC7A6
:104BE000EFFF1200C9C1C4F1CAC1C5F1CBC1C6F102
:104BF000CCC1C7F1CDC1C8F1D5C1D4F134AA08D018
:104C000058ECBEF02A0EE66E0A0EC1ECB9F00FD0D9
:104C1000ABECBAF00CE0100EE66EE66AB4ECC2F053
:104C200004ECB8F0D45103ECC4F093ECC4F0ABEC5A
:104C3000BAF004E038ECBCF0ADC7EFFF1200B9ECFD
:104C4000B6F03BDF000916E1C0EC10F0FE0EDB50C1
:104C500002E165DF01D0C6DFCDECBDF0248A1EACD9
:104C600004D002010983098102D0020106830501F3
:104C700047834781B5EFB6F0C0EC10F00101C45195
:104C80000CE0C40503E13C0EC55D07E3C95105E036
:104C9000C90514E13C0ECA5D11E235ECB9F0348A65
:104CA00010D8349A6DEC10F01C8A35ECB9F01C9ACF
:104CB000188447ECBBF018945FEFBDF002D86DEF9D
:104CC00010F00DC103F0C9C19AF2CAC19BF2CBC169
:104CD0009CF2CCC19DF2CDC19EF2D5C100F01EEC7C
:104CE000C0F0DEC1E2F134AA08D058ECBEF0540E98
:104CF000E66E060EC1ECB9F011D0050E005C0EE0B8
:104D0000100EE66EE66A0101B4ECC2F004ECB8F0F5
:104D1000540EE66E060EE66E31ECBCF0016A050E2E
:104D2000005C03E000501EECBBF0F9DE03C00DF1A7
:104D30009AC2C4F19BC2C5F19CC2C6F19DC2C7F123
:104D40009EC2C8F100C0D4F134AA1ED0010138A31C
:104D50000ED0D193E2B3D183D195E2B5D18512962D
:104D6000D1B312861294D1B512846AEC8BF0010192
:104D7000D09DE1BDD08DD095E1B5D085CF95E0B582
:104D8000CF85F6ECC1F018D00101D45103E1D09DDC
:104D9000E1BDD08D030ED45D0FE1F6ECC1F021EC46
:104DA000BAF006E00101D095E1A506D0D08504D087
:104DB0000101CF95E0B5CF8534AA09D0500E21EC82
:104DC000BFF02A0EE66E0A0EC1ECB9F00CD0050E4B
:104DD000005C09E0100E21ECBFF0D451100DCDECB9
:104DE000C1F031ECBCF00701AD6B010138ECBCF057
:104DF000EF6A04903BB104803B913BB33B813B9312
:104E000004B03B83129C3BB1128C129E3BB3128EBA
:104E1000CDECBDF0248A3DDB1EAC06D00201098733
:104E200009850983098102D00201068305014881B1
:104E3000BF0E476F1200B9ECB6F00101628521EC9C
:104E40001AF0B5EFB6F0370E005C02E2370E006ED6
:104E500000509F0802E29F0E006E630E005C08E2A5
:104E6000370E005CE824496E090E97ECB7F005D0C8
:104E7000630E005C9EECC3F0090F006E0201D4517A
:104E800002E0030E00260050150802E2150E006E27
:104E900012002EECC2F00201215110E12050010B52
:104EA0000DE124510BE13250100B08E12750200B8B
:104EB00005E0DC5103E130A003D03090000E68D053
:104EC000FE0EDB5002E0990E01D00A0E4BECB8F05A
:104ED00072ECBCF08C0ED1ECBDF00201D45103E0B9
:104EE000790ED1ECBDF02C5120E1020EDB507EECAE
:104EF000B9F01BE30A0E4BECB8F0496E020EDB5022
:104F0000495C13E311AE11D0119E5CEC1CF0020160
:104F1000068D090E6FECB7F00501478964EC1CF0B3
:104F200066ECB2F00201780E2C6F010EDB50006EC1
:104F300000509F0802E29F0E006E00504B6E4C6ABC
:104F400005011851070D28ECBFF0030E0F0B04E00C
:104F5000C0ECBBF0E806FCE149C018F574DF005076
:104F6000DF6E00C09EF7090E016E01012AB901062D
:104F70001350010B06E00150D880005402E20150AA
:104F8000006EE66AE66A0050E66E8CECBAF0DF501E
:104F9000496E030EE15C02E2E16AE552E16E4950BE
:104FA000B5EFB6F0B9ECB6F0016A0A0E015C19E291
:104FB000FE0EDB50010B06E0230E0124E4ECB8F0FA
:104FC000155C0AE0FE0EDB50020B09E02D0E0124F9
:104FD000E4ECB8F0155C03E101500C6E02D0012A3C
:104FE000E4D7B5EFB6F0B9ECB6F0800E0C6E17AEA4
:104FF00017D0179E1750010B03E11750100B10E04C
:10500000100E0C6E2FECC1F0CDDFE552080E155CD2
:1050100002E1200E0C6E100E155C02E1400E0C6ECB
:10502000B5EFB6F0B9ECB6F0E8ECBBF02FECC1F0A0
:1050300042EC0AF0E552A7ECC3F00101A86FA851B9
:10504000640DBFECB7F0A2ECC3F05C0F1AECB8F043
:10505000006EACECC3F02FECBFF000504B6E4C6A0E
:1050600001014B50495CD86F4C504A58D96F29A662
:105070000BD09E512FECBFF00101D851495C0E6E50
:10508000D9514A580F6E06D09E510F6AD8250E6E20
:10509000D9510F22640E8EECC1F03DC0A8F139C089
:1050A0009EF1B5EFB6F0B9ECB6F0E8ECBBF0DB5032
:1050B0009FECB8F0030E77ECC6F00101A85D02E0AA
:1050C000000E1BD0FE0EDB509FECB8F0020E77EC0A
:1050D000C6F09E5D006E00BE006C040E005C0AE32C
:1050E00020ECC2F009E0945107E0A85105E0190E48
:1050F000005C02E2010E01D0000EB5EFB6F01DEC2F
:10510000BAF0920E49180EE14A500CE1006A0DEC1B
:1051100022F0B20E02ECBDF021860201776B696BC2
:10512000289E072A1DECBAF0930E49185CE14A50FC
:105130005AE1010EE66E57DFE5520A0E0C5C32E2D0
:1051400002017751050833E36951020830E3772BF8
:1051500028BE692B010E016E070E015C13E20128C7
:105160009BECB7F0EF50006E060E015C05E1800E7F
:10517000010115150C10006EFCECC3F000C0EFFF30
:10518000012AEAD70101159F36AD2DD00C5002E15E
:10519000540E02D0300E0C24006E800E001086ECEF
:1051A000BCF010D0200E0C5C12E128AE02D0258E8F
:1051B0001AD0288E0101158FD20E86ECBCF00101A9
:1051C00036AD11D00501930E4B6F1E0E0BD0400E65
:1051D0000C5C04E1980E076E1A8805D0100E0C5C6A
:1051E00002E19A0E076E1DECBAF0980E49186EE1B6
:1051F0004A506CE1010E016E070E015C0DE2FCEC01
:10520000C3F0EF9EFCECC3F0EF500E0803E1FCECA2
:10521000C3F0EF6A012AF0D70FC1A8F10A0E01010D
:105220001003F35011259E6F0A0E1203F35013253D
:105230009F6F0A0E1403F3CFA0F1A26BA2C1A1F1DC
:10524000040E0201775D0DE269510BE112C1A8F174
:105250000A0E01011303F35014259E6FA06BA0C129
:105260009FF10201690508E111C1A8F19FC19EF1FA
:10527000A0C19FF10101A06B020E0201695D0EE168
:1052800010C1A8F10A0E01011103F35012259E6FFF
:105290000A0E1303F35014259F6FA06B9A0E076E2E
:1052A000FFEC0AF0006E00500AE10101A85103E191
:1052B0009E51380802E2258E120043ECBAF000C07D
:1052C0002BF1298447ECBBF02EEC1DF01DECBAF05D
:1052D0009A0E491805E14A5003E1010136ECBFF08E
:1052E000120023ECC0F02582238A12003EC2A7F1EF
:1052F0003FC2A6F140C2A5F10101A46BA36B1FA49C
:1053000002D078EF2CF09CEF2CF004902C50100B76
:1053100001E00480DFECB2F02C50100B01E0010E34
:10532000496E0450010B495C02E04CECBBF01200EA
:105330007BECC6F001018DA715D0FE0EDB5008E016
:10534000FD0EDB5005E1DF68CFA102D0010EDF6E5C
:10535000FE0EDB5007E1FD0EDB5004E0010EDF6EB8
:10536000CFB1DF68DF5021E029ECB8F0A76BA7C10F
:10537000A4F1A7C1A3F11BECC5F001E0010E496E39
:10538000DF0402E0000E01D0010E491802E0B0DA9D
:1053900001D0D2DA7EEC04F01EAC03D00201098108
:1053A00002D00201068305014781E552B5EFB6F050
:1053B0000101A76BA66BA56B02018851E824496E19
:1053C000640E6FECC3F06FECE5F03AC0A4F1320E5E
:1053D000EFECC1F088C23EF06FECE5F03EC0A3F107
:1053E000020189A102D078EF2CF09CEF2CF01FEC89
:1053F000C5F09AC23BF03C6A3D6A3E6A400E406E80
:10540000420E416E0F0E426E436A2EECE3F037C03F
:10541000DEFF38C0DEFF39C0DEFF3AC0DDFFDD52FF
:10542000DD529BC249F04A6A4B6A4C6A100E406ECC
:10543000270E416E426A436A79ECB7F0F6ECB8F099
:105440009CC249F04A6A4B6A4C6A640ED6ECBDF0C5
:1054500079ECB7F0F6ECB8F00A0E02019D03F350B8
:105460009E25496E4A6A4B6A4C6A94ECC2F0DECFC4
:105470003BF0DECF3CF0DECF3DF0DDCF3EF0DD5245
:10548000DD52040EE15C02E2E16AE552E16EB5EF45
:10549000B6F007AE52D02B50400B03E02C50200B3F
:1054A00023E0800E0101C41505E1C4510CE1320E68
:1054B000C55D09E2C46B320EC56FC86BC8C1C7F1C8
:1054C000C8C1C6F111D0100E2B5D0EE2200E006E89
:1054D0000050C45D09E300C0C4F1C86BC8C1C7F186
:1054E000C8C1C6F1C8C1C5F12B50400B03E02C5018
:1054F000200B23E1800E0101C91505E1C9510CE122
:10550000320ECA5D09E2C96B320ECA6FCD6BCDC1D6
:10551000CCF1CDC1CBF111D0100E2B5D0EE2200EDF
:10552000006E0050C95D09E300C0C9F1CD6BCDC16B
:10553000CCF1CDC1CBF1CDC1CAF12B50400B03E072
:105540002C50200B1DE02050400B03E11250080BA3
:105550000FE12050400B12E01F50020B03E11250EC
:10556000040B06E11F50020B09E01250080B06E085
:1055700029ECB8F0BBDEF3ECBBF002D0FEECBBF0E4
:105580002B50400B03E02C50200B16E11F50020B58
:1055900011E01250040B0EE055ECB9F0A7DE9EC1ED
:1055A000BFF19FC1C0F1A0C1C1F1A1C1C2F1A2C1AF
:1055B000C3F102D009ECBCF01F50020B18E102014C
:1055C0008951010B03E18951020B11E0ABECBAF0F8
:1055D00006E02050800B0BE0050E9D5D08E1205099
:1055E000400B05E060ECB9F0E3DEF3ECBBF0010149
:1055F0003BA974D0BAC19AF2BBC19BF2BCC19CF268
:10560000BDC19DF2BEC19EF2F2DE3BC0C4F73CC0FC
:10561000C5F73DC0C6F73EC0C7F7BFC19AF2C0C1CB
:105620009BF2C1C19CF2C2C19DF2C3C19EF2DFDEFA
:105630003BC0C8F73CC0C9F73DC0CAF73EC0CBF776
:105640000701C451C85FC551C95BC651CA5BC75188
:10565000CB5B0101D2A108D0400E0701C8271F0E65
:10566000C923000ECA23CB23049C1E50200B01E04B
:10567000048CD8800701CB51FF0A08E6680EC85D8C
:10568000C50EC959FF0ECA59FF0ECB5919E3CB35C8
:10569000000ECB1909E6D880980EC8553A0EC955A8
:1056A000000ECA55000ECB550BE3C8C70EF0C9C794
:1056B0000FF0DFECB8F0A50ED3ECB6F01E8A01D0E7
:1056C0001E9A0450400B01E0010E496E1E50200B43
:1056D00001E0010E495C02E03AECB9F02BAC95D048
:1056E000800E071401E191D0100E01012B5D01E342
:1056F0008CD02CBA0DD014ECBCF0C9C1A3F1CAC136
:10570000A4F1CBC1A5F1CCC1A6F1CDC1A7F10CD0BC
:1057100060ECB9F0C4C1A3F1C5C1A4F1C6C1A5F143
:10572000C7C1A6F1C8C1A7F143ECBAF02C50200BB9
:105730002DE0005001012B5D29E000C00DF100C0FB
:105740002BF12BC1D3F13DECBFF026ECBBF0056E85
:105750002CAA06D0050EE66E0524DBECBDF005D0C4
:10576000050EE66E05508BECBCF02BECB7F00E0E80
:1057700005248EECB8F00101D29B00BAD28B096AE5
:10578000DBDB20820201010E246F01D0BEDD0701A8
:10579000BE510101C45D04E0DDEC0BF0C4C1BEF7F5
:1057A00001012B5132E12B50080B2FE0020E3A5D24
:1057B0002CE1F1ECC2F004E0CEECBEF0E806FCE136
:1057C0000701C2510E1802E1C3510F181EE0006A12
:1057D0005A0E0E1807E10F5005E1590EC21901E1EA
:1057E000C3510AE0590E0E1808E10F5006E15A0E97
:1057F000C21903E1C35101E1002A0EC0C2F70FC074
:10580000C3F70050E66E02D8E5521200B9ECB6F0CC
:10581000010139516BE12B5169E12B50080B66E016
:10582000FE0EDB5003E1020E3A5D60E1F1ECC2F0E6
:1058300004E0CEECBEF0E806FCE10EC0C2F70FC0FB
:10584000C3F7190E29ECBEF003E2036802681DD00D
:10585000410E29ECBEF015E29CECBAF0190E495E3F
:10586000000E4A5A4950016EB6ECC1F00800F550DE
:10587000026EB6ECC1F0F62A90ECBCF0F550036E67
:1058800004D069C302F06AC303F0010196A904D0F1
:1058900069C302F06AC303F0FE0EDB5007E10701A3
:1058A000BF51025C03E1C051035C20E002C0BFF7BE
:1058B00003C0C0F7410E29ECBEF011E20101965180
:1058C000100B0DE1010EE66EE66A0350E66E025023
:1058D000E66E66ECBAF00B0EE0ECBDF005D0FE0E05
:1058E000DB5002E043ECBFF059ECBDF0B5EFB6F091
:1058F0000101A751A227A251090803E20A0EA25FE3
:10590000A12BA651A127A151090803E20A0EA15F0C
:10591000A02BA551A027A051630803E2640EA05F4D
:105920009F2BA4519F279F51630803E2640E9F5F42
:105930009E2BA3519E2712000101A751A25FA251E5
:105940000A0803E20A0EA227A107A651A15FA151EE
:105950000A0803E20A0EA127A007A551A05FA051E3
:10596000640803E2640EA0279F07A4519F5F9F5124
:10597000640803E2640E9F279E07A3519E5F1200F6
:1059800002ECC1F02BBC03D01AD82F9E10D02CAA49
:1059900007D02050400B0AE01F50020B08E106D050
:1059A0002050400B04E01F50020B01E008D8020E0B
:1059B000E15C02E2E16AE552E16EB5EFB6F002ECBD
:1059C000C1F00101E851010BDE6EDD6A1F50020BD0
:1059D00006E02050400B03E014ECBCF002D060EC79
:1059E000B9F0A76BA7C1A6F1A7C1A5F1A7C1A4F102
:1059F000A7C1A3F120ACE8912050400B0FE1D45196
:105A00000DE11BECC5F001E0010EEDECB9F002E098
:105A1000000E01D0010E491875E170D02050400BE6
:105A200012E03450400B0FE01BECC5F001E0010E1A
:105A3000496E020ED45D02E0000E01D0010E49183D
:105A400061E17ADF60D02050400B19E1D40503E01A
:105A5000020ED45D14E127ECC0F011E201010F0E3B
:105A6000A56FE651040B01E0010E496E020ED45DF4
:105A700002E0000E01D0010E491840E043D0E2ECF4
:105A8000BEF014E00101090EA56F010EA66F050E10
:105A9000A76FE651040B01E0010EEDECB9F002E056
:105AA000000E01D0010E491829E02CD02050400BE7
:105AB00013E1B6ECBCF010E001010A0EA56FE6514F
:105AC000040B01E0010EEDECB9F002E0000E01D094
:105AD000010E491813E016D02050400B14E1ABEC36
:105AE000BAF003E0040ED45D0EE1010EA46F140EB3
:105AF000A56F040ED45D07E1E6A504D01DDF01010A
:105B0000E88101D0F5DEC6ECBEF015E02050400B78
:105B100012E1050ED45D0FE0040ED45D0CE0A36B22
:105B2000A46B500EA56FA76BA7C1A6F1E6A502D086
:105B3000DFDE01D001DF25ECBAF01BE2100E2B5D99
:105B400050ECBBF00101A46BA4C1A3F124ECC5F09F
:105B5000A56F29ECC5F0A66FA76BE651040B01E019
:105B6000010E496E2EECC5F0491802E0E5DE01D0C9
:105B7000BFDE3FECB9F003E1CAECBEF019E006016C
:105B8000F0510101A05D14E10601EF5101019F5D9B
:105B90000FE10601F1510101A15D0AE10601F25197
:105BA0000101A25D05E10601EE5101019E5D0CE0DF
:105BB0009EC1EEF69FC1EFF6A0C1F0F6A1C1F1F6CD
:105BC000A2C1F2F62BECB3F0020EE15C02E2E16A54
:105BD000E552E16EB5EFB6F0D9CFE6FFE1CFD9FFE0
:105BE000BAC19EF1BBC19FF1BCC1A0F1BDC1A1F181
:105BF000BEC1A2F10101A86BFE0EDB50090807E24D
:105C00002996FE0EDBCFE6FF12EC28F0E5520101EB
:105C1000006B800E01011315036E800E010110153B
:105C2000026E010EEA6E9E5105D89F5103D8A05115
:105C300001D814D0076B066F0A0E065DD8A003D0FA
:105C4000066F072BF9D700510E0FE96E0751EF6E63
:105C5000E92A0651EF6E002B002B000CA1C114F1B4
:105C6000A2C115F10101A85107E10A0E01019E5DD3
:105C700003E20101100E0E6F0701BABB03D0010150
:105C8000100E156F0701BAAD05D00101100E146F8B
:105C900014C115F11DBC03D00101108F03D00250B7
:105CA000010110130101138F0101A85109081AE223
:105CB0000201365117E08CECCFF00101020E006FAB
:105CC0009EC100F04DECD5F0A8C100F00101006BC1
:105CD0004DECD5F0010EE66EE66A5BEC07F0E5529E
:105CE000E55223D00101A8511FE007010701BA5175
:105CF000200B1AE1288C14C115F113C114F112C143
:105D000013F111C112F110C111F10FC110F10EC147
:105D10000FF10A0E496E49C043F0A8C13EF06FEC86
:105D2000E5F03AC00EF101D0289CE552E7CFD9FF4B
:105D30001200D9CFE6FFE1CFD9FF020EE126010E16
:105D4000A8C1DBFF2BC1DFFF0101D551EA6AB40F07
:105D5000E96E070EEA22EFCFBBF7BFC19EF1C0C1CB
:105D60009FF1C1C1A0F1C2C1A1F1C3C1A2F1010162
:105D7000A86BDF50090806E22996DFCFE6FF12EC98
:105D800028F0E5520101016B800E01011B15026E26
:105D9000010EEA6E9E5105D89F5103D8A05101D83B
:105DA00016D0076B066F0A0E065DD8A003D0066FEB
:105DB000072BF9D70151160FE96E0751300FEF6E1F
:105DC000E92A0651300FEF6E012B012B000C300E2B
:105DD0000101A12501011C6F0101A85107E10A0E73
:105DE00001019E5D03E20101200E166F0701BBADAC
:105DF00003D00101200E1C6F0101188F01011B8FC0
:105E00000101A8511DE007010701BB51200B18E15A
:105E10001BC11CF11AC11BF119C11AF118C119F1EA
:105E200017C118F116C117F10A0E496E49C043F0A7
:105E3000A8C13EF06FECE5F03A50300F0101166F4B
:105E4000A8C1A9F1010EDBCFA8F1020EE15C02E2CC
:105E5000E16AE552E16EE552E7CFD9FF1200E6ECC8
:105E6000C0F0830E096E0A0EE66E01010D03F350B9
:105E7000E66E5E0EE66E020E2BECB7F0DE0E8EECDA
:105E8000B8F00050DF6EFE0E70ECC6F00101E59D2B
:105E90002E9EB90E005C16E1FF0E02015E5D12E05F
:105EA0002E8E020E01012B5D0DE1050E0201635DD8
:105EB00009E1210E5F5D01E1606B280E645D02E186
:105EC0003C0E656FA30EDF5C02E10101E58DE5523A
:105ED000B5EFB6F08C0E02018D1909E10A0E8E198C
:105EE00006E18C0E8F1902E10A0E901907E0800E70
:105EF0008E1504E1800E901501E1000C010C0201E9
:105F0000915102E1925107E0FF0E915D04E0FF0E16
:105F1000925D01E0000C010C2B50080B0CE03CECF6
:105F2000C2F009E12B5105E1010EE66E6FDCE5528E
:105F3000120043ECBFF0120018B038D00DC1E6FFDC
:105F4000BFEC51F0E552C6DF000902E0D1ECBCF035
:105F50000DC1E6FFDBEC51F0E552D1DF000903E0B3
:105F60000201916B926BB3EC12F079DF0101565193
:105F7000080B03E12B51090809E2FF0E02018A5DBB
:105F800002E1320E8A6F8AC248F108D0FF0E8C5DA2
:105F900003E1320E8C6F02D08CC148F16AEC3AF00A
:105FA000DAECB8F0E66AF6ECBCF0B6DFCDEFBDF0A7
:105FB000E6ECC0F0FD0EDB50100DF350DF6E010E6D
:105FC000096E0201680E986FFD0EDB5009080AE2A7
:105FD000020E096E690E986FFD0EDB50F00F100D6A
:105FE000F350DF6EFE0EDB50FF0802E0FBECC2F068
:105FF000DF50E552B5EFB6F00201875103E087515B
:10600000330802E20D0E876F8851D3ECB7F007E238
:106010004950FA08000E4A5402E21E0E886F89BFEA
:10602000896B93510E0803E2936B0101D09B120020
:106030002AECC2F0FF0811E0FBECC2F00F0EF9EC05
:10604000C3F000C02BF101018A51100B06E00A0ECB
:1060500045ECB7F002E2FE0EDB682BC10DF1020148
:10606000756B0101E695E5992B5109081AE2100EAE
:106070002B5D006E0050BAECC2F00BE0A2ECC3F056
:1060800001010D6FE2ECB6F0EF380F0B0201756FF6
:1060900008D0FE0EDB680101090E0D6F0DC12BF15A
:1060A000258E2BA605D007011187140EE0ECBDF05C
:1060B00022A603D0010EE0ECBDF00701128F12936F
:1060C00012C7E6FF120EE66E480ECEECB6F034ECC8
:1060D000B8F0100E2CECC3F029A403D07EEC04F031
:1060E00029940F0E0101CE15D46FCE390F0BD56F49
:1060F000D551060802E2D4C1D5F1D40501E1CF9112
:10610000020ED45D01E1CF8192ECC5F00A6ED2811E
:10611000040EE66E0B0EDF24E66EDC0EE66E010E5C
:106120002BECB7F00101DF8134ECB8F0FE0EDB5050
:10613000FF0803E198C209F002D0100EDF26100E0E
:106140000FECC6F0870EE66E020E2BECB7F054DFB4
:10615000FE0EDB50FF0852E026ECBBF0DF6E0B0EAC
:10616000F9ECC3F08AECB8F008E01F0ECF17E00E90
:106170000014CF1392ECC5F00A6E0C0EF9ECC3F0CC
:10618000440E0101D017BB0E0014D01395ECC5F0DE
:10619000470E0101D117B80E0014D11395ECC5F0CC
:1061A000980E0101D217670E0014D21398C209F09D
:1061B0000A0EE66E030EDF24E66E8A0EE66E020E0F
:1061C0002BECB7F026ECBBF0DF6E0C0EF9ECC3F055
:1061D000440E0101DD17BB0E0014DD1395ECC5F074
:1061E000470E0101DE17B80E0014DE1395ECC5F062
:1061F000980E0101DF17670E0014DF13096AC4C18E
:1062000019F5C5C11AF5C6C11BF5C7C11CF5C8C132
:106210001DF5C9C11EF5CAC11FF5CBC120F5CCC102
:1062200021F5CDC122F518B41CD012941296129A01
:106230001F92010138A30CD0D1A102D0128A1F8273
:106240001296D1B312861294D1A509D0128407D028
:10625000FCECBEF00101DE95DE93D195D1936AECA2
:106260008BF025ECBAF03DE25C0E0D251AECB8F08F
:10627000006E00500101C45D016E01AE03D0C45137
:10628000005C016EE651040B03E10150030803E3D7
:10629000015019080AE2050E05ECBDF0C40EE66EC9
:1062A000010E92ECB7F000C0C4F100500101C95DCD
:1062B000016E01AE03D0C951005C016EE651040BC2
:1062C00003E10150030803E3015014080AE2050E3C
:1062D00005ECBDF0C90EE66E010E92ECB7F000C001
:1062E000C9F1E5ECBDF0CBEC20F083EC0BF0129C97
:1062F00001013BB1128C129E3BB3128E10EC5BF08D
:10630000129801013BB9128864EC1CF00101D09F86
:106310001190118299EC07F0DDEC45F08FEC45F01F
:10632000096A010137A702D0C3EC3FF0FEECBBF0D5
:1063300009ECBCF001DEE1EC04F00101246B1DBCB2
:1063400004D007019D6B3DECBFF0010EE552B5EFA7
:10635000B6F0E6ECC0F00A0E01012B5D11E2C5C1FA
:10636000E6FFC4C1E6FFF7EC1CF0E552E552005031
:1063700001012B5D05E00701020EFDECC4F06ED0BB
:106380000A0E2B5D02E248C18CF134ECB8F05CECF3
:106390001CF00101D09F38A30DD0F80ED117D19178
:1063A0001FB2D181D19312B6D183D19512B4D185C8
:1063B0009EEC39F02BC1D3F104ECC3F0050E8BEC4D
:1063C000BCF00FECC6F018ECB7F00A0EDF24016E3B
:1063D0000101D539F00BD4112DECBEF0050EE66E9F
:1063E000CF0EE66E010EE66E0B0EDF24F3ECC1F06D
:1063F000050EDBECBDF0E66E050EDF24F3ECC1F01C
:106400001CBA24D034ECB8F001015651080B03E15A
:106410002B51090802E248C18AF21EECAAF03AC1E7
:106420008BF2FE0EDB50FF0803E198C209F002D0A8
:10643000100EDF26100EE66E870EE66E020E0FECD3
:10644000C6F018ECB7F0096AC0EC10F0010137A7EC
:1064500002D0A3ECBBF0096A0201206BE552B5EF54
:10646000B6F0E6ECC0F00F0EDF6EF40E060100177A
:10647000F00E0517DF500617E552B5EFB6F006012E
:106480000691009501910299019914991399049923
:1064900003911200B9ECB6F03CECC2F001E0010E41
:1064A000496EFE0EDB5002E0000E01D0010E4918CD
:1064B00003E00601058502D00601058701018AA1D6
:1064C00002D00601068DB5EFB6F00050040A4AE08E
:1064D000070A22E0010A1BE0030A17E0010A01E0B3
:1064E0001200060105833CECC2F001E0010E496E8A
:1064F000D051400B01E0010E491802E00601058170
:106500000601EA5131E0068B1200E66A02D0010E64
:10651000E66EC0DFE5521200060100813CECC2F0DD
:1065200001E0010EDBECBCF002E0060105810A503F
:1065300003E0030E0A5C02E1060105719CECC0F069
:1065400002E00601068B32A00FD03CECC2F001E065
:10655000010EDBECBCF003E006010587120006012A
:1065600005851200060100831200800E071406E064
:106570002050010B03E1D4C100F003D009EC1CF062
:10658000006E6FDF65EF32F01200B9ECB6F08AEC06
:10659000B8F00DE10A0403E0020E0A5C04E1D051F8
:1065A000040B16E10BD0CF51040B08E011D0D40539
:1065B00007E127ECC0F002E2420E17D0450E15D0DD
:1065C000020ED45D07E127ECC0F002E2400E0DD0D0
:1065D000440E0BD0040ED45D02E1460E06D0D0511D
:1065E000400B02E1430E01D0410E28ECB7F019EC4C
:1065F000BAF0030E005C12E10A0403E0020E0A5C2A
:1066000005E10101D051040B05E106D00101CF5194
:10661000040B02E0540E17D0550E15D0000402E111
:10662000520E11D0020E005C02E1500E0CD0040E8E
:10663000005C02E1560E07D00101D051400B02E18F
:10664000530E01D0510E28ECB7F0B5EFB6F02EEC9A
:10665000C2F033B835D02050800B12E11450100B2B
:106660000FE01450200B0CE10101D45106E0030EA1
:10667000D45D03E0050ED45D03E11498FEEC46F012
:106680008AECB8F003E0050ED45D01E1D29D1390D1
:10669000D45103E113908AB51380030ED45D05E154
:1066A0000A5003E013908EB51380139A13A0138A37
:1066B00082EC0AF010EC5BF057EC15F0CBEC20F01C
:1066C0002582C0EC2CF0010EE66E5FDFE552B9ECDE
:1066D00013F0F7EC19F033B849D069EC15F0FEEC83
:1066E00046F0BAEC0DF054EC1BF0A7EC1AF028B20F
:1066F0003DD01C98349027AA02D00DEC07F00E6A0A
:106700000F6A88ECC0F004E1100E0E6E270E0CD05C
:10671000050ED45D04E1240E0E6E2C0E05D0D2A120
:1067200004D0400E0E6E1F0E0F6EDFECB8F0A40EFC
:10673000D3ECB6F09CEC1AF06F0E28ECB7F04DECF1
:106740004AF011EC1BF087EC19F076EC15F056ECE2
:1067500012F06BECB7F002E008EC1AF07EEC12F0ED
:1067600053EC1FF074EC5BF099ECB2F03398030E2D
:10677000E15C02E2E16AE552E16EB5EFB6F08C98B9
:1067800000000000030EE66E95EC53F0E552040E97
:10679000095CE66E95EC53F0E5520150E66E95EC1F
:1067A00053F0E552E8ECE4F0006E00008C88120033
:1067B000D9CFE6FFE1CFD9FF8C9800000000060E8C
:1067C000E66E95EC53F0E5528C8800000000000066
:1067D0008C9800000000020EE66E95EC53F0E55236
:1067E000040E095CE66E95EC53F0E5520150E66E3E
:1067F00095EC53F0E552FE0EDBCFE6FF95EC53F03F
:10680000E5528C88040EE66EBAECE4F0E552E552EF
:10681000E7CFD9FF120002ECC1F00050DF6E010E8D
:10682000DB6A3CD8DF50005C31E0680E095C02E1B5
:10683000012A0106040E095C16E2F29EA698095090
:10684000636E0150626EDF50616E7F9E7F9C7F841D
:10685000550E7E6EAA0E7E6E7F82F28E040ECFECF7
:10686000C2F07F9413D0010EDB2ADFCFE6FFA0DF5A
:10687000E55285DFDF50005C02E070EC0BF0DF508A
:10688000005C04E0050E7EECB9F0EDE3020EE15C85
:1068900002E2E16AE552E16EB5EFB6F002ECC1F05A
:1068A000010EDB6A040E095C0AE20950636E0150B6
:1068B000626E7F9E7F9C7F806150006E12D0010EC1
:1068C000DB2A5DDF0050DF6E5ADF0050DF5C02E044
:1068D00070EC0BF00050DF5C04E0050E7EECB9F0CC
:1068E000EEE3020EE15C02E2E16AE552E16EB5EF31
:1068F000B6F0B9ECB6F049ECBFF013E0FC0EDBCF1C
:10690000F3FFDB2AF3508EECB8F0FD0EDBCFE9FF8E
:10691000DB2AFE0EDBCFEAFF01E3DB2A00C0EFFF3C
:10692000EAD7B5EFB6F0B9ECB6F049ECBFF016E037
:10693000AFECBDF013E3F6ECC3F005E24950A40858
:10694000000E4A540BE34DECBDF0016E60ECBEF05E
:1069500001E3DB2AEF502DECBEF0E7D7B5EFB6F040
:10696000B9ECB6F01F0E0501235D0DE2232B255176
:10697000EA6A270FE96E050E94ECC3F0252B25512A
:106980001F0801E2256BB5EFB6F0B9ECB6F0030EC7
:106990000A5C54E10E6A0F6AFE0EDB500D0803E13B
:1069A0001F0E0E6E0F6AFE0EDB500A0803E11D0E6D
:1069B0000E6E0F6AFE0EDB50090803E1EF0E0E6E3D
:1069C0000F6AA0ECC0F003E10E68020E0F6EFE0E1F
:1069D000DB507F0804E1B50E0E6E030E0F6EFE0E47
:1069E000DB501F0821E27F0E45ECB7F01DE2410E9F
:1069F00045ECB7F00CE3FE0EDB505A0808E3200E1E
:106A0000496EFE0EB1ECC3F0FE0EE7CFDBFFFC0ECD
:106A1000496E8D0E4A6E010E4B6EFE0EDB50E00F7E
:106A2000CFECC5F099ECC4F00E500F1049E00FC048
:106A3000E6FF96DFE5520EC0E6FF3DD0FE0EDB50CE
:106A4000090803E1200E42ECBBF0016A400E015C34
:106A500037E2E60E4A6E9B0E4B6E010E4C6E0150F5
:106A6000A9ECB7F0FE0EDB50495C28E1030E066E80
:106A700001B0068C01B2068A01B4068801B606860A
:106A800001B806842350040B09E1200E011406E02E
:106A90006F0EE66E65DFE55223840BD02350040BA6
:106AA00008E0200E011405E17F0EE66E59DFE55285
:106AB00023940650E66E54DFE55202D0012AC6D771
:106AC000B5EFB6F0E6ECC0F0800E45ECB7F003E3AE
:106AD000200E42ECBBF00201050E2D6FFE0EDB50C6
:106AE000740810E1010E2D6F030E0A5C07E1050129
:106AF00023515FECC4F0020F02012D6F0501106BF2
:106B00001D822BD0FE0EDB5028E0DF6A150EDF5C05
:106B100011E2A0ECC4F00BE1DF2AD9ECB9F02CECC7
:106B2000C0F0DF2AD9ECB9F02CECC0F003D0030E92
:106B3000DF26ECD7150EDF5C04E12FECC1F025DF7A
:106B4000E552200E45ECB7F003E2200E42ECBBF01C
:106B50002FECC1F057EC65F0E552E552B5EFB6F019
:106B600002ECC1F023A012D01DB009D00201535D88
:106B70001CE30701016B026B53C254F216D00201F1
:106B8000532B535180081BE2800E18D01DA010D04B
:106B9000070E0701015D09E2012B02910243020E7B
:106BA0000201535D02E30701028F0201010E06D0CC
:106BB0000201532B5351800802E2800E536F1D9047
:106BC00023B01D802350010B03E1020E535D04E04E
:106BD0001D50020B01E18AD01DA204D00701CC0E8A
:106BE000026F0FD0070102910243028F070ED88077
:106BF0000155016E01500106000903E002910243B4
:106C0000F9D700C709F00101B5A7E88B020154517B
:106C100007081DE254513F0802E23F0E546FC8ECD2
:106C2000BDF006E0200EACECB9F0200E2CECC0F06C
:106C3000BAECBCF00CE00701035109E0800E020140
:106C40005425006E03C701F007010307E4DD780E49
:106C50000701025D18E2298A02C7E6FF3CEC04F056
:106C6000E552DF6EDF500EE0C8ECBDF00BE02D51B9
:106C700004E0DFCFE6FF26DF04D0DFCFE6FF57ECEE
:106C800065F0E552299A0101E89BB5A72FD00701CD
:106C9000035105E002C700F003C701F0BCDD0701A6
:106CA000035106E01D50020B03E11C0E025D1BE1C7
:106CB00003510AE01C0E025D07E1CC0E006E0307D3
:106CC00003C701F0A8DD1D820101B5970AEC5CF055
:106CD000230E155C03E1410E6FECB7F0249223AC58
:106CE00003D0248201D003070701026B096A020E58
:106CF000E15C02E2E16AE552E16EB5EFB6F03FEC2D
:106D0000B9F00CE11B0E0101B95D08E11850400B10
:106D100005E084848C808D8A8D8C12000601505190
:106D2000040B02E08D8C01D08D9C5051080B02E0C9
:106D30008D8A01D08D9A5051010B02E08C8001D0D8
:106D40008C905051020B02E0848412008494120053
:106D5000000012000601D99D8850800B01E0D98DFA
:106D6000D99F8850400B01E0D98FD9998850080BE2
:106D700001E0D989D99B8850040B01E0D98B12001E
:106D8000B9ECB6F0FD0EDB5045ECB7F008E3FE0EB3
:106D9000DBCFE6FFFD0E68ECBEF00AE207D0FD0E89
:106DA000DBCFE6FFFE0E68ECBEF002E2010E01D082
:106DB000000EB5EFB6F02EECC2F02EB254D082B079
:106DC00003D00701290E76D082B203D007012C0E22
:106DD00071D0DF6A060EDF5C43E2DF50040DF35032
:106DE000830972ECBCF0050EDF5C03E1DE52BB0EE2
:106DF000DD6E33ECC5F000C045F700501A082EE2F6
:106E0000F00E005C2BE2FE0EDB5002E1010E56D0CC
:106E100033ECC5F000C046F700501A081FE2F00E30
:106E2000005C1CE233ECC5F000C047F700501A08C4
:106E300015E2F00E005C12E2080EE66E46C7E6FFB1
:106E400045C7E6FF89ECB9F009E0080EE66E47C7D2
:106E5000E6FF46C7E6FF89ECB9F002E1DF2ABAD7C0
:106E6000060EDF5C02E1000E29D0010ED1ECBDF070
:106E700070ECBEF010E20C0EE66E020EDB50370F27
:106E8000E4ECB8F0E66E46C7E6FF89ECB9F003E142
:106E9000020EDB2AEDD770ECBEF00FE245C748F7D3
:106EA00046C749F747C74AF7020EDB50080DF350B3
:106EB000DF1007014B6F4B5101D0800E496E030E5E
:106EC000E15C02E2E16AE552E16E4950B5EFB6F0ED
:106ED000C4ECBBF07CECC0F006E1EEECBCF003E0EF
:106EE00001011E0EAC6F01012D0E176F1FA402D001
:106EF0002B0E176F0201405107E13F5105E13E5152
:106F000003E10101200E176F63ECB7F040C23EF0C1
:106F100031ECB9F00101186F300E3A24196F300EC0
:106F200002013F2501011A6F0701BAAB05D0300EEF
:106F300002013E2501011B6F0101198F12002AEC8D
:106F4000C2F0C9ECB7F0EFCFDFFF0101A36BA46B78
:106F5000A56BA66BA76B1DAE03D0050EA56F32D037
:106F6000E9ECBDF0EF50400B03E12750040B1DE0AE
:106F70002FECC1F08AEC0BF0E55200C0A5F10050F7
:106F800063081BE20101A56BA42B7D0E005C02E1EE
:106F9000190EA56F13ECC6F0FA0E49180EE14A500F
:106FA0000CE1A42B320EA56F08D0E9ECBDF0EF5038
:106FB000200B02E0A72B01D0A62B2AAE03D0020E95
:106FC000DDECB6F0E552B5EFB6F0A60E006E00505F
:106FD00055ECBBF035C100F06AECD5F0300E010184
:106FE0001A5D05E1B6ECC3F002E1200E1B6F020151
:106FF000060E3D6FCBEF20F0B9ECB6F0910E496E66
:107000009E0E4A6E010E4B6E050E4F6E4FC043F042
:10701000FE0EDBCF3EF06FECE5F03EC04CF04D6A6B
:1070200060ECC2F0006E8CECCFF00101020EDDECE2
:10703000BFF0128F0C0E45ECB7F003E20E0E0F6F8F
:107040000ED00E0E106FFE0EDB50630802E2100E23
:10705000106F0F0E45ECB7F002E2090E116F140E1F
:10706000146F120E156FB5EFB6F0B9ECB6F09CECDC
:10707000CFF00101012BFE0EDB50006E6AECD5F063
:107080002B50100B07E1640E45ECB7F003E2010151
:10709000200E176F2BA807D001014D0E1B6F570E46
:1070A0001C6F188F14D0FD0EDB5003E10101198F06
:1070B00007D00A0E45ECB7F003E20101200E186F6D
:1070C0000101570E1B6F33B602D02A0E1C6FB5EFAD
:1070D000B6F0B9ECB6F0CBEC20F0FE0EDB5003E0DE
:1070E00079ECC0F003D000682FEC22F009ECB8F086
:1070F0001AE0020E0101395D0FE1A50E485D0CE1B9
:107100009CECCFF0830EE66EB30EE66E010EE66EDB
:1071100011ECD6F0E5520BD0010EE66E65EC05F0F1
:10712000A60FE66E03D0E66A48C1E6FF9EDFE55291
:10713000E5522BA807D0006823EC22F048C1E6FFF7
:107140005BDFE552B5EFB6F0C4ECBBF07CECC0F011
:1071500008E1EEECBCF005E00101D45102E0AC9195
:10716000AC4349C100F06AECD5F0640E0101495D01
:1071700002E2200E166F0A0E495D02E2200E176F22
:10718000890E006E6BEF21F0270E6FECB7F0010156
:10719000500EAC6F3B51200B06E1EEECBCF003E06F
:1071A00001011E0EAC6F1200B9ECB6F06BECB7F03B
:1071B00003E0CFECB7F003E028C100F008D0DEEC2C
:1071C000BEF003E058C100F002D054C100F0B5EFAA
:1071D000B6F0C70E02ECBDF0010EE66EE5DFE5523B
:1071E0006AECD5F0300E01011A5D05E1B6ECC3F092
:1071F00002E1200E1B6F1200B9ECB6F047ECB8F0BC
:10720000EF50400B03E12750040B04E001018E51C5
:10721000020B6AE047ECB8F0EF50200B03E0275078
:10722000040B02E00101A26B47ECB8F0EF50400BF9
:1072300003E12750040B58E00101A4510EE0A551D1
:107240000CE1FE0EDB5005E1A05102E1A15101E08D
:10725000A46BA06BA0C1A1F147D05A0EA55D16E1A9
:1072600063ECB7F0A0C13EF080ECC0F0006EFE0E03
:10727000DB5007E1005003E10101A15102E00101EF
:10728000A56B0101A16B0050A05F2ED0A05102E1BF
:10729000A1512AE0A151496E4A6AA0510A0D82EC1F
:1072A000B9F0A5510A0DF6ECBFF085ECB8F0D8C1E5
:1072B00042F0D9C143F015ECE5F039C0D6F13AC03F
:1072C000D7F10101D651D7110FE0D6510E5ED7513B
:1072D0000F5AFE0EDB5001E1A56B0A0E8EECC1F0D9
:1072E0003DC0A0F139C0A1F1B5EFB6F0B9ECB6F0F0
:1072F0002FECC1F0E66A80DFE552E5529EC19AF2BA
:107300009FC19BF2A0C19CF2A1C19DF2A2C19EF2BD
:107310009CEC2CF001019E510DE1320E9F5D0AE2C2
:107320009AC29EF19BC29FF19CC2A0F19DC2A1F1A5
:107330009EC2A2F102016F2BB5EFB6F00101DE9300
:10734000D1B3DE83DE95D1B5DE851200010138A30D
:1073500006D0D19312B6D183D19512B4D185EEDF88
:1073600004B0B6DD6AEC8BF071EF29F00A0E020171
:107370003F03F3504B6E4C6A4051640D28ECBFF054
:107380003E5101014924DA6F000E4A20DB6F0A0EDC
:10739000006E0701BAAB02D0010E006E1FB403D01D
:1073A0000101EEECBDF028AA1AD013ECC6F0100EC5
:1073B000D8804956270E4A560101DB514A18E8AEDB
:1073C00002D04A3404D04950DA5D4A50DB591FE2FA
:1073D00000508AECC2F0DA274A50DB2318D0005064
:1073E0004A6AF00F496ED80E4A2201014A50DB1951
:1073F000E8AE02D0DB3504D0DA51495CDB514A58A3
:1074000006E200508AECC2F0DA5F4A50DB5B1F8470
:10741000800EDB1503E01F94EEECBDF00050BEECD7
:10742000C2F01EECBFF04AAE04D0396C3A1E000E1A
:107430003A2239500101DA5F3A50DB5B640EBEEC50
:10744000C2F054ECB7F03DC040F239500101DA6FA0
:10745000DB6B0A0EBEECC2F054ECB7F03DC03FF25D
:1074600039C03EF234EF3AF02F8E0480A6EF39F0A7
:107470000A01DA9F82EC0AF0016A0101D4510EE19F
:107480000701BABF11D00A0E016E3CECBAF03E50B3
:10749000006E0150005C18E2005015D0030ED45D60
:1074A00011E10701BAAF02D0160E0DD0030E0A5C2F
:1074B00002E1140E08D00A5002E11E0E04D065EC61
:1074C000C3F001D0160E016E0150160802E2160E2E
:1074D000016E12001200B9ECB6F000AE14D0FF0E2F
:1074E0000002F3CF6FF26F0EE96E020EEA6EEFCF7D
:1074F0003EF0FE0EDBCF43F06FECE5F03EC0EFFF59
:1075000002016F6D09D000C03EF0FE0EDBCF43F0EC
:107510006FECE5F03EC06FF2B5EFB6F0E6ECC0F010
:1075200033A202D0D6EC45F02F50200B5DE1235062
:10753000800B5AE12450010B57E13050400B54E1CD
:107540001FA618D075ECBEF00101269902016F51FB
:1075500002E0010126890101269B02016FAF02D0E2
:107560000101268B010126A93FD01DAC3DD039EC8D
:107570000AF03AD024C100F001012699005001E040
:107580002689269B00BE268B26BB006C3FECB9F0FB
:107590001CE12E50100B0DE01E50040B0AE11B5095
:1075A000080B07E1005002E025EC07F0006A01013A
:1075B000246BCAECBEF00DE03D0EB95D0AE0D89038
:1075C0000032D89000322EA004D0D8900032D8904B
:1075D0000032005007E00101268D269F26BB268F32
:1075E000246B02D001012699010126A902D09BEC4F
:1075F00004F001012651100B06E02B50200B37E060
:107600001D50400B34E11F50080B16E03B51200B7E
:1076100013E13BB329D07DECBEF0010127990201B3
:107620006F5102E0010127890101279B02016FAF21
:107630001ED00101278B1BD025C100F027990050D7
:1076400001E02789279B00BE278B279927BB006C69
:107650000090004200500AE00701460EA26F0101AF
:10766000278D279F27BB278F256B01D027992B506C
:10767000200B03E01D50400B0DE001012651100BC3
:1076800001E02BD32751100B01E027D32050200B12
:1076900001E123D3D7CADCFAD6CADDFA0601D551F7
:1076A000D595010B01E0D585D551D597020B01E0A9
:1076B000D587D5918650040B01E0D581D5938650AE
:1076C000020B01E0D5830F0ED515F7ECB9F000A041
:1076D00019D09BEC04F006015051040B0CE0325021
:1076E000010B09E13050040B06E100AE02D0DA07CD
:1076F00009D0DA2B07D000AE03D00101250702D054
:107700000101252BDAC600F00601D599005001E0F1
:10771000D589D59B00BED58BD5A92ED0D5BB006C05
:1077200000900042005028E0DA6B50A525D00101FE
:107730003751010B06E01250080B03E11250040B05
:107740000FE0288A0601D5BB289A10DE1EAC03D0B4
:107750000201098702D0020106810501478D0CD084
:10776000AAC224F10601D5AB04D0AAC224F10101BA
:10777000246D0101268927840601D751D795010B75
:1077800001E0D785D751D797020B01E0D787D951B0
:10779000D791200B01E0D781D951D793100B01E08D
:1077A000D7830F0ED715F7ECB9F000A00CD09BECE7
:1077B00004F00201140E2B6F00AE03D00601DD07AA
:1077C00002D00601DD2BDDC600F0D799005001E0A4
:1077D000D789D79B00BED78BD7A95BD1D7BB006C0D
:1077E00000900042005001E154D1DD6B010E0D6E9E
:1077F000D7BB0D681950100B04E12050800B01E13C
:10780000DFD001018DB525D133B631D020BE04D0F3
:10781000740E006E23EC22F0FF0E0D5C0CE10201F1
:10782000050ED8800055000E01551EE2060E005FC1
:10783000000E015B19D071C201F02B50100B07E153
:1078400002017151640803E25A0E015C016E01509D
:107850000B5C0AE20201880E005D130E015904E27E
:10786000060E0027000E012311EC0AF00ED10201D2
:107870001D6B640E016E026AA8ECC0F002E0C80E37
:10788000016E2BA804D0960E016E0A0E026E0150F6
:10789000E66E0250E66E480EE66E010E07ECB7F09B
:1078A00009ECB8F00CE1010148510A0808E2010EA8
:1078B000481505E00D0402E1482B01D048072A8451
:1078C0000901ED6BEE6B11EC05F053EC1FF031ECA0
:1078D000C0F0E5520201320E046F48C15BF248C1AC
:1078E0008CF10101E783E795E79748C102F009ECC5
:1078F000B8F004E00101E7935A0E025E0250E66E12
:1079000071EC08F0E552A8ECC0F015E02B50100B1C
:1079100012E10D0404E1650E0101485D07E0800EEF
:107920000D1409E0640E0101485D05E1318EEEECB5
:10793000B8F001E01C9419ECBAF03150800B11E161
:107940002050800B0EE1EEECB8F00BE100500BE0A4
:10795000050E005C08E0030E005C03E1020E0A5C09
:1079600002E00D5001D0020EF3ECBDF031AE25D097
:10797000319E049819A006D004886FEC09F0050E1A
:10798000DDECB6F00101395111E009ECB8F006E088
:107990007D0EE66EB30EE66E010E02D065ECBDF014
:1079A0000EECC3F003E1FA0EDDECB6F004A802D051
:1079B0006AEC09F00D50F3ECBDF00201078B65D0C5
:1079C00024A01CD03484FAECBCF008E0C80EE66EAB
:1079D000280EE66EB80EE66E030E0BD049DD190ECA
:1079E0000124E66E190ED8800154E66ED70EE66EBD
:1079F0000A0E07ECB7F0A7ECC4F047D06BECB7F079
:107A000006E0CFECB7F003E12750020B1DE0320E89
:107A1000006E0050E66E080EE66E490EE66E010E30
:107A200007ECB7F0A4EC38F00101E793E795E7879E
:107A300049C1E6FF71EC08F0E55249C113F5ADEC20
:107A40005BF00201068721D019ECBAF001018DA587
:107A500003D01EEC07F019D06CEC15F0500EE66E5A
:107A6000350EE66E010E02ECB7F056EC12F0E5ECC6
:107A700037F00101E793E795E79735C1E6FF71EC31
:107A800008F0E552020108832A842D8E02011E0EA1
:107A9000206F0601D851D895010B01E0D885D85147
:107AA000D897020B01E0D887D951D891800B01E01B
:107AB000D881D951D893400B01E0D8830F0ED81547
:107AC000F7ECB9F000A00CD09BEC04F00201140E0E
:107AD0002B6F00AE03D00601DC0702D00601DC2BC1
:107AE000DCC600F0D899005001E0D889D89B00BED0
:107AF000D88BD8A9F2D0D8BB006C009000420050BF
:107B000001E1EBD0DC6B010E0D6ED8BB0D682CA62D
:107B10004DD06BECB7F003E0CFECB7F00AE0280EE5
:107B2000E66E280EE66E010E02ECB7F037ECC5F0FB
:107B300011D01DECBEF010E02150020B0DE12C968F
:107B4000C6ECB9F02196E20EE66E940EE66E010EDA
:107B5000A7ECB8F0E55220D011ECBEF00BE11E0E00
:107B6000E66E580EE66E010EE66E40EC6FF0E552E2
:107B7000E5520FD01E0EE66E540EE66E010E02ECBC
:107B8000B7F00101E793E795E79754C1E6FF71EC81
:107B900008F0E55276EC15F01DECBEF004E0215043
:107BA000020B01E196D0E9EC38F093D023AE39D046
:107BB00021B68FD0016A0101D45102E0010E016E9D
:107BC000015063ECC2F0EF50006E13ECC6F0190EDA
:107BD000426E436A0DECB7F0190E4A02F3CF4AF039
:107BE0004902F3CF49F0F4504A264950006E0D0483
:107BF0000AE1E5ECC2F004E6E20E495C000E4A58E8
:107C000002E2190E0026FF0E0D5C05E10050180877
:107C100002E2190E005E015063ECC2F000C0EFFFFB
:107C200045D024A038D034840CEC0EF0ECECC1F03C
:107C300004E249501408000E4A540EE30101D451E5
:107C40000DE10A01D6514B6E4C6A4C3407E24B50A1
:107C50000C08000E4C5402E20CEC0EF0ECECC1F0FF
:107C600004E249503808000E4A540EE30101D45191
:107C70000FE10A01D6514B6E4C6A4C3409E24B506D
:107C80001408000E4C5404E20CEC0EF00CEC0EF058
:107C900015EC0EF01ED02FAA0DD021B61AD00E0E64
:107CA000E66E930EE66E020E02ECB7F01DEC05F0E8
:107CB000238A0FD021B00DD021B60BD03C0EE66E3A
:107CC000660EE66E010E02ECB7F033EC4AF035ECCE
:107CD00005F02D8E02011E0E206F1DAC66D007012F
:107CE000BA83B0EC07F001013B91129C3B51010BB0
:107CF00001E0128CE66A49EC27F0E552006E005074
:107D00000F0802E20F0E006E100E0002F3CF0EF20B
:107D1000B5EC22F01D9A050E07019D250201D880C1
:107D20000E5501E21D8A2A50800B13E10D5111E01E
:107D3000050E07019D5D02010E5D03E20DEC07F0EB
:107D40001D881D50100B31E01D50200B2EE002014C
:107D500009D02A50800B0AE11D50800B07E11D500D
:107D6000200B04E0FA0E0D6F1D981FD02ABE02D022
:107D70000AEC07F02BBA17D01E0EE66E050E8BEC40
:107D8000BCF0E66ECEECB9F00AE019C5C4F11AC534
:107D9000C5F11BC5C6F11CC5C7F11DC5C8F1AAC2F6
:107DA00024F10101269B010126891D50800B0DE164
:107DB00001012651100B01E17ED01F50080B01E19B
:107DC0007AD02050200B01E176D002011E0E206FE8
:107DD0001DAC02D0140E206F2BAA2FD01DBC16D0C4
:107DE00001014451630801E2446B800E241506E052
:107DF000FB0E245D03E2246B000E12D0800E2415CE
:107E000059E12451030856E2246B09D00101246B87
:107E10002AAE09D0050116514DE1320E166F010E42
:107E200050ECBFF047D0AD51030844E3010E50ECD5
:107E3000BFF00101140EAD6F3DD01E50400B03E0AA
:107E40000951010B37E11EAC02D0098101D0068334
:107E5000050147812B8C2C8A29ECB8F0D4C1E6FFB0
:107E60009FEC37F0E55275ECBEF01D50800B06E03C
:107E70000101245103E178EC2CF016D002016FAF20
:107E80000AD0BAC7E6FF76EC39F0E5520201AA51F2
:107E90000101242709D06F5107E0BAC7E6FF1FECA4
:107EA000BCF0AA510101245F02016F51DCE12D8277
:107EB0007EEC04F01D9E01012751100B4BE01F507A
:107EC000080B48E02050200B45E002011E0E206FF9
:107ED0001DAC02D0140E206F1EAC02D0098301D05D
:107EE0000683050147832B8CD5C1DFFF2C9A55EC07
:107EF000B9F0DFCFE6FF9FEC37F0E5527DECBEF046
:107F000002016FAF0DD0DF50C9ECB7F0EF50E66E55
:107F100076EC39F0E5520201AB51010125270CD076
:107F20006F510AE0DF50C9ECB7F0EF50E66E1FEC7E
:107F3000BCF0AB510101255F02016F51DFE12D82E1
:107F40006BECB9F024A606D00101010EAC6F07015D
:107F5000140E536F2BAC06D023ECC0F02B9C258263
:107F60002CAA238A0101279926992794E552B5EF77
:107F7000B6F03B0E00ECB8F00101320EAC6F2F886A
:107F800033C119F21200010137A70AD04D0E096E54
:107F90000F0EE66E100E0D03F350F8ECBDF010D08E
:107FA000030E096E0F0EE66E140EF8ECBDF02BEC0E
:107FB000B7F0030EE66E230EE66E230EE66E0A0E93
:107FC0002BECB7F0096A1200B9ECB6F0030E096E9B
:107FD000140EE66E000EE66E0A0E01ECC5F0040EFD
:107FE000E66E260EE66E0A0EE66E260EF3ECC1F085
:107FF000FE0EDB501EE0010137A70AD04D0E096EC0
:108000000F0EF8ECBDF0E66E100E0D03F3500ED01F
:108010000F0EF8ECBDF0E66E140EF3ECC1F0030E9B
:10802000E66E230EE66E0A0EE66E230EE66E18EC82
:10803000B7F0096AB5EFB6F0030E096EAA0EE66E48
:108040002A0EE66E0A0EE66E300EF1EFC5F0C2EFB4
:10805000C5F0010121A1B4EF44F0219102010F0705
:108060000F5101E0C4D0640E0F6F3D510CE03D5143
:10807000010803E3EEECB8F006E002013D073D51D4
:1080800002E1CBEC20F03196150E0101555D0BE0BD
:1080900002011651171103E01607000E175B165167
:1080A000171101E12F8C01018B5104E08B078B51DB
:1080B00001E13196020120510CE01F50080B09E04C
:1080C0002007205106E11DAC02D01D8E02D02DBE2E
:1080D0002D9E300E0401F75D06E10201066B076B71
:1080E000086B096B05D0340EF75D02E267EC90F087
:1080F000020119511BE00501105118E12750400BF6
:1081000015E119ECBEF012E1190719510FE10C50FD
:10811000006E555106E07F0E5515006E189A55BF3A
:10812000188A010EE66E005048ECBEF002015807B6
:1081300058510BE10101515102010B5D06E2410E64
:1081400000ECB8F00101AC69258EEEECB8F009E066
:1081500001019751010B05E0765103E13CECD7F0AA
:1081600002D0AEECD7F0ACECC0F011E01B50100B1D
:108170000EE12150020B09E0050ED45D06E0040E6D
:10818000D45D03E01E50200B02E1060104790101D9
:108190003851100B06E11350020B05E01950200B6B
:1081A00002E106010D752850400B01E0010E020F9F
:1081B000016E2850400B01E0010E050F026E0368AE
:1081C0001DAC08D0FCECC3F0EF7EFCECC3F0EF502C
:1081D000800B036E02012D5101E02D077A5104E05E
:1081E0002250100B01E17A07325101E03207DF51D2
:1081F00037E0DF07DF5134E1080E155C31E1215033
:10820000200B2EE00101AA512BE1258E2C9ECFECF4
:1082100087F02950100B1EE0C40EE66E010EDBEC59
:10822000BDF0E66ECEECB9F003E12B50200B12E06E
:108230001D8C01013B91129C0D0E55ECBBF0010110
:10824000C80EAC6F2A9E1D9E430EE66ED30E6BECDD
:10825000BDF006D0120E00ECB8F00101960EAC6F26
:108260000301D75117E0D707D75114E1000E0201DF
:10827000BE5DA30EBF59800EC059360EC15907E22C
:10828000D151BE27D251BF23000EC023C123030109
:108290000A0ED76F0201D75109E0D707D75106E17F
:1082A000D85102E1010ED86F35ECB0F01EAC09D008
:1082B0000201D507D55105E167EC90F00201030EEC
:1082C000D56F19ECBEF040E02050400B3DE0195056
:1082D000400B3AE0BAECBCF003E11950200B34E05B
:1082E00002013707000E385B1950200B0AE0F2EC50
:1082F000BCF009E1B9ECB9F004E10101E451100B63
:1083000002E1000E01D0010E0490E8B0048019ECE7
:10831000BEF003E00450010B17E0376B386B01012E
:10832000E49904A006D00201196B19C255F20AECB7
:108330005CF039EC09F00101B5A705D0249223BC0B
:108340002482E5ECBCF0209402013C5101E03C07A2
:10835000335101E03307315101E0310730510AE078
:108360003007305107E1D4ECC2F001E14A5002E09D
:1083700083EC0BF00201185109E01807185106E1CF
:108380004CECBBF00201D45101E1119410071051E3
:108390003FE1280E106F1AAC0FD031EC32F0D4C18F
:1083A00000F065EC32F00601017901A931D0D5C1A8
:1083B00000F065EC32F02CD01BA803D00601047944
:1083C00027D01CA206D00101E6B522D00601147107
:1083D0001FD01950200B06E001013851100B02E1AB
:1083E00006010D752450020B03E1BEECBEF010E057
:1083F000020130510DE1D4ECC2F001E14A5008E035
:108400002C50800B05E12C50400B02E1060101715C
:1084100002012B5101E02B070701A25105E0A20741
:10842000A25102E1B4ECBDF002012A5116E02A0784
:108430002A5113E16BECB7F003E161ECD6F00DD0FB
:1084400007019F51A01109E09F5101E09F07A05132
:1084500001E0A0070201020E2A6F020129510CE07F
:108460002907295109E1178E17901788080E156EF4
:108470002CAC02D0100E156E0101AE5169E0AE07B2
:10848000AE5166E11BECBDF0006E0201A95107E0A0
:10849000830E096EA9C201F04EEC34F0096AFF0E9A
:1084A0000201845D28E084C24FF0506A516ADD0EFB
:1084B000496E990E4A6E010E4B6EB9C14CF04D6A71
:1084C0004E6AD4ECC0F00900F5504F24F36E090059
:1084D000F5505020F46E0900F5505120E1ECC1F048
:1084E0000800F550006E0201842B005004E18469FD
:1084F0000101ADECC4F0005013E00101190EAE6FA4
:108500000050E66E62EC65F0E5520201A95102E00E
:10851000A92B1ED00101B22B000EB323B42318D017
:108520002850080B03E13050080B04E028960101A5
:10853000E8970ED00201A95105E0A96B0101FA0EDE
:10854000AC6F05D00101D890AC33D890AC33E8972C
:108550000201285104E02807285101E1259E2751F6
:1085600007E02707275104E10601416941C640F6AB
:108570000101AA510DE0AA07AA510AE1090E155CF2
:1085800007E13FECB9F004E10101FA0EAB6F1A8A82
:108590000101AB5101E0AB070701535101E0530763
:1085A00002012F5123E02F072F5120E1000E060179
:1085B000E76EBE19E8AE02D0BE3503D0E750D880D2
:1085C000BE5502E2BE0701D0BE2B000EE76EBF19FA
:1085D000E8AE02D0BF3503D0E750D880BF5502E2E5
:1085E000BF0701D0BF2B0201050E2F6F155105E00B
:1085F0001507155102E1FCEC5FF00201215124E066
:10860000210727AA21D020BC1AD01A50800B17E0CE
:10861000800E071414E02050010B11E1216B1A9E0B
:108620000A01DA8F82EC0AF091EC6AF01EAC03D0FA
:108630000201098902D00201068B0501478502016A
:10864000215102E1238A25820D5107E01D50400B84
:1086500004E00D070D5101E11D8E0501165101E0E9
:1086600016070201355105E03507355102E1F2ECFC
:1086700008F00201B05101E0B0072C5101E02C07D5
:108680000101AC5101E198D0AC07AC5101E094D0AC
:10869000B59DB59F2F98E4951C921B9830AC02D0E5
:1086A00043EC47F02FBAF2DA23BE84DA2582238A1C
:1086B000279820BA02D065EC22F0208A290E155C9A
:1086C00032E12150200B2FE00101AA512CE11DECD9
:1086D000BAF0930E491804E14A5002E136ECBFF0BB
:1086E00015683FECB9F002E11E8417D001013B711F
:1086F000129C3B51010B01E0128C41EC8AF0540EAC
:108700006FECB7F001013BA108D04B0EE66ECC0E2A
:10871000E66E52EC08F0E55204D0550EE66E45ECDC
:1087200022F0E5521A860101E8A90AD0E899E88703
:10873000920EE66E950EE66E010EA7ECB8F0E552CD
:108740002550040B39E00B0E155C36E12150200B4F
:1087500033E00101AA5130E120982594B59BB599E9
:10876000E67DE6AD1BD0E8A30AD06F0EE66EB30E31
:10877000E66E010E14ECB7F00101198F0AD0A10EBC
:10878000E66E950EE66E010EA7ECB8F0E55201011B
:10879000E887E883500EE66EC60E0CD0670EE66ED4
:1087A000B30EE66E010E14ECB7F00101198F500EF6
:1087B000E66E4E0E31ECB7F002011D5101E01D07CF
:1087C000045101E004071E5101E01E071F5101E0A2
:1087D0001F07345101E034070101AD5101E0AD073D
:1087E0000201235101E02307395101E039073A51D1
:1087F0001CE02150200B0AE1110EEFECC1F03AC24F
:108800003EF080ECC0F002E10601067B02013A076F
:108810002150200B05E02050400B02E073EC05F0E6
:1088200002013A5102E1BDEC04F0060143510AE0B5
:108830004307435102E15A0E436F25860F0E435DF5
:1088400001E225960201225108E02207225102E1AD
:10885000A0EC5FF002011E0E216F3B5110E0010100
:108860002651400B0CE102013B073B5108E144C19A
:1088700000F018869CEC87F00201010E246F0201C3
:1088800024513FE0240724513CE10101395103E028
:108890000901010EEB6F0901ED6B0201780E2C6FDF
:1088A0000101E78FDFECB2F00201186BD45101E156
:1088B00011944CECBBF020A204D0209271EC29F072
:1088C00011D035ECC0F0249C70EC13F0640EDDEC9C
:1088D000B6F03CECD7F0B2ECBCF004E0E851400B51
:1088E00001E0F9D918B002D0B4ECC4F0189002013C
:1088F00006891EAC02D0098709850501BF0E476FA6
:1089000048810201365104E03607365101E12582E3
:10891000255101E02507D65109E00501105106E176
:108920000201D607D65102E17EEC08F002011B518C
:1089300006E01B071B5103E1630E28ECB7F00201B0
:108940001C5106E01C071C5103E1B10E28ECB7F0E6
:1089500002011A5105E01A071A0502E156EC0EF061
:1089600002012E5101E02E07120006014F6B4FC687
:108970004EF64FC64DF64FC64CF64FC64BF612009C
:1089800002ECC1F0DE52010EDD6EFE0EDB501AE18C
:1089900087ECC4F0050EE66E200EDF24E66E4B0E6B
:1089A000E66E060E2BECB7F0050E0FECC6F0BA0E15
:1089B000E66E010E2BECB7F00F0EF9ECC3F0005091
:1089C000DF6E096A0101BA51630805E3BA510EE18D
:1089D000320EBB5D0BE2360E006E0DEC22F0FE0E89
:1089E000DB5001E1C2DF010EDB6A20D0FE0EDB505E
:1089F0001DE12C50800B07E0DF50090804E207015D
:108A0000BA9BB0EC07F0DFCFE6FFECEC2DF0E552BF
:108A100001018A51100B0AE00A0E445D07E23BECAB
:108A2000C5F0DFCFE6FF8EEC75F0E552020129516B
:108A300015E1640E0101445D0BE263ECB7F044C143
:108A40003EF031ECB9F00101166F300E3A2405D03A
:108A50004D0E166F030E4415310F176F016A050E88
:108A6000015C2FE25E0E496E9C0E4A6E010E4B6E4B
:108A70000150EA6A4B0FE96E060EEA22EFCF4CF086
:108A80004D6A60ECC2F0026E2D0E025C05E1010140
:108A9000B65102E1200E026E0201295110E1020ED0
:108AA00001241FECB9F002C0EFFF015008E12B9A3E
:108AB0002A0E025C04E12C50800B01E02B8A012A73
:108AC000CED70201295102E10101188F010EDB50BE
:108AD000D2ECBEF002E2E16AE552E16E4950B5EF38
:108AE000B6F00FECC0F0016E4451ADECB8F0050EDD
:108AF000E66E4B0EE66E060EE66E200E0124F1EFDA
:108B0000C5F00201050EB86FF00EB96FFA0EBA6F1C
:108B1000140EBB6FF00EBC6FFA0EBD6F1200016A2F
:108B20000101D45102E0010E016E0150A1ECB7F039
:108B3000EF50006ED2AD006A015063ECC2F0EF500E
:108B4000E66E0150A1ECB7F0010E77ECC6F0E66ED0
:108B50000050E66E250EC0ECB8F001011496D2511B
:108B6000400B01E014861200026A0101D45102E0B8
:108B7000010E026E025063ECC2F0EFCF49F0190E05
:108B800097ECB7F0D2ECBAF002E1200E1B6F4E0E5C
:108B9000186F520E196F8FEF45F0238E1F96B4EFAA
:108BA00045F024801F96F40E02EFBDF0249033921E
:108BB000C6EFB9F0239EC6EFB9F0020EE66EBD0E09
:108BC00022ECB7F00101D0BB0FD0BB0E28ECB7F000
:108BD000010EE66E200EE66EE66A2F0EE66E33ECB0
:108BE00013F0B7ECC5F039D0070E0201935D18E21F
:108BF0009351E824496E4A6AFF0E5AECC3F0E66EC0
:108C0000060ED8809355070DF3500A0FE66EBC0E82
:108C1000D3ECB6F0010EE66E200EE66EE66A16D0D4
:108C2000F30EE6ECBEF0BC0ED3ECB6F002019351AD
:108C30000A0802E2030E01D0010EE66E0F0ED88084
:108C400093550C0DF350E66E800EE66E2F0EC0ECC1
:108C5000B8F0B90EE66EF4EC12F0E552010114948E
:108C6000D051200B01E01484120002019329D2ECB0
:108C7000BAF002E1200E1B6F4E0E186F420E196FF4
:108C8000DDEF45F02F8A1F9635EF46F02F9AC6EF9D
:108C9000B9F00D5017E0B2ECBCF014E00501105132
:108CA00011E10D6A279A01013689200E1B5D05E04E
:108CB0001BC1E6FFDCEC0EF0E5521CC1E6FFDCEC6C
:108CC0000EF0E55212003BECC5F02BC1E6FF8EEC36
:108CD00075F0E552120027ECC6F0050EDF6E080EA7
:108CE000DF5C1DE2070EDF5C07E101011551800B1F
:108CF00003E0520E82ECB7F0DF509BECB7F057EC7C
:108D0000BFF00BE30050390808E3300E005C02E1CD
:108D1000540E006E005082ECB7F0DF2AE0D7E55227
:108D2000B5EFB6F02CEF0BF08CECCFF00A5018E05A
:108D30001F0E006E010196BB02D03F0E006E030EA7
:108D40000A5C02E02D0E006E4DECD5F001010E51D3
:108D500002E1100E0E6F002B8B0E006E56EC21F010
:108D60009CECCFF0E20E496E8E0E4A6E010E4B6EF9
:108D70000A502DECC6F017C1E6FF16C1E6FF3AEC2B
:108D800008F0E552E552010136AD02D08EECD3F089
:108D90001200328000680DEC22F079ECC0F01F96D2
:108DA000C3DFB5EF32F032902CEC0BF0F5D92F98F1
:108DB00012002BECC1F0140DBFECB7F094ECC0F036
:108DC00005E0DFECB8F0230ED3ECB6F00AEC12F0BD
:108DD000140EDDECB6F0B5EFB6F0B9ECB6F0B6C2F5
:108DE00000F0FE0EDB5001E1006AB7C2E6FF005062
:108DF000E66E240ED3ECB6F0B5EFB6F01450100BBF
:108E000001E0010E496E3350010B495C01E1120093
:108E100082C789F7339014A80ED0338014A80BD0E2
:108E200014AA03D082C7E6FF07D0E66AC2DFE55284
:108E3000010EE66E04D0E66ABCDFE552E66ACDDFDD
:108E4000E552120007018251140DBFECB7F086EC19
:108E5000BAF019C116F11AC117F11BC118F11CC1E2
:108E600019F10101200E1A6F480E1B6F5A0E1C6F6C
:108E7000300E165D02E1200E166FFEEF46F0308CCC
:108E80001F9622EF47F0309C2F980101AC6B23987E
:108E9000B59F2CEF0BF00101AC5103E02450080BFF
:108EA00003E0B551200B01E02F880050ACECB9F085
:108EB0000101AC5106E02F50100B03E1FA0EAC6F2C
:108EC00024861200010E0701D89054375537E80662
:108ED000FBE121AC02D0070154810D0E0701565D64
:108EE00001E2562B1200219C8450020B01E0218CE0
:108EF00007014C5111E121AC78D04C2B010E546F7D
:108F0000556B566F3098576F4F51FE0BE8424F2507
:108F10004E6F010121931200010121A366D021931C
:108F200007014C0562E121BC52D030A84DD00C0E97
:108F3000565D47E2D89055335433006A5F0E005CAB
:108F40001BE2FC0E4B6E8D0E4C6E010E4D6E0050F2
:108F50004E6E50ECB8F0545149180CE155514A1876
:108F600009E1200E0026610E005C02E3200E005E87
:108F700092DF02D0002AE2D75F0E005C22E10701F7
:108F80001F0E541901E155510AE01D0E541901E15B
:108F9000555105E0EF0E541905E1555103E1200E3E
:108FA000006E79DFFF0E0701541902E1020E551918
:108FB00006E0B50E541905E1030E551902E11FEC48
:108FC00065F007014C6B1200308862EF47F07ADFE2
:108FD00030A804D00701010E576F06D00701572BA8
:108FE00057510C0801E24C6B3098120007AE06D0C6
:108FF0008450020B02E0219C01D0218C07014C51CE
:1090000010E121BC75D00101219307014D6B07AE22
:109010006FD0020E4C274F51FE0BE8424F254E6F8A
:1090200012004C050BE14C2B4FC74EF70101219369
:1090300021AC5ED00701080E4C6F1200010121A384
:1090400057D02193070E07014C5D46E14C6B21ACD4
:1090500040D00101AC5103E02450080B03E0B551AE
:10906000200B01E02F88E60E496E9B0E4A6E010E22
:109070004B6E07014D515025B4ECC5F0006E810ECA
:10908000005C02E1506B1BD0800E005C03E1200EFF
:10909000506F15D00D0E005C03E00A0E005C02E17B
:1090A000200E0BD00B0E005C02E12A0E06D00A0E39
:1090B000005C05E0005003E00050ACECB9F00101A9
:1090C000AC5109E02F50100B06E1FA0EAC6F24866C
:1090D0001200080E4C6F1200080E4C5D04E121AC2A
:1090E00007D04C6B12004D914D4321BC4D894C2B48
:1090F00012009CECCFF08AECB8F016E19CECC0F0CA
:1091000006E0600E496EB30E4A6E010E05D0ED0EFC
:10911000496EC00E4A6E010E4B6E04ECB8F04BC0A7
:10912000E6FF50ECB7F018D0EAC600F00050020895
:1091300002E2020E006EBA0E496E8E0E4A6E010EEB
:109140004B6E00502DECC6F00601EA51020804E215
:10915000EA05300F01011C6F54EC1BF0E4EC0DF03C
:10916000006E00500A01D65D04E200C0D6FA3AEC67
:10917000B9F012000101D45105E1308479ECC0F05E
:109180001F9603D000682FEC22F079EF48F030945E
:109190002CEC0BF0CCEF48F0040EE66EEA0EE66E17
:1091A000060EE66EA00EF3ECC1F0140E016E3CC18B
:1091B00000F00BEF34F0E6ECC0F0E0C649F0E1C699
:1091C0004AF0FFECC3F0060139ECC0F00CE3DEC658
:1091D0004BF0DFC64CF0D8904B364C36E0514B5C30
:1091E000E1514C5820E2DE51E0250E6EDF51E121C5
:1091F0000F6ECEECBEF0FDECBDF0030EC0ECBBF08C
:10920000E804FCE149500601E25F4A50E35B9CEC54
:10921000BAF0030EC0ECBBF0E804FCE149500601D3
:10922000E2274A50E323DEC6E0F6DFC6E1F6FDECB6
:10923000BDF0FFECC3F0FFECC3F039ECC0F00BE382
:10924000FDECBDF0C0ECBBF0C0ECBBF04950DE5D06
:109250004A50DF5902E2DF6A09D0E251DE5DE35194
:10926000DF5902E2010E01D0020EDF6EFDECBDF00F
:10927000FFECC3F04950E225E46F4A50E321E56F6B
:10928000DF50E552B5EFB6F01DBC1200219C8450B2
:10929000020B01E0218C21AC03D002016C2B02D027
:1092A00002016D2B1F9E0601E65109E121AC4BD056
:1092B000010EE66FDE6BDF6BE76BE86B44D0E60513
:1092C00015E121BC40D0020EE66F75DF006E005044
:1092D0000BE0070E0601E85D07E2E82BE791E743A4
:1092E0000050010801E2E78F06011FD0020EE65D83
:1092F0002AE121AC1DD0E2C64BF0E3C64CF0030ED0
:109300000F0B05E0D8904C324B32E806FBE106012A
:109310004B50E25D496E4C50E3594A6E4950DE5D58
:109320004A50DF590EE2010EE66FDE6BDF6B0BD0A9
:10933000E451E425496EE551E5214A6E39ECC0F06F
:1093400002E2030EE66F030EE65D43E1E791E743B9
:10935000E78F070ED880E855016E0150010600091D
:1093600003E0E791E743F9D7780EE75D30E20101CA
:10937000AC5103E02450080B03E0B551200B01E091
:109380002F88E7C6E6FF3CEC04F0E552006E200EA5
:10939000005C03E300506E0802E22A0E0BD0298A1B
:1093A0000050ACECB9F00601DE51E45DDF51E55947
:1093B00003E2200EACECB9F0299A0101AC5107E0B0
:1093C0002F50100B04E12486FA0EAC6F3086060194
:1093D000E66B1F8E12000101E583D45102E154DFD8
:1093E00007D01F9EB6ECBCF002E07DDD01D0FEDDB3
:1093F0000101E5931200800E071420E02A50020BB1
:109400001DE12050200B1AE00201A95117E10101D2
:10941000D45104E10601EA51010806E38AECB8F0F0
:109420000DE19CECC0F00AE02A0E0101B51506E141
:10943000290E155C10E12150200B0DE0800E071461
:1094400009E1CFECB7F006E00601EC5103E00201C0
:109450002D5101E0000C010C0201395103E1120E03
:109460006FECB7F01200E6ECC0F066C1DFFF21A29E
:1094700005D0010166515FECC4F0DF5E1EBCDF6AFF
:10948000DFCFE6FF720E22ECB7F0308002010783D7
:1094900034B0E2DFE552B5EFB6F0E6ECC0F067C1FC
:1094A000DFFFDFCFE6FF710E22ECB7F00201078786
:1094B000E552B5EFB6F002ECC1F0D00EDE6E070E4D
:1094C000DD6EA4ECC0F004E28C0EDE6E0A0EDD6EE2
:1094D000090E2B5D0DE25F51020B0AE02250100BCA
:1094E00007E13450800B04E102010B517D0804E2D6
:1094F000B80EDE6E0B0EDD6ED7ECB7F002E3000E99
:1095000001D0010ED2ECBEF002E2E16AE552E16E5A
:109510004950B5EFB6F002ECC1F064EC0FF029EC65
:1095200040F0EEECBCF002E056DF02D01FBE1F9E02
:109530002450200B06E00201245103E199ECB2F023
:10954000249A02012B5102E0AAEC36F00101B75136
:1095500011E1E66A49EC27F0E552006E1DAC93EF8D
:1095600051F007019D51F00BE83A9D5D00249D6F7D
:1095700093EF51F0B7050DE1AFEC66F0B5EC22F0DA
:1095800020EC15F01E92E8A093EF51F01E8293EFAD
:1095900051F0020EB75D04E1C2ECCFF093EF51F051
:1095A000030EB75D07E12EB493EF51F0BCECD4F09D
:1095B00093EF51F0040EB75D01E0A0D002012551F8
:1095C00002E093EF51F01750100B06E11750010B1A
:1095D00003E11750200B02E0000E01D0010E229093
:1095E000E8B0228021AA44D05EECBFF022A036D0A1
:1095F0000101AA512AE1090E155C17E13FECB9F00F
:1096000014E10101AB510BE1A00E176ECBEC07F09A
:1096100000093CE0B2ECBCF039E11A8637D01650B4
:1096200035E1AB6B900E176E1FD0165002E1010EA4
:1096300001D0100E8009176ECBEC07F0000926E070
:10964000B2ECBCF023E11A8421D016501FE1AB6BC1
:10965000ABC1AAF1810E176E219A06D0165016E101
:109660002250010B13E1219A0201020E256F0ED048
:1096700031B40CD0E66ADBEC36F0E552000906E0C6
:1096800031840201020E256F07AE256B3150040BA9
:1096900002E193EF51F00201255102E093EF51F006
:1096A0003194DF6B5EECBFF0165002E193EF51F0A6
:1096B0009BEC04F00201A96B0101280EAA6F0201C4
:1096C000020E256F218A176A1650156ECBEC07F033
:1096D00000090BE001013651800B07E00201355112
:1096E00004E1040E006EC3EC6AF028B602D001015A
:1096F000AE6BD9EC0AF02A8493EF51F0050EB75DFA
:1097000028E1EEECB8F016E01B50080B13E172EC08
:10971000B8F010E2BFECC5F072ECB8F00BE2BFECB1
:10972000C5F072ECB8F006E202011E0E186F4CECA8
:10973000BBF0118401012651100B02E093EF51F0B0
:109740002751100B02E093EF51F0AAEC36F093EFA3
:1097500051F0060EB75D07E120AA93EF51F077ECC8
:1097600006F093EF51F0070EB75D02E193EF51F071
:10977000080EB75D01E072D32550800B0AE00201AC
:10978000285107E1020E87ECC2F002011E0E286F7D
:10979000259E25AC03D03FECBBF0259C25AA03D029
:1097A000F2EC08F0259A01013651800B1BE0020112
:1097B000355118E11AA404D0040E87ECC2F01A94B3
:1097C0001AA604D0070E87ECC2F01A961AA804D085
:1097D000060E87ECC2F01A981AAA04D0050E87EC80
:1097E000C2F01A9A0101B5BDB9D0B5A979D020AEA1
:1097F0000FD0AD5101E08DD02BA805D00B50E66EF7
:10980000FCEC37F003D0E66AACECABF0E55281D06B
:10981000E8AD12D026AD06D0100E156E26BF156A23
:1098200059EC8AF02550020B04E101012651400B4E
:1098300014E063EC46F011D032A012D026AD0DD06A
:10984000B6ECBCF002E00101967BD9EC0AF011EC19
:109850001BF054EC1BF094EC46F00101269D37D030
:109860002C50400B03E12C50800B33E026AD51D03F
:10987000FEEC06F00101B6511DE1630EE66E440EEA
:10988000E66E010EE66E2EEC6FF0B7ECC5F044C14B
:109890000CF202013B6B95ECBCF0000917E02C5078
:1098A000800B14E001018E51100B10E10201100E2B
:1098B0003B6F0CD0290EE66EB6054A6A4B0F496E17
:1098C000060E32ECC3F03EECC0F0E5520101AD6B88
:1098D00020D021B61ED059C200F00DEC22F019D0D4
:1098E000B5A305D025A215D02592228212D0B5A10C
:1098F00010D025A206D025922BC1E6FFECEC2DF06E
:10990000E5520201215105E11A50400B02E1B5EC8C
:1099100032F0A0EC11F0006EFF0820E0540E005C65
:1099200007E18CECCFF0220E006E0DEC22F016D089
:10993000180E005C03E16DECB1F010D0FF0E015C7D
:109940000DE08CECCFF00101140E116F0D0E126FB3
:10995000050E006F0150006E4DECD5F00101B5BF52
:1099600065D2B5ABE8D02CA603D0E9EC38F048D2EC
:1099700030AC03D022EC47F043D22FAA05D023AA63
:109980003FD235EC46F006D023AE08D023AA38D219
:10999000B4EC45F049EC46F0239A97D019A803D0CF
:1099A00031ECC0F0AFD03050040B1BE0D45119E1C2
:1099B00027AD0DD0010E0D6E27BF0D680A0EE66EA5
:1099C000EA0EE66E060E02ECB7F03AECB9F0235060
:1099D000200B04E101012751400B3DE079EC48F0F8
:1099E0003AD032A03CD027AD14D0010E0D6E27BF67
:1099F0000D680AC006F1030E2AECBCF006C10AF09D
:109A000004ECC3F00A5018ECC2F0CCEC48F00501AD
:109A100047852350200B03E0B2ECBCF004E00101C9
:109A20002751400B18E0D9EC0AF0C0ECC4F094ECDC
:109A300046F002010881050147871EAC02D00201F1
:109A400009851F50020B05E0B6ECBCF002E071EC9A
:109A5000BDF027EC33F00101279D239A37D02C501D
:109A6000400B03E12C50800B33E023AA04D0239A4F
:109A70003EECC0F047D027ADC3D1279D010E0D6E3F
:109A800027BF0D68006A050EE66E0050E66EB60E42
:109A9000E66E010E07ECB7F00601030E426F0101FE
:109AA000B6510EE0B629496E010E495204E0E8466F
:109AB000FE0B4906FCE10601426F1E0E436F02D009
:109AC00071EC45F03EECC0F0E5520101AD6B98D170
:109AD00020AE1AD0AD5101E093D109ECB8F001E00D
:109AE0008FD10B50016E2250100B03E13450800BCC
:109AF00002E02BEC5EF0006A005015ECBAF035EC99
:109B000038F0E552E5527CD121B67AD15AC200F044
:109B100018EC22F09D0E02015A5D01E071D16BEC50
:109B2000B7F006E0CFECB7F003E10101320E23D02D
:109B30000101330E20D0B5B363D1B5A71ED01950A3
:109B4000400B04E01950040B01E05AD19CECCFF01B
:109B50000A0E006E6BEC21F00101040E016F03C7C9
:109B600000F019AC02D0A3EC04F06AECD5F019AC0B
:109B700047D10101200E1A6F43D13BAB2BD1080E08
:109B8000006E0050D880765501E2766B27AD1CD070
:109B9000279D010E0D6E27BF0D680050E66E760EF4
:109BA000E66E010E02ECB7F0020E0101765D03E0F5
:109BB000050E765D05E127BF02D0762B01D0760732
:109BC0000601426B0101AD6BAD5101E019D120508E
:109BD000200B01E115D10201A95101E011D1070EBD
:109BE0000101765D41E19CECCFF062EC13F00101E4
:109BF0002B0E166F00010FAE0BD001012D0E166F4C
:109C0000FF0ED8800E560F56010E0E26000E0F22A4
:109C1000E70E42ECC0F002E247ECC0F00E500F102D
:109C200003E10101200E166F9CECBAF015ECBEF0BA
:109C3000C5ECC2F039C049F03AC04AF04950006E54
:109C40000101012B6AECD5F08EEC04F0300F01011C
:109C5000176F300E175D02E1200E176F198F640E1B
:109C60001A6F420E1B6F83D0060E765D1EE19CECD0
:109C7000CFF05FEC13F086ECBAF00101410E166FE5
:109C8000460E176F560E186F300E195D01E0B8D0F2
:109C9000200E196F300E1A5D01E0B2D0B6ECC3F0A1
:109CA00001E0AED0200E1B6FABD0040E765D03E05A
:109CB000050E765D46E19CECCFF00498050E01019F
:109CC000765D09E14F0E166F530E176F430E186F36
:109CD00085ECBEF018D0500E166F410E176F048839
:109CE00009ECB8F006E00101580E186FEAC900F05F
:109CF0000DD00101490E186F0A0E496E4A6AA5C7B8
:109D00003DF0A6C73EF00BECC6F0006E049000AE2E
:109D100002D0006C04800101030E016F8BECBBF0DC
:109D200004A002D02D0E196F430E1C6F04B8188FBB
:109D3000050E765D65E14E0E1A6F2F0E1B6F410EFC
:109D400017D0760517E19CECCFF05C0EE66EB30EF3
:109D5000E66E010E7FECC6F00BC200F06AECD5F0A7
:109D6000300E0101195D02E1200E196F1B8F560E96
:109D70001C6F46D0080E765D22E1FAECB8F0E66A78
:109D8000F8EC21F0E552300E0101165D02E1200EE3
:109D9000166F410E1B6F480E1C6FA80ED8800E5414
:109DA000610E0F5409E2016B560EE66EB30EE66EBD
:109DB000010EE66E50ECB7F00101188F21D0030EB2
:109DC000765D03E1CCEC0EF01BD0765119E182EC0C
:109DD000D7F016D0020119510BE02750400B10E1CB
:109DE000140E0101AC5D0CE23B0E00ECB8F008D0A3
:109DF0000101B5A105D023AA03D0239A99EC2EF036
:109E0000A0EC11F0006EFF0811E0540E005C0AE1B6
:109E100079ECC0F04E0EE66EB30EE66E010E7FECEE
:109E2000C6F004D00050006E18EC22F00101AD51D4
:109E300001E079D2140EAD6F0201565101E05607D0
:109E4000020E685D01E06FD22B0E0101B95D04E0E6
:109E5000080EB95D01E067D2258265D2090EB75DB3
:109E60000AE106015051515D01E15DD250C651F643
:109E70007FEC36F058D20A0EB75D05E1A8ECD3F0BE
:109E800092ECD3F050D20B0EB75D01E04CD2B8513A
:109E900001E143D2B80548E124ECBDF001E33DD235
:109EA00024ECBDF001E339D21B50080B01E035D2A0
:109EB000A4ECC0F012E2770E00ECB8F08EECD3F018
:109EC00098ECC5F0420EE66EB30EE66E010EE66E3D
:109ED0004CEC11F0E552E5521FD2C80EFAECC5F079
:109EE00018EC10F00701A80E3FECC5F00DE2310EA2
:109EF000E66EB30EE66E010EEDECB7F0290EE66EDF
:109F0000B30EE66E010EA2D0760E3FECC5F001E373
:109F100004D2180EE66EB30EE66E010EEDECB7F04D
:109F2000770E00ECB8F0CED0020EB85D01E0CDD0D7
:109F300080EC0EF0EEECB8F001E18FD02050040B75
:109F400001E08BD02050400B01E087D05E0EDE6E2A
:109F5000010EDD6E25ECBAF004E2900EDE6E010E0D
:109F6000DD6EE6A504D0F40EDE6E010EDD6E21B2CC
:109F700004D0640EDE26000EDD22D7ECB7F001E33C
:109F8000CCD11B50080B01E0C8D180EC0EF0ECECFA
:109F9000C3F0D7ECB7F001E3C0D180EC0EF0050EB2
:109FA000DDECB6F0D7ECB7F001E3B7D12CA609D0C1
:109FB0006BECB7F003E0CFECB7F00AE022ECC4F0B2
:109FC00007D0010166519AECBCF0665F33EC4AF0B1
:109FD000460EFAECC5F0D7ECB7F001E39ED1170EB0
:109FE0006FECB7F02CA609D06BECB7F003E0CFEC28
:109FF000B7F011E022ECC4F00ED0000EE66EB30E06
:10A00000E66E010EEDECB7F0010166515FECC4F0B5
:10A01000665F33EC4AF0960EFAECC5F0BBECC3F089
:10A02000320EB0ECC0F00201D151495CD2514A5815
:10A0300001E373D1ED0EE66EB20EE66E010EEDECAD
:10A04000B7F0E50EE66EB20EE66E010E03ECBFF061
:10A0500038ECBEF03DEC0FF060D15BEC4AF000094B
:10A0600001E15BD11B50080B01E057D180EC0EF0F1
:10A070005BEC4AF0000901E150D1170E44ECC5F049
:10A08000A4ECC0F009E2D70EE66EB20EE66E010E49
:10A09000EDECB7F0320E0BD048511E080CE2C90EA1
:10A0A000E66EB20EE66E010EEDECB7F01E0E0BEC96
:10A0B000BAF0640EF0D0B60EE66EB20EE66E010E89
:10A0C000EDECB7F083ECBAF028D1030EB85D45E1B2
:10A0D000060150932450020B12E11F50020B04E0C2
:10A0E00055EC25F0000909E01250080B03E112506D
:10A0F000040B05E0D8ECBFF002E0060150832450C9
:10A10000020B13E1BEECBEF010E1020130510DE193
:10A11000D4ECC2F001E14A5008E02C50800B05E17C
:10A120002C50400B02E1060101812050200B01E17F
:10A13000F4D02D50100B01E0F0D08050100B01E056
:10A14000ECD08050100B01E0E8D007012A0E246FFC
:10A15000390EE66E61EC11F0DFD0040EB85D01E05F
:10A16000A6D01F50080B01E1A0D0EEECB8F001E141
:10A170009CD0DEECBEF001E098D0BAECBCF001E07F
:10A1800094D00498049A6BECB7F058E0D70EB6EC74
:10A19000B9F01DECBEF011E1F6ECC3F00EE249504F
:10A1A0009808000E4A5409E20050ECECBFF004E6B7
:10A1B000D20E4B5C000E4C5818E3E851800B3DE08A
:10A1C00000504D6E4E6AD8904E5004E6980E4D5C8D
:10A1D000000E4E580AE300504F6E506A50342DE284
:10A1E0004F50D208000E505428E259ECC1F025E03F
:10A1F0000101E87F76EC15F09BEC04F02050200B79
:10A200001AE06BECB7F017E011ECBEF014E0AE0E04
:10A21000E66EB20EE66E010E14ECB7F00101E8BF77
:10A2200007D0A60EE66EB20EE66E010E14ECB7F085
:10A230000101960EAC6F048A2A9C04881DECBEF0C6
:10A2400034E10450200B31E15651040B2EE004B8E8
:10A2500004D0D70E006E25EC21F02ABC12D0E5EC1C
:10A26000C2F004E68F0E495C000E4A5856E259ECE3
:10A27000C1F053E02A8C50EC0AF00201090E336F52
:10A280004CD0F6ECC3F00BE249508F08000E4A5454
:10A2900006E22A9C140EE66E4FEC1DF03DD0020142
:10A2A00033513BE150EC0AF038D02A9C36D0050EF1
:10A2B000B85D33E1A30EB6ECB9F00101E5A105D01C
:10A2C0000050E66E1CEC6BF0E55204902150020B3E
:10A2D00001E00480C00E005C02E2219204D0005034
:10A2E000F00801E221822150020B02E08F9001D0A0
:10A2F0008F800450010B496E2150020B01E0010ECA
:10A30000495C0BE09BEC04F0B9EC13F033EC4AF041
:10A310003AECB9F037ECC5F0E5520101B82BB85171
:10A32000050801E2B86B0101B72BB7510B0801E238
:10A33000B76B020EE15C02E2E16AE552E16EB5EF55
:10A34000B6F0016A750E015C0CE2A30E496E9A0E1E
:10A350004A6E010E4B6E29ECC4F02DECBEF0012AC2
:10A36000F1D71200026A400E025C08E2B00E02242D
:10A37000016E320E2DECBEF0022AF5D71200C0ECB1
:10A38000C3F0060F016E040E15ECBAF08D0EE66EEA
:10A39000020E2BECB7F0096AB5EFB6F0C0ECC3F0D3
:10A3A000060F016E040EE66E8D0EE66E020E54EC84
:10A3B000C3F0B5EFB6F0C0ECC3F00A0F016E020EA9
:10A3C00015ECBAF0910EE66E020E2BECB7F0096AAE
:10A3D000B5EFB6F0C0ECC3F00A0F016E020EE66EE8
:10A3E000910EE66E020E54ECC3F0B5EFB6F0E6EC5B
:10A3F000C0F0340E65ECBFF0010E096EDF6A100E7E
:10A40000DF5C3AE2026A100E025C34E240ECC2F019
:10A4100003E0050E025C06E1DF50E824820FE4EC65
:10A42000B8F0006E020403E0060E025C07E1DF50A4
:10A43000E824820F010FE4ECB8F0006E020EDF5C3E
:10A4400003E3030EDF5C0AE10A0E025C02E1110E77
:10A45000006E0B0E025C02E1240E006E0C0E025C1C
:10A4600005E10A0EDF5C02E11B0E006E0BEC34F01E
:10A47000022AC9D7DF2AC3D7020E096EDF6A090E86
:10A48000DF5C12E2026A100E025C0CE240ECC2F0E9
:10A4900003E0050E025C02E11C0E006E0BEC34F0D2
:10A4A000022AF1D7DF2AEBD7096A4BDFDF6A200ED9
:10A4B000DF5C09E2100E006E800EDF24016E0BECF3
:10A4C00034F0DF2AF4D7DF6A0B0EDF5C03E24ADFE9
:10A4D000DF2AFAD7DF6A090EDF5C3AE2DF28006E76
:10A4E0000038F00B006E090E0012DFCFE6FF42ECE1
:10A4F0000AF0E552E2ECB6F000C0EFFFE2ECB6F095
:10A50000EE52090EEF6EE2ECB6F0020EF2ECB8F08D
:10A510002C0EEF6EE2ECB6F0030EF2ECB8F0010E8A
:10A52000EF6EE2ECB6F0040EE7ECC1F0050EE7ECDE
:10A53000C1F0070EE7ECC1F0080EE7ECC1F0060E23
:10A54000E7ECC1F0090EF2ECB8F0EF6ADF2AC3D7EE
:10A5500026D830D8DF6A060EDF5C14E2DF5002E155
:10A56000030E01D0010EE66EDF50C9ECB7F0BCEC73
:10A57000B8F0DF0403E0020EDF5C02E10701B585FD
:10A58000DF2AE9D7C2ECC5F0FD0E016EDB0E2DEC23
:10A59000BEF00101010EB56FE552B5EFB6F0020E47
:10A5A000096E5A0EE66E000EE66E030EE66EA20E01
:10A5B000F1EFC5F07BECC6F0030E096EFE0E70ECF9
:10A5C000C6F0850E005C02E0010EDF6E2D0E65EC1C
:10A5D000BFF0140E05ECBDF0000EE66E0A0E92EC14
:10A5E000B7F00A0E05ECBDF0CA0EE66E0A0E92EC4C
:10A5F000B7F0040E05ECBDF0260EE66E0A0E92ECE6
:10A60000B7F0DF501DE00F0E05ECBDF0140EE66E46
:10A610000A0E92ECB7F0030E05ECBDF0230EE66EC9
:10A620000A0E92ECB7F00A012D0E1B6F1BCA1AFA24
:10A630001BCA19FA410E206F20CA1FFA20CA1EFA3F
:10A640000A01D46BDA6BDA81D56B380ED66F040E43
:10A65000D86F3C0ED96F190ED76F016A020E015CDC
:10A660000CE20150050D48ECC5F0000EE9260A0E7B
:10A67000EA22360EEF6E012AF1D70101D46B050EE6
:10A68000D45D1AE20701010EAD6FFF0EAD5D11E062
:10A69000C0EC10F0CBECBBF0A7ECB9F019ECC0F0BB
:10A6A0000701AD5160ECC3F051ECBAF00701AD0702
:10A6B000ECD70101D42BE3D70701AD6B0101D46BBB
:10A6C000DFCFE6FFE4EC3FF0E5521CEC40F0030E78
:10A6D000096EFE0E016E850E2DECBEF0096AE55284
:10A6E000B5EFB6F00490049201013EB104803EB390
:10A6F00004820450010B02E08E8E01D08E9E4051E8
:10A70000E8240A0FE66EE66A9BECE3F0E552E552B8
:10A710000C0EBB6E006A01013E5104E1100E3F03B6
:10A72000F350006E0050BC6E1200B9ECB6F02FEC86
:10A73000C1F068ECE4F0E552000902E0C69EF7D7EC
:10A74000B5EFB6F0C79EC698C78C1200C78EC688F4
:10A75000C78C1200D9CFE6FFE1CFD9FF030EE12667
:10A7600035EC0EF0E668930EE66EF4ECE3F0E5529D
:10A77000E552AA9EC26A000000000000000000002E
:10A780008A8A209A3386278AD7EC10F00601B66BA6
:10A79000B76B70EC0BF024ECB2F099ECB2F092686D
:10A7A0008F0EE66EE66815ECE2F0E552E552CF0E4C
:10A7B000E66EE66866ECE3F0E552E552050EE66EFD
:10A7C00086ECE4F0E5520101010E3E6F0101030E3B
:10A7D0003F6F0101020E406F85DFE668870EE66E6F
:10A7E000CAECE3F0E552E552B09E0201320E116F61
:10A7F000000EA56EA26E9F6EA282D08E010EC26E5A
:10A80000C16A0A0EC06E0F01DF0E256F0F01F70E31
:10A81000246F0F01E00E236FDB0E006E25EC21F09C
:10A8200000C04AF5010EDB6A100EF36E010EDBCF9D
:10A83000F4FFF350F45C28E2890E496E9C0E4A6ED8
:10A84000010E4B6E010EDBCF4CF04D6A4E6A495043
:10A850004C24F36E4A504D20F46E4B504E20F86E4F
:10A86000F4CFF7FFF3CFF6FF0800F550E66E010EC8
:10A87000DB50EA6AC50FE96E060EEA22E552E750A0
:10A88000EF6E010EDB2AD0D70101266B0101269164
:10A890008850010B01E02681010126938850020BAC
:10A8A00001E02683F28E060150697FEC36F01CEC45
:10A8B000D5F001017E0EB26F940EB36F010EB46F2E
:10A8C000020184690601506B7FEC36F00101010E34
:10A8D000B56F8CECCFF09CECCFF004EC65F006018A
:10A8E00017810601416941C640F60601426B138A91
:10A8F000128011881182138613880A01380ED66FD0
:10A900000A01010ED76FCAEC15F092ECD3F0E4EC1B
:10A910001BF0010EE66EDBEC36F0E552166E010E12
:10A92000E66EDBEC36F0E552000901E0F8D7640E84
:10A93000E66EBAECE4F0E5521C9E99ECB2F0096ABE
:10A94000FC0E016E4EEC34F0001CDF6EFC0E016E4E
:10A95000DF50006E0BEC34F0FC0E016E4EEC34F068
:10A96000DF50005C06E01E0EE66E61EC11F0E55271
:10A970004ED0830E096EFC0E016E4EEC34F0001CBE
:10A98000DF6EFC0E016EDF50006E0BEC34F0FC0E3F
:10A99000016E4EEC34F0096ADF50005C06E0210ED7
:10A9A000E66E61EC11F0E55232D0FD0E016E4EEC18
:10A9B00034F0DB0E005C03E1200E165C02E117DDD3
:10A9C0001ED0020E016E4EEC34F000C02AF1370E9C
:10A9D000016E4EEC34F000C05FF1110E016E4EECD2
:10A9E00034F000C039F1120E016E4EEC34F000C0AC
:10A9F0003AF10F0E016E4EEC34F000C037F1E00E6C
:10AA0000016E4EEC34F00050800801E2ABDC07012F
:10AA1000B00E606F040E616F07018969D9EC0AF00E
:10AA2000016A090E015C0DE28050100B0AE18050B2
:10AA3000100B07E1280EE66EBAECE4F0E552012AAD
:10AA4000F0D7090E015C08E307012B0E246F390EC5
:10AA5000E66E61EC11F0E552C80EE66EBAECE4F079
:10AA6000E55299ECB2F0AAEC36F01F860001116AAB
:10AA7000126A136A146A800E076E176A219A750E9D
:10AA8000E66EE66A280EE66E010EE66E79EC34F0AC
:10AA9000E552E552E552E552020E096E5A0EE66E97
:10AAA000A20EE66E000EE66E030EE66E79EC34F052
:10AAB000E552E552E552E552030E096E2A0EE66EA6
:10AAC000E66A000EE66E0A0EE66E79EC34F0E552A8
:10AAD000E552E552E552AA0EE66E300EE66E2A0EFB
:10AAE000E66E0A0EE66E79EC34F0E552E552E55278
:10AAF000E552FE0E016E4EEC34F0096A850E005CE4
:10AB000001E058DD060EE66EF00EE66EB40EE66E5F
:10AB1000070EE66E79EC34F0E552E552E552E55267
:10AB2000040EE66EA00EE66EEA0EE66E060EE66E09
:10AB300079EC34F0E552E552E552E5520601EA516E
:10AB40000A0802E20601EA6B0601EC51010802E282
:10AB50000601EC6B200EE66E800EE66E620EE66E6F
:10AB6000070EE66E79EC34F0E552E552E552E55217
:10AB7000830E096EF90E016E4EEC34F000C071F2D6
:10AB800002017151C80803E20201C80E716FF80E8C
:10AB9000016E4EEC34F0339A6E0E005C01E1338AA4
:10ABA000DF0E016E4EEC34F00101E391720E005C99
:10ABB00002E10101E3817E0E096E0C0EE66EE66A8B
:10ABC000B60EE66E020EE66E79EC34F0E552E55212
:10ABD000E552E552096A01019C51040802E20101B3
:10ABE0009C6B1B0E165C10E10101368F0101368D46
:10ABF0000101369136833695010EE66EDBEC36F0B8
:10AC0000E552000901E0F8D7090E165C09E11B8640
:10AC1000010EE66EDBEC36F0E552000901E0F8D7F4
:10AC2000FEEC0AF001018DAB06D001013C9F010151
:10AC30003C9D01013B9F01013781010196890A0179
:10AC4000D56901013895FF0E01019A5D04E0FF0E00
:10AC500001019B5D04E101019B6B9BC19AF1800E98
:10AC60000201BE1908E1910EBF1905E1B70EC01926
:10AC700002E1360EC11905E10201BE6BBF6BC06B6C
:10AC8000C16BE90E0101E76E9919E8AE02D0E73415
:10AC900002D0E750995D0CE3170E0101E76E991998
:10ACA000E8AE02D0993503D0E750D880995502E23A
:10ACB0000101996B0A0E0101985D04E301019851AD
:10ACC000640803E201011E0E986F01010101575152
:10ACD000200B07E0010101015751100B02E10101B6
:10ACE000579BB6C201F0BDC202F0FF0E015C07E047
:10ACF000015005E0FF0E025C02E0025008E1020193
:10AD00007C0EB66F0201FA0EB76F81EC45F00101BF
:10AD10008351050802E20101836B0101845102089D
:10AD200002E20101846B0101425104E00101425140
:10AD3000020803E20101020E426F01016D51230876
:10AD400003E201010A0E6D6F01015F8D0101505197
:10AD500004E0010150510D0803E20101010E506FA2
:10AD60000601EA510A0804E20601EA6B0601EB6BF0
:10AD700001018E9D0101578301012E6B460E0101D9
:10AD8000525D04E301015251730803E20101540EC4
:10AD9000526F640E01014A5D0BE301014A51496E95
:10ADA0004A6A4A3404E24950B408000E4A5403E2A5
:10ADB00001018C0E4A6F01015551150804E3030E81
:10ADC0000101555D03E20101150E556F040E0101ED
:10ADD000475D04E301014751080803E20101050E44
:10ADE000476F01017D51496E4A6AD8904A5004E686
:10ADF000C80E495C000E4A5803E20101CF0E7D6F78
:10AE000001014D51496E4A6A4A3404E2495096089C
:10AE1000000E4A5403E201018C0E4D6F01014C51AA
:10AE2000320803E20101280E4C6F01014B51496EBB
:10AE30004A6A4A3404E24950C808000E4A5402E201
:10AE400001014B6B0A0E0101415D04E30101415117
:10AE50000F0803E201010F0E416F01013551500847
:10AE600003E20101010E356F01012851280803E2B8
:10AE70000101280E286F550E01014E5D07E0680E96
:10AE800001014E5D03E00101680E4E6FFF0E0101EE
:10AE9000695D03E00101695109E10101400E696F3B
:10AEA000780E6A6F7D0E6B6F010E6C6F010177512A
:10AEB000010802E20101776B010166513C0802E2E0
:10AEC0000101666B010167513C0802E20101676BF9
:10AED00001016851280802E20101686B01010101CA
:10AEE0008D51020B05E101013A5102E001018D8310
:10AEF00001016151030802E20101616BFF0E0101D2
:10AF00005F5D02E101015F6B01017151496E4A6AA7
:10AF10004A3404E24950C808000E4A5403E20101D1
:10AF2000C80E716F01017351496E4A6A4A3404E2D6
:10AF30004950C808000E4A5403E20101280E736FFD
:10AF400001017251496E4A6A4A3404E24950C80804
:10AF5000000E4A5403E201010C0E726F010175519B
:10AF6000496E4A6A4A3404E24950C808000E4A54FD
:10AF700003E201011E0E756F01013151010803E268
:10AF80000101010E316F3C0E0101E76E7C19E8AE44
:10AF900002D07C3503D0E750D8807C550BE3C40E3B
:10AFA0000101E76E7C19E8AE02D0E73402D0E75029
:10AFB0007C5D02E201017C6B010186510F0802E217
:10AFC0000101866B01017B510F0802E201017B6BDD
:10AFD00001016E513C0802E201016E6B01016F51EB
:10AFE0003C0802E201016F6B0601EB511E0802E210
:10AFF0000601EB6B0601ED511E0802E20601ED6B46
:10B0000001017F51640803E201011E0E7F6F0101FF
:10B010002951496E4A6AD8904A5004E6280E495C84
:10B02000000E4A580BE3010129514B6E4C6A4C3417
:10B0300004E24B505008000E4C5403E201013C0E58
:10B04000296F01018551C80802E20101856B0101E8
:10B050008551640803E20101640E856F0201875186
:10B0600004E002018751330803E202010D0E876FED
:10B0700001018751780803E20101640E876F010125
:10B0800093510C0803E20101060E936F01019551E3
:10B090000C0803E20101060E956F010188511E089C
:10B0A00002E20101886B01018AAF02D001018A6BC3
:10B0B00001018DAF02D001018D6B01018EAF03D074
:10B0C0000101060E8E6F010196AF03D00101600EE3
:10B0D000966F1E0E0101895D04E301018951280864
:10B0E00005E201011E0E896F01018A9101018B5158
:10B0F0000A0802E201018B6B01017A51190804E28E
:10B1000001017A6B01018A930101705104E0010190
:10B1100070511E0803E201011E0E706F01013E51C5
:10B12000010803E20101010E3E6F1E0EE66EE4EC23
:10B1300010F0E552000909E00101010E3E6F010126
:10B14000030E3F6F0101020E406F72EC53F0318825
:10B1500005014B69F2EC08F00101E383010129517B
:10B16000E8240301B86F17EC1DF0300E01018425AF
:10B170000401F76F020E0101845D03E10401340E46
:10B18000F76F59EC96F004013B0EFE6F0501106B52
:10B1900010C512F510C511F50501800E156F44ECB0
:10B1A000B6F0F3CF49F0F4CF4AF049504A1005E128
:10B1B0002A0EE66E61EC11F0E55207013C0E826F3B
:10B1C0000101D56BD5C1D4F10701AD6B91EC6AF0EB
:10B1D0000701BA81D9EC0AF03FEC1AF033EC4AF0DF
:10B1E0000101389564EC1CF07FDA99ECB2F018ECB0
:10B1F00010F0F3CF0EF0F4CF0FF01F0E0E5C010E27
:10B200000F5806E3D30ED8800E54020E0F5411E2ED
:10B210000EC049F00FC04AF0040ED8904A324932AD
:10B22000E804FBE149C024F75A0EE66E61EC11F028
:10B23000E552550EE66E020EE66E400EE66EFAEC34
:10B24000B1F0E552E552E552020EE66E400EE66EB2
:10B2500036ECB2F0E552E552006E550E005C08E0A7
:10B2600000C024F75D0EE66E61EC11F0E5521ED0D1
:10B27000B70EE66E020EE66E400EE66EFAECB1F028
:10B28000E552E552E552020EE66E400EE66E36ECF1
:10B29000B2F0E552E552006EB70E005C07E000C068
:10B2A00024F75D0EE66E61EC11F0E552E66A020EDF
:10B2B000E66E400EE66EFAECB1F0E552E552E5526C
:10B2C0000201410E976FE1EC04F0010197A111D04A
:10B2D0007DECD6F0000905E07CECD6F03CECD7F034
:10B2E00008D00701010E246F1B0EE66E61EC11F011
:10B2F000E55244ECABF02B96229601013A51010144
:10B30000941101E17CD0150EE66E020EE66E440E3D
:10B31000E66EFAECB1F0E552E552E5522A0EE66E21
:10B32000020EE66E460EE66EFAECB1F0E552E5521C
:10B33000E552020EE66E440EE66E36ECB2F0E552D1
:10B34000E552150802E1000E01D0010E006E00501A
:10B3500014E001013A5108E000C024F7600EE66EE7
:10B3600061EC11F0E55208D00701030E246F240EA2
:10B37000E66E61EC11F0E55242D001013A5118E05D
:10B38000020EE66E460EE66E36ECB2F0E552E5527F
:10B390002A0802E1000E01D0010E006E005008E004
:10B3A00000C024F7630EE66E61EC11F0E55227D081
:10B3B000120EE66E440EE66E36ECB2F0E552E55241
:10B3C000006EC00E001601013A510CE0005008E07A
:10B3D00000C024F77E0EE66E61EC11F0E55201D05C
:10B3E0002B860DD0C00E005C09E00701040E246F0F
:10B3F000240EE66E61EC11F0E55201D022861B921C
:10B400002580E66818EC30F0E55239C1E6FF1AEC09
:10B41000B1F0E5520101B581219401013BBB06D099
:10B4200006015085060150977FEC36F00101D4519A
:10B4300004E0030E0101D45D04E10A01D46B149C05
:10B4400004D00A01020ED46F148C87D971EC29F054
:10B450000201320E246F0101100EB96F0501010EB9
:10B46000176F0901020EE56F0201582B03010A0E46
:10B47000D76F0201320E226F88EC87F09BEC04F04C
:10B480000201D35108080AE2D7EC10F0D3C224F726
:10B49000270EE66E61EC11F0E5521B860D0EE66E8E
:10B4A000DCEC11F0E552870B006E005008E000C0A4
:10B4B00024F7390EE66E61EC11F0E55214D011EC70
:10B4C0001CF03B0E0E5C000E0F5806E3E60ED88013
:10B4D0000E54030E0F5407E20EC024F7540EE66E0E
:10B4E00061EC11F0E552030EE15C02E2E16AE55223
:10B4F000E16EE552E7CFD9FF12003C0E0101B95DC4
:10B5000003E3B951400801E2000C010C01013B7B4F
:10B51000279D256B1DD8238A258201013BBB13D0B3
:10B5200009014F0EE66F460EE76F060150A707D0E0
:10B530000901560EE66F420EE76F010136890601DA
:10B54000436B43C642F601013BBB0480FDEF07F0AD
:10B5500006015097509501013BBB07D021B403D0A1
:10B560000601508512000601508712000A01D651CB
:10B57000F3EFC3F0D4C100F0005003E0030E005C11
:10B5800033E100500EE10101D07D0901430EE66F69
:10B590000101D0AD02D076ECBDF00101D0AD20D0DC
:10B5A00010D021ECBAF00FE00101D0750901440E72
:10B5B000E66F0101D0A502D076ECBDF00101D0A567
:10B5C0000FD004800DD00101CF750901440EE66F44
:10B5D0000101CFA502D076ECBDF00101CFB504800A
:10B5E000FDEC07F0D4EFBFF0000403E0020E005CB6
:10B5F00016E1C0EC10F0000402E1020E01D0010ED1
:10B60000006E09014C0EE66F020E005C03E104803F
:10B61000550EE66FFDEC07F000C0D4F167D81200BC
:10B620000101325103E16BECB7F002E0000E01D0F2
:10B63000010E1492E8B014826BECB7F003E1B4ECA5
:10B64000C0F00CE16BECB7F007E0CFECB7F004E131
:10B6500001013B51800B02E1000E01D0010E14905C
:10B66000E8B0148012006BECB7F00BE0E2ECBEF037
:10B6700008E109EC1CF0050804E03CECC2F001E133
:10B68000000C010CB8ECC0F003E001018151120084
:10B69000010178511200B8ECC0F003E001018251C1
:10B6A0001200010179511200B9ECB6F0B8ECC0F00B
:10B6B00005E0FE0EDB500101816F04D0FE0EDB5071
:10B6C0000101786FB5EFB6F0B9ECB6F0B8ECC0F0A8
:10B6D00005E0FE0EDB500101826F04D0FE0EDB5050
:10B6E0000101796FB5EFB6F039EFC3F021902792E1
:10B6F000D4C100F00050800802E2050E006E060E74
:10B70000005C01E3006A000402E10101CF91020E36
:10B71000005C02E10101CF8100C0D4F1248A20BE87
:10B7200003D035ECC0F002D027EC33F0CBEF20F0A3
:10B73000E6ECC0F0030EDF6E01014951496E4A6A22
:10B74000B00E3D6E040E3E6E0BECC6F0D880DF549A
:10B750000201506FE552B5EFB6F0E6ECC0F026B04E
:10B760000ED0320EDF6E080E0101495D02E2080EB6
:10B77000496FDF50D880495502E2DFCF49F1D8DF69
:10B78000E552B5EFB6F050C2B0F122AE34D0006A47
:10B7900001013D510C0803E3070E3D5D02E20C0E72
:10B7A0003D6F070E3D5D4D6E4E6A020150510DEC2E
:10B7B000B8F0006E13ECC6F00101B0514B6E4C6A4C
:10B7C000FF0ED8804B56000E4C564A504C18E8AE2F
:10B7D00002D04C3404D04B50495C4C504A580BE2D8
:10B7E0000050D880B05507E223A003D00050B02706
:10B7F00002D00050B05FBAECBCF008E102012D515C
:10B800000601EA1106E02750400B03E11D92B0EC5F
:10B8100035F01200050E55ECBBF0580E86EFBCF06B
:10B82000F9DF258E1200180E6FECB7F0010136AD6E
:10B8300003D0580E86EFBCF0258E1200B9ECB6F09E
:10B84000050EE1261FA20FD0BFC1DFFF010EC0C150
:10B85000DBFF020EC1C1DBFF030EC2C1DBFF040E22
:10B86000C3C1DBFF0ED0BAC1DFFF010EBBC1DBFFDE
:10B87000020EBCC1DBFF030EBDC1DBFF040EBEC167
:10B88000DBFF030EDF5C42E3DF50180807E21C0E0B
:10B89000DF5C04E201019651010B24E10101E5BDE9
:10B8A00007D0DF50180815E21C0EDF5C12E22ED024
:10B8B000190EDF5C2BE01A0EDF5C04E1010EDB5099
:10B8C0005F0824E31B0EDF5C04E1290E7EECB9F077
:10B8D0001DE32B50100B06E12E50800B03E02B5183
:10B8E000090802E2F36A17D0630EE66E020EE66EF6
:10B8F000C4ECC3F0CEECB9F009E1C4ECC3F05E0EC9
:10B90000E66E020EE66ECEECB9F004E08CDF010EBE
:10B91000F36E01D0F36AF46A050EE15C02E2E16ABB
:10B92000E552E16EB5EFB6F065C301F022A802D092
:10B9300078C301F00E0E015C01E2010C100E015CF7
:10B9400001E2020C120E015C01E2030C140E015C18
:10B9500001E2040C160E015C01E2050C1B0E015CF9
:10B9600001E2060C220E015C01E2070C080C2BEC34
:10B97000C1F06CECC6F0F00801E2006A0050B5EFCF
:10B98000B6F0B9ECB6F02FECC1F0F1DFE552E5EC22
:10B99000C2F004E6BE0E495C000E4A5809E26E0E83
:10B9A000496E960E4A6E010E4B6E27ECC2F001D026
:10B9B000B00E0E6E0F6AE5ECC2F004E6AA0E495C0A
:10B9C000000E4A580BE2C40E496E950E4A6E010EE7
:10B9D0004B6E27ECC2F00101D86F02D00101D8698B
:10B9E000D96BB5EFB6F0E6ECC0F0049034B8048043
:10B9F000B30E016E0150C9ECC3F009ECB8F012E0CF
:10BA00000E500101D66FD76BB30EC9ECC3F00E50C8
:10BA10008AECC2F00101D6274A50D723D6C10EF0D6
:10BA2000D7C10FF00101E6A502D0D86BD96BD8C100
:10BA300061F3D9C162F334B80BD113A64DD00B50CA
:10BA4000016E2250100B03E13450800B02E003D949
:10BA500013D009ECB8F010E00701BD514D6E4E6AED
:10BA60000B500DECB8F0016E2050800B05E0090181
:10BA7000EC5102E0ECC901F0050E0124496E0A0EFA
:10BA800097ECB7F0016E015005E12250400B02E047
:10BA9000010E016E6BECB7F003E03450400B05E093
:10BAA00001C09FF702010A0E08D007019F51015CF7
:10BAB00005E301C09FF702010C0E2A6F35DF070175
:10BAC000A06F2B50100B03E1040E0B5C01E2A06B86
:10BAD0003FECBCF08CECBAF019ECBAF004800050EA
:10BAE00009E03450400B06E1030E005C04E1020E55
:10BAF0000A5C01E10490070E016E04A004D0090E57
:10BB00004BECB8F0016E0F0E01140201736F070EBB
:10BB1000731701380F0B016E04A0016A13A408D03B
:10BB2000020EE66E73C2E6FF0150E66E8CECBAF0D0
:10BB300052C100F00101E6A502D04AC100F013ECA9
:10BB4000C6F085ECB8F033ECC2F0C8ECC2F015ECEE
:10BB5000BEF04DECC5F00E500B6E19ECBAF0040EB1
:10BB6000005C0BE0000409E0020E005C06E0030E3E
:10BB7000005C0AE1020E0A5C07E00201AF51D880C6
:10BB80000B5402E20BC0AFF20101E6A507D003019E
:10BB9000636B646B676B686B656B5AD0B70EC9ECEF
:10BBA000C3F0D8C163F3D9C164F303016151635D8C
:10BBB0006251645906E3010E6325616F000E642132
:10BBC000626F61516325676F62516421686F6751CD
:10BBD0006725496E685168214A6E67C34BF068C398
:10BBE0004CF0030ED8904B364C36E804FBE149503C
:10BBF0004B240301676F4A504C20686F6351615DAD
:10BC0000496E625164554A6E33ECC2F067C33DF031
:10BC100068C33EF015ECE5F03DC067F33EC068F345
:10BC200067C365F367C349F068C34AF04B6A4C6A5F
:10BC30004C34000E4C1809E6D880FF0E4954000E13
:10BC40004A54000E4B54000E4C5402E20301656945
:10BC5000E552B5EFB6F048C101F02B50100B05E1ED
:10BC600009ECB8F002E0D9C201F0120019ECBAF008
:10BC700000500DE03450400B0AE1050E005C07E077
:10BC8000030E005C03E1020E0A5C01E0000C010CF3
:10BC90000482ECDF000901E00492348604A23496A9
:10BCA0003498A1DE34B8120019ECBAF00498049666
:10BCB000030E005C01E10486000403E0020E005C58
:10BCC00001E104882250400B01E1FCD02250100B0E
:10BCD00001E0F8D03450800B01E0F4D03350080B71
:10BCE00001E1F0D002011D5101E0ECD01950010B2F
:10BCF00001E1E8D004820494B9DF000901E0049274
:10BD0000040E005C01E10484A6DF01505FECC4F086
:10BD1000026E63ECB7F001C03EF06FECE5F03EC0A0
:10BD200007F1020E0101075D02E2020E076F0751E3
:10BD30000A0802E20A0E076F0450040B07E0020132
:10BD4000735104E1D8900132D89001320490205010
:10BD5000800B33E00901ED5130E009ECB8F02DE043
:10BD60000901EE51020829E2030E006EEE51190896
:10BD700002E2020E006EEE51280802E2010E006E91
:10BD8000EDA104D000508DECBEF00480020E09013C
:10BD9000ED150FE013ECC6F002010051495C0151B2
:10BDA0004A5807E200508AECC2F0005F4A50015B3B
:10BDB0000480040E0901ED1776D001500B5C42E2BD
:10BDC0000201880E005D130E01596DE203016C0E35
:10BDD000635D000E645967E204B20AD00B50015C47
:10BDE0000E6E0F6A0E50020100270F5001235AD029
:10BDF00002011E5158E10A0E1E6F0150AF5D20E294
:10BE0000AF5103E1735101081BE204A802D0020EF6
:10BE10001E6F0450080B0FE0030E0A5C03E0735121
:10BE2000010809E2010107518DECBEF01F5107E046
:10BE30001E911E4304D0020E0027000E0123048031
:10BE4000AF6B31D00150D8800B542DE2010E036E40
:10BE500004A208D007C103F004A804D0030E030213
:10BE6000F3CF03F003500E6E0F6A0450020B06E08E
:10BE70000450080B0DE002011F510AE001500B5C59
:10BE8000496E4A6A33ECC2F085ECB8F0C8ECC2F0F7
:10BE9000020100510E5C01510F5805E20E50005F87
:10BEA0000F50015B048004A00DD002010251001963
:10BEB00002E10351011906E011EC0AF000C202F29E
:10BEC00001C203F20201205102E00F0E206F1200A6
:10BED0007BECC6F0000E00092DE11750010B03E0CA
:10BEE000200E155C27E01950200B12E102011951B8
:10BEF0000FE1230E155C1EE00B0E155C1BE0090E16
:10BF0000155C18E0090E155C15E0220E155C12E0B8
:10BF1000BCECC0F004E091EC87F000090BE120508C
:10BF2000800B06E10201685103E03250200B02E071
:10BF3000000E01D0010EDF6EDF50E552B5EFB6F016
:10BF4000030EE66E85EC13F0E5528A868C9469EC5C
:10BF500015F06BECB7F003E03450400B11E08FECC0
:10BF600009F000090DE00AEC07F07EEC13F06F0E0B
:10BF700028ECB7F0C80E35ECBBF00DEC07F002D0A2
:10BF80007EEC13F0060150917FEF36F05BC248F172
:10BF90005CC200F25DC201F211EC0AF053EC1FF03A
:10BFA000E66AF6ECBCF0239612000101B05103E101
:10BFB0002B820850076E2050010B12E06BECB7F09B
:10BFC0000FE11750800B03E025ECBEF006E0205097
:10BFD000040B06E1B9ECB9F003E02CD913EC67F0DF
:10BFE00012000101050EAF6F2050010B04E0195043
:10BFF000020B01E0AF6B12001FECC5F001013951DB
:10C000002BE105C2DFFF19ECACF0DF500201055D4A
:10C0100023E0010E69C3DBFF020E6AC3DBFF030EE0
:10C020006BC3DBFF010EE66EBEECACF0E552010E19
:10C03000DB500301695D08E1020EDB506A5D04E13B
:10C04000030EDB506B5D08E068ECABF099ECB2F0EE
:10C050001C820101960EAC6F040EE15C02E2E16A03
:10C06000E552E16EB5EFB6F00201185107E0186B2A
:10C070004CECBBF00201D45101E111946BECB7F030
:10C0800009E12050010B06E1B4ECC0F003E12050BF
:10C09000800B08E0BAECBCF005E11E50400B02E159
:10C0A000228CD18022BC06D0E66AE66A740ED3ECFC
:10C0B000B6F019D009EC1CF0050813E13350080B59
:10C0C00010E000C249F001C24AF0030E0F0B04E079
:10C0D000C0ECBBF0E806FCE149500201005F4A50A9
:10C0E000015B11EC0AF002010A0E1E6FAF6B20AE6D
:10C0F0001C84C80E1F6F77EC13F0780E006E005092
:10C1000035ECBBF01DEC15F00201226B8A96320E65
:10C1100035ECBBF055ECC1F014E12B50080B11E0ED
:10C120002250100B0EE101013A050BE06BECB7F069
:10C1300007E12050800B04E102011E0E156F01D0B3
:10C140005BDF2050800B0EE12050010B0BE16BEC0C
:10C15000B7F008E03450400B05E102012D5102E038
:10C16000050110511DAC02D039EC0AF0208C31824F
:10C17000D5CA85F219ECBAF0360E026E380E036E8F
:10C18000BAC17DF2C6ECC4F03EC07EF249EC2AF0A2
:10C19000BAC17BF2C6ECC4F03EC07CF21FA20AD04A
:10C1A000BFC17BF263ECB7F0C0C13EF06FECE5F0CD
:10C1B0003EC07CF222AC06D00701098F919A8C8494
:10C1C00064ECB2F02F8EC0EC2CF00201FA0E236F5B
:10C1D000238A2582319222AC02D04CECC0F0B5EC1F
:10C1E00032F021AE11D0219E46EC09F017ECC3F0DD
:10C1F00019ECC1F009E019ECC1F006E019ECC1F04E
:10C2000003E039EC09F016D81200E6ECC0F00501A5
:10C2100023072451EA6A270FE96E050EEA22EFCFC1
:10C22000DFFF242B24511F0801E2246BDF50E5526D
:10C23000B5EFB6F081EC1DF00201196B19C255F291
:10C24000C8ECBDF007E0200E01011C5D03E0200EEC
:10C25000ACECB9F00101B06B006AC3EF6AF04B0EB1
:10C26000026E140E0301655D08E30A0E01012B5DE9
:10C270001BE11E0E0301655D17E2100E01012B5D2F
:10C2800013E22B50100B03E0640E485D0EE02B50C0
:10C29000100B0AE13C0E485D08E0020E395D04E136
:10C2A0005A0E0224485D01E0000C010C7BECC6F044
:10C2B0001B50080B0AE13FECB9F009E1340E010113
:10C2C000B95D03E03A0EB95D02E1000E36D001011E
:10C2D000815102E0825104E1450E15ECB8F0DF2AED
:10C2E0000101785102E0795104E1480E15ECB8F0F3
:10C2F000DF2AB5DF00091CE16AEC2FF0000906E037
:10C300003C0E15ECB8F0D1ECBCF0DF2A7FEC2FF03E
:10C31000000907E03F0E15ECB8F00201916B926B3B
:10C32000DF2A0701BC5104E1420E15ECB8F0DF2A08
:10C33000DF5002E07FDF2094DF50E552B5EFB6F02A
:10C3400025ECBAF002E27B51120086511200E6ECB5
:10C35000C0F00750DF6E27AA03D002011E0E216F26
:10C36000050110510201191103E13751381109E09B
:10C370001D50040B0FE01D50080B0CE01E50010B6C
:10C3800009E01750800B08E02750200B05E105015C
:10C39000105102E04FDF45D2075021E127BA04D007
:10C3A0003FECBBF0020E56D081DF000901E039D22C
:10C3B0000201245101E035D220B002D055DE0AD06E
:10C3C0002D5108E00501105105E1BEECBEF002E17F
:10C3D0003FECBBF0B5DF050DF3CFAFF1CBD00704D9
:10C3E00018E10101AF5101E018D21F9C55ECC1F0DA
:10C3F00002E01F8C05D0BEECBEF002E16AEC09F051
:10C400000101280EAF6F20AE02D0050EB06F072AD3
:10C4100016D0020E075C15E10201155102E01E0E56
:10C42000156F27BA06D00101B05101E0F6D10850CE
:10C4300028D10101AF5101E12BDC74EC09F0B5DD2D
:10C44000ECD1030E075C3CE127BA06D0006AC3ECCE
:10C450006AF0070E076EE5D12BA218D05BC1AFF1D1
:10C460000101B05105E06CDF050DF3500101AF276C
:10C470002B922050010B04E01950020B01E0AF6B2E
:10C4800002012D5103E0006AC3EC6AF00101AF51D3
:10C4900006E06BECB7F00FE03450400B0CE11F509E
:10C4A000400B05E102012D5102E16FEC09F00101A1
:10C4B000280EAF6FE5D026B8B0D148EC5EF0ADD114
:10C4C000050E075C2EE10101AF5101E0A6D1072A5C
:10C4D000269820B0A2D11C0E016E32DFE824012480
:10C4E000006E0201765107E00050765D04E2090E0D
:10C4F000076E268892D131820701099F918A64ECE8
:10C50000B2F0209C85C2D5FA23ECC0F06BECB7F0FA
:10C5100003E03450400B03E00101050EAF6F319290
:10C520007CD1060E075C28E10101AF5101E075D115
:10C5300020B01ED02650100B0DE1325109E06BECFB
:10C54000B7F003E03450400B03E0B4ECC0F002E17C
:10C55000F7DC0ED032C122F226A80AD0F1DE9EEC22
:10C56000C3F0006E00500201225D02E200C022F220
:10C570000201566B072A51D1070E075C24E1010125
:10C58000B0510FE117AE0BD025ECBEF003E03EEC4E
:10C5900088F005D0C0EC09F0000901E0179E0850B2
:10C5A000076E02012D5101E038D12A5106E03450C6
:10C5B000400B03E13FECBCF003D0E66AE66AE66AB2
:10C5C0001BEC24F047D0080E075C4BE10101B05191
:10C5D00006E01D50040B03E01D50080B02E108505B
:10C5E000076E02012D5101E118D148EC5EF074ECA8
:10C5F00009F002012E5101E010D1A2EC0CF000096B
:10C6000001E10BD10501020E266F235111E0FDDD82
:10C61000006E020E0A5C02E1005010D0016A0501B2
:10C62000235102E0F2DD016E005015ECBAF00ED09D
:10C63000105114E1020E0A5C07E1030EE66E150EBE
:10C64000E66E24EC13F007D0E66AE66A160EE66E94
:10C650002AEC13F0E552E552E552DFD002012D6BD2
:10C66000DCD0090E075C28E1020176417F0B7625BC
:10C670000101D880B15507E20201766B76C2B1F1B3
:10C68000050E076ECAD01EB0C8D0010EB16F320EB3
:10C69000AF6F010E076E6BECB7F003E002012D5196
:10C6A00008E0BEECBEF005E12750200B02E13FECB4
:10C6B000BBF00B0E086EB1D00A0E075C06E121BA82
:10C6C0009FD0179E0B0E076E9DD00B0E075C01E0EE
:10C6D0009CD01750800B39E12050010B06E0205010
:10C6E000040B03E1B9ECB9F030E16BECB7F003E017
:10C6F0003450400B0CE02050800B09E11E50010B20
:10C7000006E01D50040B03E01D50080B1EE16BEC0E
:10C71000B7F00CE03450400B09E12050040B06E167
:10C72000B9ECB9F003E0F2ECBCF00FE02050800B64
:10C7300009E01D50040B09E01D50080B06E0B9ECA0
:10C74000B9F003E055ECC1F051E017AE0ED025EC86
:10C75000BEF005E03EEC88F0000907E162D0C0ECD5
:10C7600009F0000902E0179E5CD06BECB7F023E003
:10C770003450400B20E1CFECB7F01DE119AA06D0F0
:10C7800039EC09F0E6EC06F087EC19F0BAECBCF0F5
:10C790000AE01950400B07E0249223BC248239ECB4
:10C7A00009F0E5ECBCF00101885105E088C1E6FF25
:10C7B0004FEC1DF0E552B1C176F20101B15102E03A
:10C7C000010EB16F26A802D048EC5EF007019D6B08
:10C7D000030E076E800E086E2050800B03E1175089
:10C7E000800B08E020940C0E086E04D022A802D022
:10C7F00087ECADF00101AF5105E12650100B02E1CD
:10C8000048EC5EF074EC09F008D00C0E075C05E112
:10C8100021BA03D0F2EC89F007D8DF50075C01E0C1
:10C820001C8CE552B5EFB6F020AECFD01D50040BF6
:10C83000FDE01D50080BFAE02A840101B59B238A14
:10C84000B59925829D510BE01FA203D09DC1D5F162
:10C8500002D09DC1D4F149EC2AF076EC5BF0225075
:10C86000100B03E13450800B04E0C6EC5FF0349E03
:10C8700087D0F5DC000974E009ECB8F071E1FBEC5D
:10C88000BFF000C20EF001C20FF00EC04DF00FC09D
:10C890004EF04F6A506A51ECC5F079ECB7F04DC0DC
:10C8A00040F04EC041F04FC042F050C043F02EEC7B
:10C8B000E3F037C02EF738C02FF739C030F73AC051
:10C8C00031F763ECB7F00BC23EF0EFECC3F0006E53
:10C8D000005037ECB7F0C40E406E160E416E020EDB
:10C8E000426E436A2EC73BF02FC73CF030C73DF085
:10C8F00031C73EF044ECE4F03BC02EF73CC02FF7CC
:10C900003DC030F73EC031F7005037ECB7F048C1BA
:10C9100049F037ECC1F044ECE4F03EC0EDFF3DC01F
:10C92000EDFF3CC0EDFF3BC0EFFF07012E512F1183
:10C93000301131110CE0DC0E2E5D000E2F59000E6F
:10C940003059000E315903E22EC700F007D02EC730
:10C9500024F74B0E15ECB8F0DC0E006E0BEC34F047
:10C9600018A804D0C6EC5FF018980AD00901EC5161
:10C9700007E009ECB8F004E00BC0D9F20901ED6B57
:10C98000209E33A403D027EC33F005D0010EE66ED1
:10C99000C5EC32F0E5522298D5ECB9F0CBEC20F0A2
:10C9A000010136BF04D0050E87ECC2F00ED036ADC3
:10C9B0000CD0E385E783E795E7970601FB29FC6F39
:10C9C00065C3E6FF71EC08F0E552800E076E1200B9
:10C9D0002F50100B04E00101E851080B13E0070190
:10C9E000535110E10101B551200B0CE13B51200BDB
:10C9F0000AE03FECB9F007E0A95105E10101E85177
:10CA0000080B01E1000C010C070EE66EE66A200E31
:10CA1000E66E440EE66E060EE66EFBECE1F0050EE9
:10CA2000E15E120045C644F646C645F647C646F6E0
:10CA300048C647F649C648F64AC649F6120049C6EE
:10CA40004AF648C649F647C648F646C647F645C6BA
:10CA500046F644C645F60601200E446F1200B9ECB6
:10CA6000B6F031AA02D007ECBFF00101E551020B8C
:10CA70000CE0280E0901BB5D08E2BB51BB2BEA6A42
:10CA8000930FE96E090E94ECC3F00101E851200BFD
:10CA90000CE0280E0901E45D08E2E451E42BEA6AA7
:10CAA000BC0FE96E090E94ECC3F0B5EFB6F0B9EC2B
:10CAB000B6F00101E8B704D02FECC1F003D8E5527D
:10CAC000B5EFB6F002ECC1F0010EDB6A1A50010BB3
:10CAD0000AE0800E45ECB7F004E2FE0EDB502008C1
:10CAE00002E11A905CD09EDFFE0EDBCF4AF6DB50EF
:10CAF000800804E0850E45ECB7F003E30601200E44
:10CB000021D0FE0EDB50300803E10601630E1AD07F
:10CB10002950200B1CE02850080B19E1DF6A150E84
:10CB2000DF5C15E2A0ECC4F00FE1DE52010EDD6E19
:10CB3000DF2AD9ECB9F006014A6F74DFDF2AD9EC9D
:10CB4000B9F006014A6F03D0030EDF26E8D73FECA9
:10CB5000B9F012E0010EDB5004E049C6E6FF7FDFCA
:10CB6000E5524AC600F0630E005C02E1300E006E32
:10CB70000050E66E74DFE5522BDF000910E0C4ECD4
:10CB8000BBF044C616F145C617F146C618F147C6B4
:10CB900019F148C61AF149C61BF14AC61CF1020E2A
:10CBA000E15C02E2E16AE552E16EB5EFB6F0E6EC77
:10CBB000C0F00750DF6E2392100E075C13E11C0ECD
:10CBC000076E02015151010B03E11D50040B02E1FC
:10CBD000110E92D05151040B27E11D50080B01E0BA
:10CBE000B3D022D0110E075C09E12380228E02010E
:10CBF000080E516F2382076A120EA5D0120E075C31
:10CC000006E123902382030E076E130E9CD0130EB1
:10CC1000075C0CE11C0E076E02015151040B04E18C
:10CC20001D50080B01E090D0140E66D0140E075C66
:10CC300010E12380228E180E076E1D50040B01E0B8
:10CC400083D01D50080B01E07FD02382076A150EA8
:10CC50007AD0150E075C0CE101012AAF03D0020166
:10CC6000020E516F229E2382020E076E160E6BD0AB
:10CC7000160E075C05E12382020E076E170E63D0C5
:10CC8000180E075C07E10201020E516F2382076A4A
:10CC9000190E59D0190E075C06E1229E2382020E5E
:10CCA000076E1A0E50D01A0E075C05E12382020EA1
:10CCB000076E1B0E48D0170E075C08E101012ABF62
:10CCC00003D00201020E516F1B0E16D01B0E075C23
:10CCD00005E12390228E2382030E33D01C0E075CC5
:10CCE00033E12390800E076E02015151010B03E1E5
:10CCF0001D50040B03E1110E076E26D034AC0BD08F
:10CD000009EC1CF0010802E1520E01D0500E28EC93
:10CD1000B7F0349C19D01750800B16E1BAECBCF078
:10CD200004E0090E0201535D0AE30601EA5104E042
:10CD3000080E0201535D03E302012D5105E0238239
:10CD4000080E076E100E086E23A202D0C3EC5BF033
:10CD5000DF50075C01E01C8CE552B5EFB6F01C9685
:10CD600012000201566BE66AE66AE66A8CECBAF0DB
:10CD700002012A6B07019F6B0B6A20B003D0208051
:10CD800034EC60F01200E6ECC0F00201050E2D6FED
:10CD9000280E2E6FE6DF020E0A5C05E153ECBDF0B3
:10CDA000140ED3ECB6F00501040E266FE552B5EF74
:10CDB000B6F0348C0101D051400B02E1530E01D08A
:10CDC000510E28EFB7F00101E351020B18E03C517E
:10CDD000800B15E12050010B12E12550040B0FE1EF
:10CDE0002450020B0CE1E3932F88B50EE66EC00EC3
:10CDF000E66E010E14ECB7F00101AA0EAC6F120042
:10CE0000B4ECC0F004E12050010B01E1000C010C76
:10CE100001015651800B05E0020E005C03E00004A6
:10CE200001E0000C010CE6ECC0F0E2ECBEF005E025
:10CE300053ECBDF0140ED3ECB6F020902094070113
:10CE40009D6B12ECC5F0E552B5EFB6F01DECBAF0F3
:10CE5000800E491841E14A503FE10101E39B199ED0
:10CE6000D190FF0E05014B5D04E04BC507F04B6907
:10CE700012000101E5A503D0E59576EC15F034AC80
:10CE80000AD009EC1CF0010802E1520E01D0500E4C
:10CE900028ECB7F0349C20B01DD0E2ECBEF002E0EC
:10CEA000006A71DB21960201685114E13250010BD6
:10CEB00011E12C50800B0EE12C50400B0BE10101D5
:10CEC000E851400B07E12F50200B04E12350800B69
:10CED00001E11F86072A1200F8ECC4F001E005D238
:10CEE0004A5001E002D220A0229CA0EC11F0FF08E1
:10CEF00001E018D12050200B01E114D11850800B13
:10CF000001E010D10201766B76C2B1F1199219ECF1
:10CF1000BAF0349C1C901E50010B06E01D50040B0F
:10CF200003E01D50080B0DE100500BE01F50020BF9
:10CF300008E06EDF000905E0258E1F0E6FECB7F0EC
:10CF4000F1D01E50010B18E1005006E01F50020BFB
:10CF500013E15EDF000910E00101010EB16F1982DB
:10CF6000076A0B0E086E005003E14ADF000901E07A
:10CF70001C8000502CE12DD01D50040B03E01D50EF
:10CF8000080B29E100500CE0E2ECBEF009E11F5073
:10CF9000020B21E1CFECB7F003E13ADF00091BE01F
:10CFA0001DB402D0110E05D01DB604D00201516B84
:10CFB000140E076E005003E123DF000901E01C801E
:10CFC000005007E08AECB8F002E1DDDEABD0F1DE24
:10CFD000A9D0F9DEA7D0050110511EE027AA12D072
:10CFE000005003E0CFECB7F010E0005003E108DFA1
:10CFF000000901E01C80005001E1E5DECFECB7F054
:10D0000001E0C1DE1E0E076E8DD0258E840E55EC1C
:10D01000BBF064EC1DF086D020AE05D0076A0A0E86
:10D02000086E1C807FD0005064E0B9ECB9F009E0D4
:10D030002050040B06E11E50020B5BE01DECBEF01D
:10D0400058E10201195114E01E50020B07E110ECE7
:10D0500007F000090DE1B9ECB9F00AE10201376B04
:10D06000386B196B19C255F239EC09F00AEC5CF017
:10D0700055ECC1F007E0B9ECB9F0FDE0F2ECBCF022
:10D08000FAE126D01C80BAECBCF013E01950400B3A
:10D0900010E01950040B0DE020A40AD01994050EDD
:10D0A000E66ED00EE66EE80E0C24D3ECB6F001D09E
:10D0B0001C901DECBEF010E0DEECBEF00DE0C30EE7
:10D0C000E66E940EE66E010EA7ECB8F0E5521C90E9
:10D0D00020941E929BEF04F01CA024D0000E0201AD
:10D0E0002A6F07019F6F0B6E1E92076A0B0E086E68
:10D0F00019D0005017E12050010B14E1B9ECB9F040
:10D1000003E02050040B0EE00101E3939BEC04F0DC
:10D1100055ECC1F005E0B9ECB9F0FDE02094120047
:10D120001C801FDE2050200B04E1DDEC09F000091B
:10D1300003E1020134513AE03FECB9F037E0050178
:10D14000106B20902094810E076EB9ECB9F002E1CB
:10D150001B0E12D0F2ECBCF00AE09E0EE66EB20E90
:10D16000E66E010E9BECC5F0E552E55208D0DDEC11
:10D1700009F0000905E01A0EE66E45EC22F0E552D2
:10D18000DDEC09F0000910E0ACC134F2F2ECBCF0C7
:10D190000BE0DEECBEF003E001013C9D02D001019A
:10D1A0003B9F57EC15F0149077EC06F0F8ECC4F0C8
:10D1B00001E14A5038E09BEC04F027AA28D061EC4A
:10D1C000D6F002012A6B2FAA02D046EC46F030A41A
:10D1D00002D0C7EC48F030AC02D043EC47F032A0AC
:10D1E00002D0D3EC46F023AE02D0DAEC45F024A016
:10D1F00002D0D6EC45F01FA802D056EC0EF02C5011
:10D20000800B03E12C50400B02E0ADEC0CF0259AB2
:10D210001AAC02D0F2EC07F028A203D0289227EC37
:10D2200033F01C8C12002050010B14E002012D5130
:10D2300011E11750800B06E025ECBEF009E00B0E63
:10D24000155C06E02050040B05E1B9ECB9F002E0F2
:10D2500013EF67F002012A5104E03FECBCF08CECC4
:10D26000BAF017AE5DD03EEC88F0EEECB8F017E007
:10D270002F50200B14E13050040B11E12350800B90
:10D280000EE13050400B0BE12450010B08E132500D
:10D29000010B05E13250020B02E171EC29F03292F0
:10D2A0001FAA3ED01F9A01013BAB3AD0C4ECBBF0A1
:10D2B0000201315110E199EC2EF02C0E155C14E1B5
:10D2C0001750010B11E00101D451D55D0DE10201B0
:10D2D000C80E316F1200316B1C0EE66E17ECD6F0E3
:10D2E000E5520101960EAC6F1200D4ECC2F018E1C9
:10D2F0004A5016E121BA14D068EC06F0000904E1A6
:10D300003CEC26F0FCEC5FF083EC0BF0238A810E02
:10D31000076E68EC06F0000903E071EC29F0258245
:10D3200012000C04040F0701006F12000101B59BED
:10D3300019AC23D039EC09F0138225A418D09CEC49
:10D34000CFF0960EE66EB20EE66E010E4CECC3F018
:10D35000E30E0C2428ECB7F046EC09F09CECCFF07F
:10D360008E0EE66EB20EE66E010E4CECC3F00201BC
:10D370000E0E376F060E386F1200D3DF0701FA0E5C
:10D38000036F016B026B0201536B546B1D90120013
:10D3900000C709F00201555104E0800E82ECB7F09D
:10D3A0001A800701035117E0035103078EECB8F010
:10D3B000CC0E005C10E0FF0E005C0DE0800E005C07
:10D3C00006E20050E66E3CEC04F0E552006E0050C0
:10D3D00082ECB7F0E6D7096A1200CBECC5F0DBCFE0
:10D3E00055F22F88006A23882FEC22F00101320EBB
:10D3F000AC6F17A802D00201558F0201195102E04B
:10D40000010E196F179EB5EFB6F017A802D0B9EC50
:10D410003FF019AC24D039EC09F0139217ECC3F0AB
:10D42000D00ED8800E54050E0F5405E210EC5CF0BF
:10D430000201196B120013820101E683218E1BEC9D
:10D4400009F0198A10EC07F000090FE120840101AE
:10D45000E499B9ECB9F009E00101E4891200278AE6
:10D4600002012D5102E0010E2D6F1200B9ECB6F051
:10D47000198C6BECB7F003E0CFECB7F001E0199C2E
:10D4800025A410D0FE0EDB500C6E50DF2594010158
:10D49000B587239C24B2238C248219AC32D0198402
:10D4A00028802FD01950400B0EE010EC07F0000937
:10D4B0000AE0B9ECB9F007E02050040B04E11D0EBE
:10D4C0006FECB7F01ED0FD0EDB500DE102011951DB
:10D4D00003E12750400B07E02FECC1F07EDFE5525F
:10D4E0000201196B0ED0FE0EDB500C6E1FDF19BC53
:10D4F00007D04EDF0501105103E110EC5CF001D0C4
:10D5000084DFB5EFB6F00601060E406F25ECBAF0E9
:10D5100004E2A85102E00601402B02011E0E276F13
:10D52000120001012951E8240301B86F0A01190E04
:10D53000D76F360ED66F0101D45103E0030ED45DD0
:10D5400003E10A01080ED66F88ECC0F003E10A017E
:10D550003C0ED66F0A01DA8FD46B34843AEFB9F0FF
:10D56000B9ECB6F0C4EC32F0CAEC15F033882FEC0D
:10D57000C1F0C0EC17F0E552B5EFB6F0010EE66E63
:10D58000EFDFE5521200000403E16AECC3F019D0AA
:10D59000005043E0030E005C16E16AECC3F0B6EC09
:10D5A000BCF002E00AECC0F021ECBAF004E06AEC56
:10D5B00004F0BFECB7F0ABECBAF003E1640E0E6E12
:10D5C0000F6ACCEFC4F00AEC12F0930E0E6E020E4E
:10D5D0000F6E0050030819E2700E0E6E030E0F6EF0
:10D5E000050E005C04E1930E0E6E020E0F6E060E29
:10D5F000005C04E1970E0E6E040E0F6E070E005CC9
:10D6000004E1200E0E6E060E0F6ECCECC4F0020E7E
:10D61000005C05E1500EDDECB6F0F2EF08F00050D2
:10D62000030803E20201040E356F070E005C03E1FC
:10D630000201080E356F1200B9ECB6F0280E9FEC0F
:10D64000C1F0290E66ECB7F0B5EFB6F0D9CFE6FF22
:10D65000E1CFD9FFE6528C9E0000000000000000E0
:10D660008C9600000000060EE66E95EC53F0E55235
:10D670008C860000000000008C9600000000D80E90
:10D68000E66E95EC53F0E552A1C7E6FF95EC53F03A
:10D69000E552E66A95EC53F0E552E66A95EC53F0F4
:10D6A000E5528C868C8EDF6A1E0EDF5C07E2640E0C
:10D6B000E66E4FEC1DF0E552DF2AF6D7E552E55253
:10D6C000E7CFD9FF1200D9CFE6FFE1CFD9FF8C9E7B
:10D6D00000000000000000008C9600000000030E17
:10D6E000E66E95EC53F0E552A1C7E6FF95EC53F0DA
:10D6F000E552FC0EDBCFE6FF95EC53F0E552FB0E56
:10D70000DBCFE6FF95EC53F0E552FA0EDBCFF3FFEB
:10D71000DB06F35000090FE0E8ECE4F0006EFD0ECC
:10D72000DBCFE9FFDB2AFE0EDBCFEAFF01E3DB2ADA
:10D7300000C0EFFFEAD700008C86C69E8C8EE552B3
:10D74000E7CFD9FF120002ECC1F0DF6ADF2AFA0E40
:10D75000DBCFE6FF46ECBCF072ECBAF04DECBCF06F
:10D76000FA0EDBCFE6FF46ECBCF0A80EE66E030E29
:10D77000E66E4DECBCF0010EDB6AFA0EDB507EEC7F
:10D78000B9F017E2010EDB50E76E8FECB9F0E7500D
:10D79000F2ECB8F0EFCF49F0010EDB50EA6AA80FC7
:10D7A000E96E030EEA22EF50495C03E1010EDB2A29
:10D7B000E4D76BECBFF002E070EC0BF06BECBFF069
:10D7C00003E00A0EDF5CC2E30A0EDF5C02E3000E38
:10D7D00001D0010ED2ECBEF002E2E16AE552E16E48
:10D7E0004950B5EFB6F0D9CFE6FFE1CFD9FF8C9E17
:10D7F00000000000000000008C9600000000060EF3
:10D80000E66E95EC53F0E5528C86000000000000B7
:10D810008C9600000000020EE66E95EC53F0E55287
:10D82000A1C7E6FF95EC53F0E552FE0EDBCFE6FF15
:10D8300095EC53F0E552FD0EDBCFE6FF95EC53F08F
:10D84000E552FA0EDBCFF3FFDB06F350000911E0DF
:10D85000FB0EDBCFE9FFDB2AFC0EDBCFEAFF01E3A7
:10D86000DB2AEF50006E0050E66E95EC53F0E55267
:10D87000E8D700008C86C69E8C8E050EE66E4FECB7
:10D880001DF0E552E552E7CFD9FF1200D9CFE6FFF0
:10D89000E1CFD9FFE652AAEC53F00101640EAC6F60
:10D8A00004008EEC3AF0020E0701585D0FE007010C
:10D8B000925109E09BEC05F00401FD6FFDC4E6FF09
:10D8C000ACEC05F0E55288EC96F071D0070192516E
:10D8D0006EE007019251496E4A6A4A3404E24950A7
:10D8E000C008000E4A5408E20701040E246F240EFB
:10D8F000E66E61EC11F0E5529BEC05F00401FD6F62
:10D900003B0E0401FD5D0CE104013B0EFE6F0601C0
:10D91000C46B309A0101379BD9EC0AF00701586BB0
:10D92000610E0401FD5D07E30401FD51660803E398
:10D93000200E0401FD5F300E0401FD5D22E30401B1
:10D94000FD5146081EE30601C42B410E0401FD5D96
:10D9500004E2300E0401FD5F06D0410E0401FD5DBE
:10D960000A0F0401FD6F020E0601C45D08E1060105
:10D97000C339F00B0401FD250401FD6F02D0FDC485
:10D98000C3F6020E0601C45D11E1FDC4E6FF34ECEE
:10D990000BF0E552006E010EE66E4FEC1DF0E55205
:10D9A0000601C46B0050E66E47DEE5528FD70201D8
:10D9B000685102E010EC81F01C9C100E075C03E241
:10D9C000A7EC61F024D01E0E075C03E2D7EC65F0F3
:10D9D0001ED00750496E4A6AD8904A5004E6800E1D
:10D9E000495C000E4A5803E28FEC1DF010D007503E
:10D9F000496E4A6AD8904A5004E6920E495C000E7D
:10DA00004A5803E226EC67F002D07FEC28F01CBCF9
:10DA1000D3D78BEC4AF0095008E00701070E246FBA
:10DA2000240EE66E61EC11F0E55222A228D022927B
:10DA30002E98329AD4EC75F0DF682E50100B15E05A
:10DA4000010101012A51040B10E12950020B0DE1E3
:10DA5000DF500BE00D5002E1010E0D6E2E98D0EC60
:10DA600080F0D4EC75F0DF06E8D7DF5008E107015D
:10DA7000050E246F240EE66E61EC11F0E55210D70E
:10DA8000E552E552E7CFD9FF12000101D45112004F
:10DA9000080E016E0101D45102E1180E016E310E23
:10DAA000B95D09E1016AB7EC09F0000902E0100E66
:10DAB000016E6CEC15F01200200EE66E620EE66E42
:10DAC000070EE66E800EF3EFC1F02AECC2F0A9EC6F
:10DAD000BBF0EFCFDFFFFF0EDF5C02E1100EDF6E69
:10DAE000DF50E552B5EFB6F0D3DF03015E510126FA
:10DAF000015005ECC0F0046E1200C4ECBBF0010153
:10DB0000040E016F0450006E00500F0803E2100E67
:10DB1000005E04D0100ED8800054006E6AECD5F080
:10DB20000101200E1A6F050E006E300E1B5D02E023
:10DB3000040E006E04500F0805E200501FECB9F00F
:10DB40002B0E04D000501FECB9F02D0EEF6E010E1D
:10DB5000016F960E496EC20E4A6E010E4B6E5EC389
:10DB60004CF04D6A4E6AD4ECC0F0AFECC1F001014C
:10DB7000188F1200000CE6ECC0F00050EF085CE2D9
:10DB8000F00E005CDF6EDF50080861E32950010BE6
:10DB900005E10401F95102E1FA5108E00101E491C3
:10DBA0000201246B3C6B88EC96F0F0D7C4ECBBF020
:10DBB00021ECBEF0DF50FE0BE842750F096E016AE2
:10DBC000DFA002D0800E016E026A070E025C0CE23A
:10DBD0004EEC34F0005008E0FF0E005C05E0FBEC7A
:10DBE000D5F0012A022AF1D78EECD3F00101E485A9
:10DBF000080E016EDFA002D0800E0126026A780EA8
:10DC0000025C10E24EEC34F000500CE0FF0E005CC1
:10DC100009E00050036EE66EACEC05F0E552012A17
:10DC2000022AEDD73B0E035C05E03B0EE66EACEC42
:10DC300005F0E552096A15D072ECBFF027ECC2F08E
:10DC4000056EFF0E055C05E16C0E00ECB8F0258E4C
:10DC500008D0B9C157F205C0B9F129820201010EFD
:10DC6000686FE552B5EFB6F00068016A015074ECD8
:10DC7000B7F004E6AA0E495C000E4A580CE272ECBA
:10DC8000BFF029ECC4F00101B95D03E10150006E61
:10DC90001200012AEBD71200020E016E2AC100F019
:10DCA0000BEC34F02F0E016E57C100F00BEC34F08A
:10DCB000370E016E5FC100F00BEC34F00F0E016EF9
:10DCC00037C100F00BEC34F0100E016E38C100F0DB
:10DCD0000BEC34F02E0E016E56C100F00BEC34F05C
:10DCE000620E016E8AC100F00BEC34F0650E016E1D
:10DCF0008DC100F00BEC34F0660E016E8EC100F0A9
:10DD00000BEC34F06E0E016E96C100F00BEF34F0A8
:10DD1000130E016E3BC100F00BEF34F0060E010153
:10DD2000B95D0CE119B60AD0BAEC5AF024EC8AF0CD
:10DD3000020106811EBC098505014787090E010104
:10DD4000B95D02E146ECB1F0190E0101B95D01E1E6
:10DD50009771170EB95D14E119A63B79A7EC1AF07B
:10DD600071EC29F0ACECC0F004E02150020B01E1B1
:10DD7000E8893BB903D01E9A3AECB9F00501478710
:10DD8000030E0101B95D03E0040EB95D11E119B69E
:10DD900008D0030EB95D03E10701BA7102D0070193
:10DDA000BA73E5ECBDF0B0EC07F0020107812D84F9
:10DDB000100E0101B95D04E119A63E7172EC53F039
:10DDC000070E0101B95D02E119A6967DB95104E182
:10DDD00019A6337411EC1BF02A0E0101B95D02E1A2
:10DDE00019A62A751A0EB95D01E12E74280EB95DC7
:10DDF00001E12E72120EB95D02E119A62A7F12000E
:10DE000033ECC6F0FB0EDB50D880DF5403E2FB0E90
:10DE1000DB50DF6EFC0EDB50DF5C03E2FC0EDB5000
:10DE2000DF6E0DAE0CD0FC0EDB50D880DF5402E26A
:10DE3000DF0605D032B603D0FB0EDB50DF6E0D04DB
:10DE40000BE1FB0EDB50DF5C02E2DF2A05D032B6CD
:10DE500003D0FC0EDB50DF6ED2EFC4F041ECC3F018
:10DE600051ECBCF0B5EFB6F0B9ECB6F0328646EC4A
:10DE7000BCF072ECBAF051ECBCF03296B5EFB6F0F3
:10DE800041ECC3F0F1DFB7ECC5F0E552B5EFB6F009
:10DE900033ECC6F079ECBFF0E8AE02D0493403D0E1
:10DEA000E750D880495403E2FB0EDB50DF6E80EC74
:10DEB000BFF0E8AE02D0E73402D0E750495C03E29D
:10DEC000FC0EDB50DF6E0DAE0BD080ECBFF0E8AE89
:10DED00002D0493403D0E750D880495401E2DF062C
:10DEE0000D040AE179ECBFF0E8AE02D0E73402D0CD
:10DEF000E750495C01E2DF2AD2EFC4F0500E036E16
:10DF00003CECC2F005E01B50080B02E11E0E036E54
:10DF10001200E6ECC0F002DF290E0101B95D2AE132
:10DF20003651070B006E0D040EE136BF02D0368F5E
:10DF30001AD036BD03D0368D006A15D0070E005CAE
:10DF400012E2002A10D0FF0E0D5C0DE1005005E03A
:10DF5000000600AE08D0006A02D036AD02D0369D71
:10DF600002D036BF369F0050070BF36EF80E361501
:10DF7000F310366F1D0EB95D13E10D0408E156B1C3
:10DF800002D056810DD056B50BD0568509D0FF0E64
:10DF90000D5C06E156A502D0569502D056B15691B9
:10DFA000390EB95D1BE119ECBAF000500EE1010128
:10DFB0003C7F04903CBF048004B002D0E3830AD0CD
:10DFC0002386DAECB8F0239605D001013B7F04905C
:10DFD0003BBF048057EC15F027EC33F0360E0101FF
:10DFE000B95D18E16BECB7F00AE1C80EE66E320ECF
:10DFF000E66E010E02ECB7F010EC5BF00BD0C80E31
:10E00000E66E010EE66E530EE66E010E07ECB7F0FB
:10E0100057EC15F0160E0101B95D1EE1D45105E073
:10E02000030ED45D17E10A5015E0D45106E18A755C
:10E0300013908AA506D0138004D08E7513908EB5E8
:10E0400013801350010B02E0139A01D0138A54EC91
:10E050001BF002D006EC0AF0080E0101B95D07E1E1
:10E06000860EE66EB20EE66E010E14ECB7F00C0EE4
:10E070000101B95D0BE1150EE66E030EE66E550E5D
:10E08000E66E010E07ECB7F09BEC04F00B0E0101FD
:10E09000B95D15E1010EE66E840EE66E010E02EC2E
:10E0A000B7F0300E010184250401F76F020E010163
:10E0B000845D03E10401340EF76F59EC96F02E0EE7
:10E0C0000101B95D1EE134C1A8F26CEC15F01E0E21
:10E0D000E66E340EE66E010E02ECB7F087EC19F036
:10E0E0000201A85103E00101345106E00201A851E8
:10E0F00005E10101345102E0A8EC14F002010885A9
:10E100002A84110E0101B95D2EE10D0411E1080E02
:10E11000505D02E10D0E26D0050E505D1EE0030E8F
:10E12000505D16E050050FE00D0E505D1CE006D06E
:10E13000FF0E0D5C18E1030E505D02E1010E12D0DE
:10E14000050E505D02E1030E0DD0080E505D02E198
:10E15000050E08D00D0E505D02E1080E03D05005EB
:10E1600002E0010E506F220EB95D0EE1800E0D141B
:10E1700004E03C0E675D01E2672B0D0403E167518B
:10E1800001E067074DEC4AF0CAECBEF02FE1E7ABC7
:10E1900003D006EC0AF02AD00AECC0F00701BAABB3
:10E1A00003D00A0E0E6E0F6A0D040CE100010E5032
:10E1B0000101692700010F5001016A23000E6B2342
:10E1C0006C230ED0FF0E0D5C0BE151ECC5F04950F5
:10E1D0000101695F4A506A5B4B506B5B4C506C5B52
:10E1E0002BECB3F02484338827EC33F0130E0101B9
:10E1F000B95D0BE1030E4F15066F020EDDECC1F0A9
:10E20000FC0E01014F1706514F13140EB95D11E1B9
:10E21000300E4F15066F06390F0B066F020EDDEC40
:10E22000C1F001010639F00B066FCF0E4F170651F2
:10E230004F130F0EB95D09E1820EE66E520EE66EC7
:10E24000510EE66E010E07ECB7F0350E0101B95D17
:10E2500019E10701BA51E840E8403F0B0101066FA0
:10E26000030E0617DDECC1F00101040E0603F3CF27
:10E2700006F1F30E0701BA17010106510701BA139F
:10E28000B0EC07F03A0E0101B95D09E1730EE66EDC
:10E29000460EE66E520EE66E010E07ECB7F03B0E30
:10E2A0000101B95D06E11274049012B40480A6EC79
:10E2B00039F0C0ECC0F039E12050040B03E11B50F1
:10E2C000080B33E02B51000830E20D0414E12B5011
:10E2D000040B02E0140E01D0010E496E4A6A49BED9
:10E2E0004A682250040B01E0010E01ECBAF04950DB
:10E2F000EE264A50ED22FF0E0D5C14E12B50040B6C
:10E3000002E0140E01D0010E496E4A6A49BE4A6805
:10E310002250040B01E0010E01ECBAF04950EE5E10
:10E320004A50ED5AB3EC12F01E882D0E0101B95D72
:10E3300008E1320EE66E950EE66E010EA7ECB8F01F
:10E34000E552320E0101B95D2DE133A608D09B0ED6
:10E35000E66E940EE66E010EA7ECB8F01FD02B51BE
:10E3600009081EE32B5100081DE2DDECB0F0E66E5B
:10E3700048EC10F0E55209ECB8F012E100C006F1EB
:10E38000DC0EE66E010EF5ECC5F007ECB7F006C149
:10E3900000F00BEC34F0E66A91EC18F0E55202D094
:10E3A00006EC0AF0200E0101B95D23E1D4511AE117
:10E3B000500EE66E280EE66E290EE66E010E07EC94
:10E3C000B7F001012951E8240301B86F69EC13F09B
:10E3D0003FECBBF03AECB9F0A8EC14F00501478F24
:10E3E000478507D07F0EE66EB20EE66E010E14EC86
:10E3F000B7F0180E0101B95D07E1020EE66E700E6E
:10E40000E66E020E02ECB7F01F0E0101B95D1CE1D1
:10E41000020EE66E390EE66E010E02ECB7F0010157
:10E42000395104E198ECC5F0CBEC20F056ECC5F086
:10E43000006A0101395102E0010E006E00C0D8F2FD
:10E4400000C0D7F200C0EBF90A0EB95D01E08ED032
:10E4500039512CE030A227D00901E85104E10D0424
:10E4600001E082D016D0E80511E10D0408E1010EAB
:10E47000E86F730EE66EB20EE66E010E11D0E86B19
:10E480006D0EE66EB20EE66E010E0AD0FF0E0D5C4A
:10E490006BE1010EE86F790EE66EB20EE66E010ECC
:10E4A0001DECB7F061D006EC0AF060D01E86295052
:10E4B000020B0AE03A5108E03A51010802E2010E6B
:10E4C00001D0020E3A6F10D0130EE66E3A0EE66ED1
:10E4D000010E02ECB7F00A0E01013A5D03E0120EE4
:10E4E0003A5D02E10D503A2796EC07F001013A51EE
:10E4F00002E08D8303D03A5101E18D93030E3A5D22
:10E5000033E33A51130830E3000E036E026E016EDE
:10E51000030E3A5D006E080E005C0BE2010E00C0B7
:10E52000E7FFE75204E0E846FE0BE706FCE1016E78
:10E5300012D0100E005C0CE2080E005C496E010E59
:10E54000495204E0E846FE0B4906FCE1026E03D0A6
:10E55000100E005C036E010EE66E0350E66E8BEC4F
:10E56000C5F066ECBAF002D068ECABF00101B90579
:10E570000BE11E0EE66E010EE66E700EE66E010EEB
:10E5800007ECB7F00FEC1BF0050E0101B95D4FE190
:10E59000E95109E1080EE66E040EE66E470EE66EDE
:10E5A000010E07ECB7F00101E90508E1E668C80EC5
:10E5B000E66E7D0EE66E010E07ECB7F0020E01016D
:10E5C000E95D08E1C80EE66EE66A4B0EE66E010EE6
:10E5D00007ECB7F0030E0101E95D13E10701BAA3EF
:10E5E00008D0960EE66E780EE66E4D0EE66E010EC3
:10E5F00006D0320EE6ECBEF04C0EE66E010E07ECD5
:10E60000B7F0040E0101E95D08E10F0EE6ECBEF083
:10E61000410EE66E010E07ECB7F0050E0101E95D53
:10E6200004E119A6627321EC1AF00FEC1BF02C0E1A
:10E630000101B95D07E1640EE66E850EE66E010E1E
:10E6400002ECB7F0020E0101B95D09E1010EE66EC0
:10E65000310EE66E010E02ECB7F0A7EC1AF0300EA8
:10E660000101B95D10E12B51090806E20F0EE66EBB
:10E670007B0EE66E010E05D00F0EE66E860EE66E80
:10E68000010E02ECB7F0330E0101B95D0CE16CEC48
:10E6900015F0190EE66EE66A7A0EE66E010E07ECCC
:10E6A000B7F07EEC12F0370E0101B95D09E13C0EC6
:10E6B000E66E6E0EE66E010E02ECB7F057EC15F04A
:10E6C000380E0101B95D09E13C0EE66E6F0EE66E93
:10E6D000010E02ECB7F057EC15F02B0E0101B95DFD
:10E6E00026E181C306F13B0E016E03017F5104E177
:10E6F00080C306F1170E016E020E7F5D02E182C338
:10E7000006F101502AECBCF003017F5102E106C181
:10E7100080F37F0502E106C181F3020E7F5D02E115
:10E7200006C182F3010197A102D059ECD7F0240E63
:10E730000101B95D14E197A110D0170EE66EE90E44
:10E74000E66E990EE66E010EE66E48EC6FF0B7ECE1
:10E75000C5F0E55259ECD7F002D006EC0AF00D0EE8
:10E760000101B95D03E1D273E1EC04F00E0E010189
:10E77000B95D03E1D275E1EC04F0260E0101B95D4B
:10E7800032E1016AD5CA03F0D251010B12E03751D0
:10E79000080B0FE0040E036E1BA00BD0030E036EDC
:10E7A000010E016E0A011C5104E1280E216F21CADD
:10E7B0001CFAFE0E15ECBAF005011751050DA7EC79
:10E7C000B9F0140E4B260A0E4C22035000014B24C4
:10E7D000496E000E4C204A6E04ECB8F051ECBCF0CF
:10E7E0002484DDEC0BF0340E0101B95D12E12B51F4
:10E7F00000080FE2FA0EE66E2250040B01E0010E53
:10E800004A6A910F496E020E32ECC3F0B3EC12F07B
:10E810001E8898ECC0F003E0310EB95D1CE1030ED8
:10E82000D45D03E106EC0AF016D00201780E2C6FDD
:10E8300074EC6DF004C006F1200EDDECC1F0015067
:10E84000A9ECBBF006C1EFFF308E06C104F07DECF1
:10E850006DF01AEC1AF01C0E0101B95D06E119B653
:10E8600002D002017879A8EC12F0230E0101B95D03
:10E8700009E1030EE66E430EE66E010E02ECB7F000
:10E8800017EC1DF01B0E0101B95D0FE13EC1DFFF6A
:10E89000188C3E6B070EE66E3F0EE66E010E02EC24
:10E8A000B7F055ECC0F0DFCF3EF11E0E0101B95DAF
:10E8B00002E10D503327150EB95D09E10C0EE66E2D
:10E8C000070EE66E3D0EE66E010E07ECB7F05CC378
:10E8D000E6FF42EC0AF0E5523C0E0101B95D14E19D
:10E8E00019B611D050ECC6F0040A01E0010E496ED1
:10E8F000E2ECB6F04950010BF36EF346F346FB0E23
:10E90000EF14F310EF6E2E863D0EB95D32E1A7ECE9
:10E91000C3F0016EACECC3F0026E0D50022602AEE5
:10E920000ED0630E026E01060150D3ECB7F007E281
:10E930004950F908000E4A5402E2F90E016E0250E5
:10E94000630802E2026A012A0150D3ECB7F006E242
:10E950004950F908000E4A5401E2016AE2ECB6F0AF
:10E96000030E01C0EBFFE2ECB6F0020E02C0EBFFBB
:10E970002E863E0EB95D1BE1A2ECC3F0016E0D5078
:10E98000E82401260150090802E2090E016E080E72
:10E99000015C02E1090E016E030E015C02E2030E4E
:10E9A000016EE2ECB6F0010E01C0EBFF2E86400EC8
:10E9B000B95D51E129ECC5F0496E4A6A24ECC5F015
:10E9C0000A0DF3504924DA6FF4504A20DB6F2EEC25
:10E9D000C5F002E1EEECBDF00D040CE1D890DB5186
:10E9E00004E6E70EDA5D030EDB5911E2DA2B000EC6
:10E9F000DB230DD0FF0E0D5C0AE1DB3504E3DA51B9
:10EA00001908FC0EDB5503E2DA07000EDB5B2888F1
:10EA1000800EDB1503E02898EEECBDF0DAC149F07A
:10EA2000DBC14AF08CECC0F00DECB7F0E2ECB6F0D4
:10EA3000040E49C0EBFFE2ECB6F0050E39C0EBFF67
:10EA4000E2ECB6F02850100B02E0EF8001D0EF901E
:10EA50002E8671EC29F03F0E0101B95D3FE1E2EC39
:10EA6000B6F0060EEB50006EE2ECB6F00490EF50FC
:10EA7000020B01E004800D500026005006E10470F6
:10EA800004807EEC6FF00350006E7EEC6FF003505C
:10EA9000D880005404E204700480010E006E20EC63
:10EAA000C2F001E004900480E2ECB6F00450010BE7
:10EAB00002E0EF8201D0EF92E2ECB6F0060E00C069
:10EAC000EBFF100E01012B5D03015C5D06E100C050
:10EAD00048F1DAECB8F05CC300F02E86E552B5EFF1
:10EAE000B6F05C0E00245AECC5F00101100E136F55
:10EAF000145102E1100E146F1200ACECC3F058EC8C
:10EB0000BBF0A7ECC3F0006E0101030E006F4DECEB
:10EB1000D5F0060EE66E030EAFEFBBF02BECC1F0A6
:10EB2000090809E2FE0EDB50F00F006E005050ECB9
:10EB3000BBF0E3DF23D0FE0EDB50006ED2DF020E0F
:10EB400045ECB7F00DE20101010E146F080E156FD0
:10EB5000FE0EDB040DE1030E146F050E156F08D0D9
:10EB600013C112F114C113F115C114F10101156B98
:10EB7000A0ECC0F002E1090E156F158FB5EFB6F0ED
:10EB800056EC21F02E801200140E006E04A002D06C
:10EB9000110E006EC0EF75F00E0E006E04A002D0D4
:10EBA000080E006EC0EF75F01FECC5F00101B55105
:10EBB000800B04E02F50100B01E19FD09CECCFF0B4
:10EBC00007EC80F0010139510DE00A0EB95D0AE150
:10EBD000016B650EE66EB20EE66E010E7FECC6F0BE
:10EBE0000101198F090EB95D01E1198F050EB95D9B
:10EBF00049E1040E016F2A0E196FE95108E1610E17
:10EC0000E66EB20EE66E010EE66E50ECB7F0010154
:10EC1000E90508E15D0EE66EB20EE66E010EE66EE7
:10EC200050ECB7F0020E0101E95D08E1590EE66E05
:10EC3000B20EE66E010EE66E50ECB7F0030E010167
:10EC4000E95D08E1550EE66EB20EE66E010EE66E67
:10EC500050ECB7F0040E0101E95D08E1510EE66EDB
:10EC6000B20EE66E010EE66E50ECB7F0050E010135
:10EC7000E95D08E14D0EE66EB20EE66E010EE66E3F
:10EC800050ECB7F02D0E0101B95D11E10201B05158
:10EC90000EE09CECCFF0460EE66EB20EE66E010E74
:10ECA0007FECC6F02CA203D00101370E1B6F260E9D
:10ECB0000101B95D07E13751080B04E04C0E1B6FF1
:10ECC0002A0E1C6F1FA805D09CECCFF0006A6BECDD
:10ECD00021F07DEC5AF0000905E0310E03015C25BE
:10ECE0000101186F98ECC0F003E0310EB95D05E149
:10ECF000300E03015E2501011C6F3BECC5F00E0ECA
:10ED0000136F146FBAEC6DF0000907E00101006B9E
:10ED1000280EE66EF1ECD5F0E552016A370E0101DE
:10ED2000B95D08E16EC100F0016802016E0EA46FCA
:10ED3000010EA56F380E0101B95D08E16FC100F049
:10ED4000016802016F0EA46F010EA56F1E0E010176
:10ED5000B95D08E10201330EA46F010EA56F33C146
:10ED600000F00168150E0101B95D0BE1050E3D03D0
:10ED7000F350410F006E016802013D0EA46F010EB9
:10ED8000A56F200E0101B95D08E129C100F00168FD
:10ED90000201290EA46F010EA56F1B0E0101B95DC2
:10EDA00008E13F29006E016802013F0EA46F010EC9
:10EDB000A56F050E0101B95D65E1E95106E10201AA
:10EDC000470EA46F010E1FECB8F00101E90506E142
:10EDD00002017D0EA46F010E1FECB8F0020E0101BE
:10EDE000E95D06E102014B0EA46F010E1FECB8F0C5
:10EDF000030E0101E95D1DE1006B0701BAA30CD010
:10EE0000420EE66EB20EE66E010ED8ECB6F00201CE
:10EE10004D0EA46F010E0BD03E0EE66EB20EE66EE6
:10EE2000010ED8ECB6F002014C0EA46F010E1FECDF
:10EE3000B8F0040E0101E95D06E10201410EA46F84
:10EE4000010E1FECB8F00168050E0101E95D17E144
:10EE5000016A62A306D03A0EE66EB20EE66E010EAD
:10EE600005D0360EE66EB20EE66E010ED8ECB6F0A8
:10EE70000201620EA46F010EA56F020EA66F0101C2
:10EE8000050E006F350EB95D0AE1D4C1E6FF8AECCC
:10EE90000BF0E55201687CECBDF00C0EA66F015042
:10EEA00002E04DECD5F0150E0101B95D03E0200E36
:10EEB000B95D01E1148F350EB95D05E1135102E131
:10EEC000100E136F158F080EB95D19E1FAECB8F04A
:10EED000B5ECBBF00101115102E1100E116FA80E4B
:10EEE000D8800E54610E0F5408E2016B300EE66EAE
:10EEF000B20EE66E010ED8ECB6F00101138F390E9A
:10EF0000B95D0CE16BECB7F005E101013CAF05D058
:10EF1000048003D001013BBF04803EDE3B0E0101B3
:10EF2000B95D03E112B4048037DE090E0101B95D59
:10EF300009E1100E146F14C113F1010E156F11B019
:10EF4000152B2E80360EB95D0DE132C100F06BEC51
:10EF5000B7F002E053C100F029ECBAF04DECD5F067
:10EF60000101148F060EB95D39E1D4C100F00050E3
:10EF700003E1D051400B24E121ECBAF004E001019F
:10EF8000D051040B1DE1030E005C07E1030E0A5C87
:10EF900004E10101CF51040B13E1000407E1020E6B
:10EFA00001012B5D0DE02B5103080AE3020E005C0A
:10EFB0000DE1020E01012B5D09E0040E2B5D06E25E
:10EFC0002C0EE66EB20EE66E010E05D0360EE66E23
:10EFD000B20EE66E010ED8ECB6F02E800C0E0101DA
:10EFE000B95D1FE1150E555D0BE1006B230EE66E5A
:10EFF000B20EE66E010EE66EEBECD5F0E5520AD0ED
:10F0000055C100F04DECD5F0060EE66E050EE66E2D
:10F010005BEC07F0E552E5520201550EA46F010EBC
:10F02000A56F030E0101B95D0DE10701BAB102D070
:10F030000E0E01D0080EE5ECBAF07CECBDF0010E2E
:10F04000A66F2E80040E0101B95D17E10701BAB366
:10F0500006D03E0EE66EB20EE66E010E07D001013E
:10F0600000071E0EE66EB20EE66E010ED8ECB6F08C
:10F070007CECBDF0020EA66F2E80C0ECC0F02EE13D
:10F080002B5103E138ECC2F028D02250040B01E0F0
:10F09000010E010F0E6F030E006F04902250040B3F
:10F0A00001E0010E01ECBAF0EECF0EF0EDCF0FF063
:10F0B000E2EC21F00101100E116F2BB4156F2250FC
:10F0C000040B01E0010E020DF3CFF3F6F4CFF4F6DA
:10F0D0008D0E0601F327020EF4232E882D0E01015A
:10F0E000B95D01E019D124B80CD0006B42EC5BF0A3
:10F0F00058ECBBF029ECBAF04BEC5BF058ECBBF0F1
:10F100000AD180EC0EF03AECBBF080EC0EF00E5021
:10F110000101D8270F50D923D8C10EF0D9C10FF063
:10F12000010E0F0B04E0CEECBEF0E806FCE1070197
:10F130000E500A5D0F500B5905E20A510E5E0B513D
:10F140000F5A02D00E6A0F6A0EC00CF70FC00DF7EF
:10F150000201B0511CE0190EEFECC1F0B0C23EF05C
:10F1600080ECC0F004E189EC04F00201B16FB1C29F
:10F1700000F00101126B63ECB7F0CEECC3F03EC0BF
:10F1800013F13AC014F10101110E156F138F42EC07
:10F190005BF0026E006E2CA204D04BEC5BF0026EB2
:10F1A000006E0201B05157E0960E0101D86FD96B85
:10F1B0001FA003D0F00ED86FD96BB8ECC0F004E0FC
:10F1C000320E0101D86FD96B0101D8510E5CD951B3
:10F1D0000F5810E2E5ECC2F004E6F00E495C000EB8
:10F1E0004A5808E2002A640E0201B05D1DE2190EC1
:10F1F000B0271AD00C0E4A6AD825496ED9514A2236
:10F20000D2ECC3F005E20050640802E200060CD024
:10F210000201B051D3ECB7F007E24950C808000E24
:10F220004A5402E2C80EB06F0250005C73E02CB288
:10F2300008D0E66A0050E66E54EC5BF0E552E66EEC
:10F2400007D00050E66E64EC5BF0E552E66EE66ACD
:10F25000A1ECBAF05FD02CB244D042EC5BF0496E26
:10F26000640E495C09E342EC5BF04A6E4B6A4B3436
:10F270000DE202ECBEF00AE242EC5BF00701246F03
:10F280004E0E15ECB8F0EBEC80F044D0E66AE66A7E
:10F29000A1ECBAF00201FA0EB06F08ECC2F005E082
:10F2A000D8900B330A33E806FBE14BEC5BF0496E78
:10F2B000640E495C09E34BEC5BF04A6E4B6A4B34DD
:10F2C00008E202ECBEF005E2A00EE66E64EC5BF034
:10F2D000E5524BEC5BF0E66EE66AA1ECBAF02C82EC
:10F2E00019D0EBEC80F04BEC5BF0496E640E495C9E
:10F2F00009E34BEC5BF04A6E4B6A4B340AE202ECDA
:10F30000BEF007E24BEC5BF00701246F510E15ECE9
:10F31000B8F02C9225822E882E0E0101B95D1DE1D8
:10F32000CBEC20F029ECBAF06BECB7F003E011EC79
:10F33000BEF003E138ECC2F00BD034C100F068EC51
:10F34000C2F0100E136F0A0E345D02E2100E146F3D
:10F350000201340EA46F010EA56F110E0101B95DFB
:10F3600025E1156B15C114F1100E136F0D0E505DD4
:10F3700003E1010E146F17D0080E505D02E1050E77
:10F3800009D0050E505D02E1030E04D0030E505D5E
:10F3900003E1020E156F07D0500505E1010E156F50
:10F3A000006F5EECC5F00101158F2E88330EB95D3C
:10F3B00017E1020E006F080E006E8AB302D00E0E27
:10F3C000006E56EC21F07AC100F068ECC2F0100E2D
:10F3D000136F02018A0EA46F010EA56F020EA66FB5
:10F3E000300E0101B95D1BE1A0EC61F0050F58EC96
:10F3F000BBF0A0EC61F0000904E1EEECBEF05EECC5
:10F40000C5F00201860EA46F010EA56F25ECBAF0BF
:10F4100005E202017B0EA46F010EA56F2E8801018B
:10F42000B90511E170C100F04DECD5F01E0E0101DF
:10F43000705D04E1010E006F5EECC5F00201700E1C
:10F44000A46F010EA56F2C0E0101B95D11E185516C
:10F4500004E10B0EE5ECBAF006D085C100F04DECEE
:10F46000D5F00101158F0201850EA46F010EA56F65
:10F47000020E0101B95D1FE10201310EA46F010E00
:10F48000A56F0101040E62ECC5F00101310506E132
:10F49000020E006F9E0E006E56EC21F0020E01016E
:10F4A000315D09E1020E006F140EE66EB20EE66EDB
:10F4B000010ED8ECB6F098ECC0F003E0310EB95D67
:10F4C00034E148EC6DF0026A080E025C2EE2015055
:10F4D000022405ECC0F0006E100E005C03E08AEC24
:10F4E000B8F002E1020E13D00050120802E2040E3E
:10F4F0000ED00050100802E2030E09D00E0E005C80
:10F5000002E2006A05D0100E005C02E2010E006EFD
:10F51000410E00241AECB8F0D00FE66E02509BECBE
:10F52000B7F0BCECB8F0022ACFD7120E0101B95DDA
:10F5300010E1100E146F14C113F1110E156F2ABFD4
:10F54000152B02012A0EA46F010EA56F800EA66F67
:10F550002E803A0E0101B95D18E1050E006F52C10F
:10F5600000F00201520EA46F010EA56F0101E6A585
:10F5700007D04AC100F002014A0EA46F010EA56F28
:10F580004DECD5F00101148F2E88320EB95D4FE19C
:10F590002B5103E138ECC2F049D0006B0F0EE66E40
:10F5A000B20EE66E010ED8ECB6F033B603D0010110
:10F5B0000E0E0E6F25ECBAF039E3050E006F09EC64
:10F5C000B8F003E1FBECBFF01FD00101E49DB00EE9
:10F5D0000D258EECB8F00F0E005C03E300503008F0
:10F5E0000DE2230E006E0901EB510E0807E2310E09
:10F5F000EB5D04E2EBC900F00101E48D0101E4BD23
:10F6000003D000507DECC1F04DECD5F00101135159
:10F6100002E1100E136F09ECB8F008E00101158F3C
:10F62000240E136FE4AD02D0110E136F2E88270E37
:10F630000101B95D09E186EC07F09C0E0E5C630EDA
:10F640000F5802E2B5ECBBF0220E0101B95D1CE1DE
:10F65000030E006F090EE66EB20EE66E010ED8ECD8
:10F66000B6F067C100F000500FE00101020E006F1C
:10F670004DECD5F001010E0E106F0A0E675D04E22D
:10F68000100E106F0E0E116FCAECBEF054E1006B3D
:10F69000E7AB25D085ECBEF00BECC6F058ECBBF028
:10F6A0000101240E0E6F9D0E90ECC3F00EC0DEFF24
:10F6B0000FC0DDFFC80E29ECBEF004E3840E42EC5F
:10F6C000C0F004E20701080EFDECC4F0B5ECBBF09D
:10F6D0000101100E116F160E126F25822BD069C119
:10F6E0001DF16AC11EF16BC11FF16CC120F10A0E40
:10F6F000D6ECBDF01DC13BF01EC13CF01FC13DF07A
:10F7000020C13EF044ECE4F03BC01DF13CC01EF1D2
:10F710003DC01FF13EC020F18AECD5F0B4ECD5F02D
:10F720000101100E0E6F118F148F0701BABB02D0AA
:10F730000101156F2E880490100E0101B95D0AE1D8
:10F740003E5101E00480CCEC75F002013E0EA46F46
:10F75000010EA56F070E0101B95D0BE196BD048096
:10F76000CCEC75F00201960EA46F010EA56F400E51
:10F77000A66F290E0101B95D26E136AD19D08CECDA
:10F78000CFF0020EE66EB20EE66E010ED8ECB6F0C9
:10F7900001013651070B050DF3500A0F006E63ECA3
:10F7A000B7F0CEECC3F03EC014F13AC015F104D06E
:10F7B00036BF0480CCEC75F00201360EA46F010E4A
:10F7C000A56FC70EA66F0B0E0101B95D23E1845131
:10F7D00006E1050E006F0B0EE5ECBAF015D08CECCF
:10F7E000CFF00101840506E1F90EE66EB10EE66E7A
:10F7F000010E08D0020E845D07E1F00EE66EB10E38
:10F80000E66E010ED8ECB6F00201840EA46F010E74
:10F81000A56F2E88170E0101B95D13E1050E006F6B
:10F820000E0E006E3BA904D04B0E006E040E006F4E
:10F8300002013B0EA46F010EA56F100EA66FC0EC67
:10F8400075F01D0E0101B95D23E156A50BD0006BCB
:10F85000E70EE66EB10EE66E010ED8ECB6F00101D1
:10F86000148F0ED056A108D0E30EE66EB10EE66EF0
:10F87000010ED8ECB6F004D00E0E006E56EC21F05E
:10F880000201560EA46F010EA56F050EA66F2E8005
:10F890000101B95106E133B40480CCEC75F02E8837
:10F8A000328A0D0E0101B95D03E00E0EB95D29E14A
:10F8B000050E006F38ECC2F0010197A122D0050EB1
:10F8C000006F7FECBBF029ECBAF03A0EE66EB20E98
:10F8D000E66E010ED8ECB6F029ECBAF00D0EB95D6B
:10F8E00003E1D251020B06E10E0EB95D0AE1D251DD
:10F8F000040B07E0DF0EE66EB10EE66E010ED8ECEB
:10F90000B6F0190E0101B95D14E10B0E006E049002
:10F9100097B1048004B004D0010E006F440E006E55
:10F92000C0EC75F00201970EA46F010EA56F010ED9
:10F93000A66F2A0E0101B95D0BE12AB50480CCEC5B
:10F9400075F002012A0EA46F010EA56F040EA66FBA
:10F950000101040E006F160EB95D16E1050E006F71
:10F96000D45105E0030ED45D0DE10A500BE0D451F3
:10F9700004E18AA504D0048002D08EB50480CCECCA
:10F9800075F002D038ECC2F01C0E0101B95D0EE139
:10F99000050E006F020178B90480CCEC75F002010D
:10F9A000780EA46F020EA56F100EA66F180E01013F
:10F9B000B95D3CE18CECCFF0110E02017025E4EC56
:10F9C000B8F001010E6F140E02017025E4ECB8F0DE
:10F9D00001010F6F0E6A0F6A0201705103E1E8EC3A
:10F9E000BAF014D0700506E111EC1CF00101200EF4
:10F9F000106F0CD0020E705D09E159ECC0F00101EE
:10FA0000395104E0EFC90EF0F0C90FF00E0ED880A6
:10FA10000E54270E0F5402E20E6A0F6AB5ECBBF0CB
:10FA20000101115102E1100E116F148F0A0EB95D20
:10FA300060E1395120E030A213D0040E006F0901BB
:10FA4000E85102E12A0E0FD0E80508E1DA0EE66E71
:10FA5000B10EE66E010ED8ECB6F008D04B0E03D016
:10FA6000010E006F440E006E56EC21F00201E80E0C
:10FA7000A46F090E3DD01EECAAF0EEECBEF03A5198
:10FA800002E1440E0CD03A0504E1040E006F2A0E88
:10FA900006D0020E3A5D06E1040E006F4B0EE5EC57
:10FAA000BAF020D0030E3A5D1DE33A5113081AE371
:10FAB000550EE5ECBAF0030E01013A5D006E080E3A
:10FAC000005C04E21C0E146F00280BD0100E005CCA
:10FAD00005E2130E146F070E005C03D0130E146FB3
:10FAE000240E156F328A2E8002013A0EA46F010E89
:10FAF000A56F1F0E0101B95D17E1395102E10E0E2C
:10FB000003D0390504E1080EE5ECBAF008D0006B2B
:10FB1000D10EE66EB10EE66E010ED8ECB6F0020123
:10FB2000390EA46F010EA56F1A0E0101B95D3BE1FC
:10FB30002EA435D0016A1E0E015C0AE287ECBFF0EC
:10FB4000EF50E66E8EECBFF0BCECB8F0012AF3D7B4
:10FB500068ECD6F0BCECD4F00101279D269D17502F
:10FB6000800B0CE101012651400B08E12751400BAD
:10FB700005E18BEC4AF08EEC3AF0F1D7016A1E0EEB
:10FB8000015C0AE28EECBFF0EF50E66E87ECBFF04E
:10FB9000BCECB8F0012AF3D7BCECD4F00101050E9F
:10FBA00062ECC5F0328A280E0101B95D42E1050E12
:10FBB00062ECC5F02EA23BD0EEECBEF02F0EE5ECD1
:10FBC000BAF08250010B03E08250020B0DE18CEC85
:10FBD000CFF00101010E106F82B202D0040E106F3F
:10FBE000050E006F006A1DD0066A060E065C1EE256
:10FBF0000650040DF3508309006E050E065C02E109
:10FC0000BB0E006E00506CECC6F01A080DE2F00E50
:10FC1000005C0AE28CECCFF006C010F10101050E89
:10FC2000006F4DECD5F002D0062ADFD725822E8852
:10FC3000328A260E0101B95D66E1D5CA03F0D251C0
:10FC4000010B10E03751080B0DE0040E036E1BA0F2
:10FC500009D0030E036E0A011C5104E1280E216F26
:10FC600021CA1CFA0201DA5119E00101170E0E6FC8
:10FC7000010E006F035091ECBBF0EF5058ECBBF05D
:10FC80000101200E126F050E006F035097ECBBF0C0
:10FC9000EF5058ECBBF00101128F34D08CECCFF058
:10FCA0000501170506E1CC0EE66EB10EE66E010EFB
:10FCB00005D0C60EE66EB10EE66E010ED8ECB6F0BB
:10FCC0001BA009D0EEECBEF0C10EE66EB10EE66EE2
:10FCD000010ED8ECB6F005011751050DBAECB7F0DE
:10FCE000140E49260A0E4A22035002014924A46F29
:10FCF000000E4A201FECB8F068ECC2F0135102E18C
:10FD0000100E136F2E88340EB95D2EE12B5105E1D4
:10FD1000050E006F38ECC2F026D08CECCFF022B488
:10FD200006D0CC0EE66EB10EE66E010E05D0C60E04
:10FD3000E66EB10EE66E010ED8ECB6F02250040B62
:10FD400001E0010E0201A46FA56B910EA427020E23
:10FD5000A523D9ECC2F0EF50006E68ECC2F013514D
:10FD600002E1100E136F2E880F0E0101B95D1DE127
:10FD7000050E006F51C100F04DECD5F00101158F5B
:10FD8000135102E1100E136F0601426B0101515134
:10FD900002010B5D05E20601700E426F5A0E436FC1
:10FDA0000201510EA46F010EA56F230E0101B95D72
:10FDB0001AE1020E006F1E0E43255AECC5F0010138
:10FDC000006B1A0E43255AECC5F00101136B100E9F
:10FDD000146F120E156F0E5102E1100E0E6F0F51BF
:10FDE00002E1100E0F6F130EB95D1BE14FA305D09A
:10FDF000040E006F2CECC4F00DD0006B640EE5EC2B
:10FE0000BAF05D0E006E01014FA102D0600E006ECF
:10FE100056EC21F002014F0EA46F010EA56F030EE8
:10FE2000A66F140E0101B95D1EE1040E006F4FBBF9
:10FE300011D01C0E0E6F160E0F6F240E106F0D0ECC
:10FE4000116F5D0E006E4FA902D0600E006E56EC71
:10FE500021F002D02CECC4F002014F0EA46F010E71
:10FE6000A56F300EA66F2B0E0101B95D02E19CEC6F
:10FE7000D7F0240E0101B95D37E197A131D08CECA8
:10FE8000CFF0EEECBEF0000EE76E9919E8AE02D0AE
:10FE9000993503D0E750D88099550BE299C100F00D
:10FEA0004DECD5F00101100E0F6F105111E1100E45
:10FEB0000ED099C100F00001006C4DECD5F00101AD
:10FEC0000E0E0F6F105104E1100E0F6F0E0E106F1B
:10FED000050E006FB80EE66EB10EE66E010E02D092
:10FEE0002BECB9F0D8ECB6F05CC305F0055050EC43
:10FEF000BBF029ECBAF03C0EB95D0BE1140E006EBC
:10FF000050ECC6F002E0110E006EC0EC75F0328AC3
:10FF10002E883D0E0101B95D14E1ACECC3F0496ED1
:10FF20004A6AA7ECC3F0640D82ECB9F0030E006FCF
:10FF3000E2EC21F0060EE66E030EAFECBBF0328A67
:10FF40002E883E0E0101B95D07E1A2ECC3F0006E00
:10FF500071EC75F0328A2E88400E0101B95D12E114
:10FF600024ECC5F0006E040EDDECBFF0100E126F35
:10FF70002EECC5F002E10E0E126F29ECC5F0156FE4
:10FF8000148F2E883F0EB95D23E120ECC2F00AE108
:10FF9000E2ECB6F0EF50F00BE842E842E842E8420B
:10FFA0000A0803E1E2ECB6F0EF92E2ECB6F0060EDE
:10FFB000EB50006E005001E1002A4DECD5F001013C
:10FFC000135102E1100E136F180E126F158F2E8849
:10FFD000129E129C2E50100B07E01E50040B04E1E1
:10FFE0001B50080B01E1128C1E0EB95D03E01B0EC5
:10FFF000B95D05E1060EE66E050EAFECBBF0040E32
:020000040001F9
:10000000E15C02E2E16AE552E16EB5EFB6F002ECC6
:10001000C1F00101B951DE6EDD6AE9ECBDF0070EF9
:10002000EC02F3CFEDFFEF02F3CFEEFFF450ED263D
:10003000026A0F0E496E980E4A6E010E4B6E025008
:10004000E76E000EDFCF4CF0010EDBCF4DF0E75036
:100050004C26000E4D2260ECC2F0006EFBECD5F099
:10006000022A070E025CE5E3020EE15C02E2E16AAD
:10007000E552E16EB5EFB6F012000201030E686FB3
:10008000A46BA56BA6691996CAECBEF004E1E79DC6
:10009000E79BF2EC08F070EC13F00601426BA3EC66
:1000A000D3F024B898D8C0ECC0F003E0340EB95DAA
:1000B00005E12050040B02E083ECBAF0B4EC07F049
:1000C0002DA433D02D941EA602D09CEC2FF01E96AA
:1000D0005BEC0CF06EEC0CF024A405D0A3ECBBF0B0
:1000E0002494D4ECBFF01EA80BD01E980DC1E6FFDF
:1000F000CEEC51F0E5520DC1E6FFEAEC51F0E552CD
:100100002EA60ED02E96CFEC52F025ECBAF008E2D7
:1001100035ECB9F047ECBBF02EEC1DF071EC29F09A
:1001200030AE03D0309E5CEC6DF018AC03D0189C60
:1001300055ECC0F01E941200D9EC0AF0299202018D
:10014000355101E1258A70EC13F02E942E922CEC9F
:100150000BF00601426B0101B593A3ECD3F004EC64
:1001600065F02D9C0201686B0C0E076EA8EC5AF02E
:100170000101129C3B51010B01E0128C129E3B517C
:10018000020B01E0128E17A004D0E66A4D0E31EC8E
:10019000B7F09C0E28ECB7F00101E79DE79B120039
:1001A0000D500101B927B9AF02D0400EB96FB95156
:1001B000400801E2B96B1200230E00ECB8F0020E09
:1001C000006E12000101AE6BD890AC33D890AC3306
:1001D00028964CEFBAF00701099F918A64ECB2F0BF
:1001E00039ECC3F0209C33864CECC0F024984CECE6
:1001F000BBF0A0EF5FF0E66AE66AA1ECBAF0C00ED1
:100200000701081799ECB2F077EC13F08A96208C6E
:1002100033964CECC0F00701098F919A64EFB2F06D
:10022000B9ECB6F0100EE1263250200B14E01D5050
:10023000040B02E180EF87F01D50080B02E180EF14
:1002400087F0B9ECB9F002E180EF87F0F2ECBCF096
:1002500002E080EF87F002016851030A02E17EEFBD
:1002600087F0010A1DE0030A02E080EF87F02D9479
:100270002E9024982E98329A189C0101B583020181
:10028000A46BA56BA66919963CECD7F01F960101EB
:10029000269D279D0201020E686F25827FEC36F0B5
:1002A0002950020B16E02E50010B13E02E50100BBC
:1002B00010E189EC6FF029922F88D4EC75F00101E0
:1002C000B58DB58F640EAC6F4CEC6EF0D6DE57C2B8
:1002D000B9F117AE19EF87F0BAECBBF0A0EC11F052
:1002E000FF0813E0BBEC11F0006E0101395105E08D
:1002F000180E005C02E133ECC4F00101B59BB59926
:10030000179E2582238A80EF87F02E50100B12E073
:100310001E50040B0FE11B50080B0CE1090E155C7D
:1003200009E0290E155C03E11750100B03E125ECE1
:1003300007F004D00B0E155C04E19FDE179E80EFE2
:1003400087F017A0E7EF85F028B6EBEF85F0090EF0
:10035000155C02E1F1EF85F0EEECB8F066E01750C5
:10036000010B63E0080E155C06E01A0E155C03E055
:10037000100E155C5AE11550DF6E91C2F9F692C26B
:10038000FAF68DC2F5F68EC2F6F68FC2F7F690C277
:10039000F8F6100EDF5C01E118843EEC88F018944A
:1003A00071EC29F0100EDF5C0EE1006823EC22F006
:1003B00029ECBAF07FECBBF00101100E156F15C1EE
:1003C00014F115C113F1100EDF5C02E015EF87F098
:1003D00025ECBAF002E215EF87F02B51010802E399
:1003E00015EF87F0340EB95D09E17FEC2FF00009BD
:1003F00005E0F9C691F2FAC692F213D0C0ECC0F053
:1004000002E015EF87F06AEC2FF0000902E115EF2A
:1004100087F0F5C68DF2F6C68EF2F7C68FF2F8C6F3
:1004200090F2B3EC12F015EF87F02D0E0101B95DDB
:1004300037E10D0E155C02E015EF87F024A803D01C
:10044000CADE15EF87F0EEECB8F001E1BED0D3DEE6
:1004500008ECC2F005E0D8900B330A33E806FBE164
:1004600042EC5BF0496E640E495C09E342EC5BF0E0
:100470004A6E4B6A4B3408E202ECBEF005E2A00E75
:10048000E66E54EC5BF0E552E66A42EC5BF0E66E39
:10049000A1ECBAF00201FA0EB06F248815EF87F0D4
:1004A000210EB95D39E1220E155C17E1D45102E04D
:1004B000EEEF86F01F781FA80DD013A007D0020121
:1004C000FA0E1A6FD90E006E05EF87F095ECBFF0AB
:1004D00015EF87F0F2EC08F052D3120E155C04E130
:1004E0003EEC88F015EF87F0290E155C02E015EF61
:1004F00087F00701BA7BBAAB06D01FB815EF87F0BB
:10050000E66AC80E05D01FB815EF87F0E66A4E0EF2
:10051000E66E52EC08F0EBD22F0EB95D03E0340E1C
:10052000B95D56E1130E155C03E1229415EF87F0D7
:100530001B0E155C03E1228415EF87F0290E155C74
:1005400008E12F0EB95D02E015EF87F02B7415EF6F
:1005500087F00D0E155C02E015EF87F020B434D360
:100560002B51090806E2AA0EE66EB10EE66E010EE8
:100570000AD02F0EB95D0AE1D45119E07F0EE66E64
:10058000B20EE66E010E9BECC5F01CD0340EB95DC8
:1005900002E015EF87F0E2ECBEF009E10101D405BD
:1005A00003E0020ED45D06E13350040B03E0208427
:1005B00015EF87F04A0EE66E950EE66E010EE66EBA
:1005C00053EC22F0E552E552E552258E15EF87F007
:1005D000320EB95D0BE1140E155C02E1337602D0E8
:1005E00006EC0AF099ECB2F015EF87F029B201D3CE
:1005F000D9ECC4F007E198ECC0F004E0310EB95D2D
:1006000001E0D6D20A0E0C5C01E3D2D21F0E01012A
:10061000B95D23E10C040FE15F71A20EE66EB10E2D
:10062000E66E010E14ECB7F001015FA102D02D0EB1
:100630001C6F960EAC6F060E0C5C01E0F6D35F7576
:100640009A0EE66EB10EE66E010E14ECB7F00101E3
:100650005FA58FD32B0E1C6F8CD3050EB95D08E1FF
:10066000070E0C5C01E3E1D30C04E96F15EF87F092
:10067000180EB95D0DE10C0401E0D7D3930EE66EC0
:10068000B10EE66E010E14ECB7F097C21CF170D3F8
:10069000260EB95D01E0FCD10C0403E0020E0C5CF7
:1006A00002E10CC017F5070E0C5C02E13EEC88F08D
:1006B000030E0C5C01E0B4D10201DA5101E0B0D1CB
:1006C00012B609D08B0EE66EB10EE66E010ED7ECB7
:1006D000C3F0258EA5D1860EE66EB10EE66E010E34
:1006E0001DECB7F00201DA69050ED5CADBFFC6ECD6
:1006F000BEF00FE03751080B0CE0040EF36E050E50
:10070000F3CFDBFF1BA005D0030EF36E050EF3CF76
:10071000DBFF030EDB6A010EDB6A040EDB6A020EEE
:10072000DB6A1BA008D0140EF36E030EF3CFDBFFC1
:10073000DE52140EDD6E0C0EDB680D0EDB68D95038
:100740000A0FE96EDACFEAFFEE68ED680E0EDB6A9B
:100750000F0EDB6A0201DA5101E13CD1050EDB50DC
:1007600091ECBBF0030EE0ECC4F0040EDBCFEFFF26
:1007700094ECBEF0E66ADBEC36F0E552000908E0E6
:100780000201DA6B179E156A320EDDECB6F022D14B
:10079000FF0E0201DA5D08E194ECBEF0FA0EDDEC2A
:1007A000B6F00201010EDA6FD4EC75F08EECD3F0E6
:1007B000050EDDECB6F00E6A0F6A026A0250022ADC
:1007C000496E080E495C06E2990E4BECB8F0C6EC97
:1007D000B8F0F4D70A0EDBCF49F00B0E56ECBCF0A4
:1007E00010E20A0E0EC0DBFF0B0E0FC0DBFF030E84
:1007F000DB5072ECBCF0040EDB50E76E020EE7CF6C
:10080000DBFF0C0EDBCF49F00D0E56ECBCF006E220
:100810000C0E0EC0DBFF0D0E0FC0DBFF0E0EDBCF8C
:1008200049F00F0EDBCF4AF0D2ECC3F006E20E0E19
:100830000EC0DBFF0F0E0FC0DBFF030E0201DA5DFF
:1008400016E1090EDB50F36E040EDBCFF4FFF3501C
:10085000F45C0AE3070EDB509AECBFF002E3DA6BBC
:1008600079D7030EDB2A64D0040EDB2A73D7040E7B
:10087000DB50A6ECBAF001E14A5004E0020EDA5D6A
:1008800001E09FD0030EDB50A6ECBAF001E14A5024
:1008900007E01B50010B4EE0500E9AECBFF04AE30C
:1008A000030EDA6F060EDB6A080EDB6A070EDB68E2
:1008B000090EDB68020EDB50070807E2020EDB5070
:1008C000F80FE76E080EE7CFDBFF020EDB5074EC8B
:1008D000B7F004E6F80E495C000E4A5807E2020E33
:1008E000DB50080FE76E090EE7CFDBFF010EDB5090
:1008F000070807E2010EDB50F80FE76E060EE7CFA0
:10090000DBFF010EDB5074ECB7F004E6F80E495C37
:10091000000E4A5807E2010EDB50080FE76E070E83
:10092000E7CFDBFF060EDB50E76E030EE7CFDBFF02
:10093000080E39D01BA003D0030E496E03D0050E5C
:10094000496E030EB1ECC3F0030EE7CFDBFF020EDE
:10095000DA5D01E3FFD6960E0E6E0F6A1BA003D080
:10096000FA0E0E6E0F6A0E0EDBCF49F00F0E56EC2C
:10097000BCF01CE20C0EDBCF4BF00D0EDBCF4CF0CD
:100980000E0EDBCF3DF00F0EDBCF3EF00E503D5C88
:100990004D6E0F503E584E6E4D504B5C4E504C5865
:1009A00005E2020EDA6FDB50E76E10D0040EDB6A50
:1009B0000C0EDB680D0EDB680E0EDB6A0F0EDB6AB9
:1009C000C9D6050E496E040EB1ECC3F0040EE7CF94
:1009D000DBFFC0D6050EDB5091ECBBF0010EE0EC66
:1009E000C4F0020EDBCFEFFFDDEC0BF02582238A93
:1009F000820EE66EB10EE66E010E1DECB7F00A0E29
:100A00004BECB8F00E6E0F6A0EC0E6FF0FC0E6FFAB
:100A100023EC11F0E552E5523B0E66ECB7F024846E
:100A2000040E0C5C1BE1C6ECBEF016E03751080B5F
:100A300013E01B701BA006D07A0EE66EB10EE66EB8
:100A4000010E05D0720EE66EB10EE66E010E14ECCC
:100A5000B7F0D4EC75F002D006EC0AF0050E0C5C91
:100A600001E0E3D1A3ECBBF00101377737A706D053
:100A70006A0EE66EB10EE66E010E05D0630EE66EEE
:100A8000B10EE66E010E14ECB7F0C3EC3FF001D1ED
:100A90002A0EB95D01E1C9D1150EB95D46E10C041C
:100AA00010E1567F4A0E6FECB7F0010156AF03D04C
:100AB0004B0E6FECB7F0279201013B959FECBCF019
:100AC000B4D1030E0C5C15E157755B0EE66EB10EEA
:100AD000E66E010E14ECB7F0010157A5A6D1530E36
:100AE000E66EB10EE66E010E9BECC5F0E552E552E6
:100AF00070D1040E0C5C09E18D7B500E6FECB7F0E9
:100B000001018DAB92D1510E0CD0050E0C5C01E0B1
:100B100065D18D77520E6FECB7F001018DA785D1AD
:100B2000530EE66E45EC22F054D1330EB95D07E169
:100B30000C0401E07AD18A737EEC12F076D1250E96
:100B4000B95D03E0310EB95D10E1090E0C5C01E303
:100B50006CD10CC05EF35EC340F602011E0E276F1F
:100B600074EC6DF07DEC6DF060D17DEC5AF0000915
:100B700008E0080E0C5C03E20C0403015C6F2582A4
:100B800054D12B0E0101B95D10E1040E0C5C01E3A0
:100B90004CD10C0403017F6F7F51E824030F060141
:100BA000406F02011E0E276F40D129A2A9D119D092
:100BB00029B217D00D0E155C01E0A2D12050040B14
:100BC00001E19ED107019D6B83ECBAF02ED117A8ED
:100BD0001FD128A603D0E2EC80F027D1090E155CC6
:100BE00003E13DEC80F021D1140E155C15E129A242
:100BF00005D03DEC80F057C2B9F117D134EC6EF05E
:100C0000FF0E005C01E111D1140E155C02E100C081
:100C10002CF1DCEC80F009D1230E155C01E070D1E1
:100C2000080E0101B95D13E0250EB95D10E0310E2B
:100C3000B95D0DE0320EB95D0AE0210EB95D07E045
:100C40000A0EB95D04E0260EB95D01E059D1260E09
:100C5000B95D23E137A7C2D03AECC4F08EECD3F0F3
:100C60000DC1DFFF036A100E035C10E2010137972C
:100C7000C3EC3FF019CA1DFA1ECA22FA01013787D8
:100C800003C00DF1A3ECBBF0032AEDD7DFCF0DF1CC
:100C9000096A2484DDEC0BF0C8D0080EB95D06E1CA
:100CA0000201BE6BBF6BC06BC16BBFD0210EB95DC3
:100CB00043E1E7AB26D0460EE66EB10EE66E010EBE
:100CC00014ECB7F08EECD3F00101579B6A0E026E64
:100CD000750E025C14E20250096E0068036A03504C
:100CE00074ECB7F002E600ECC0F007E20350E82431
:100CF000016E0BEC34F0032AF2D7022AE9D7096A15
:100D000094D03AECC4F00101400E696F780E6A6F1E
:100D10007D0E6B6F010E6C6F2BECB3F04C0EE66E1C
:100D2000C30E31ECB7F00101C42B71EC29F00101C5
:100D3000C40771EC29F079D00A0EB95D33E139515D
:100D40001BE03050020B4AE00A0E2B5D47E2400EDA
:100D500044ECC5F0420EE66EB10EE66E010EBFEC3D
:100D6000C1F03F0EE66EB10EE66E010E1DECB7F05F
:100D70000101960EAC6F59D0400E44ECC5F00068EE
:100D80005EECC0F0056A020E016E400E055C06E2E4
:100D90000BEC34F0052A040E0126F7D7096A9CEC07
:100DA0002FF043D0320EB95D16E109ECB8F016E031
:100DB000460EE66EB10EE66E010ED7ECC3F0B00E35
:100DC0000D25016E006A0BEC34F0010EE66E48EC66
:100DD00010F0E5522AD0030ED45D03E106EC0AF0D0
:100DE00024D048EC6DF0026A080E025C08E2015063
:100DF0000224A9ECBBF0100EEF6E022AF5D71AEC14
:100E00001AF0308E670E006E23882FEC22F00DD082
:100E100017AA0BD0090E155C08E104EC65F002017D
:100E2000846B0101190EAE6F2886179E2D842582D2
:100E3000238A01012651400B03E11950080B23E0DE
:100E4000269D0701A25103E00101246B59D0EEEC6D
:100E5000B8F003E13250200B14E1010E0D6E0101D8
:100E600026BF0D6819B60D6A89EC6FF019962582B8
:100E70001A0E0101B95D3BE0280EB95D38E02D8402
:100E800036D0258E34D02751400B31E02950020B4B
:100E90002EE1279D279D256B25C124F125822E94C7
:100EA0002E9224A802D0EBEC80F0C0ECC0F003E05E
:100EB000340EB95D02E183ECBAF04CECBAF0F2EC1E
:100EC00008F0010E0D6E010127BF0D68D0EC80F017
:100ED0001E942D9C0601436B43C642F6A3ECD3F04F
:100EE00018AC03D0189C55ECC0F070EC13F0AFECCC
:100EF00066F0AFEC66F00201236B02D09CEC80F050
:100F0000100EE15C02E2E16AE552E16EB5EFB6F087
:100F10008250010BFDE08250020BFAE0640ECFEF2D
:100F2000C2F0130E155C06E01B0E155C03E0140EF8
:100F3000155C01E1010C000C640E0101BA5D15E2C3
:100F40000050E66E18EC30F0E55200090CE02EEC93
:100F50001DF025ECBAF005E2E651040B02E049EC85
:100F60002AF02988120037EC07F0120044C10CF275
:100F70003FEC32F031EC32F0360E006E0DEC22F028
:100F8000B70E02ECBDF00101B66B0601030E426F15
:100F9000509750951F965A0E436F95EFBCF071EC29
:100FA00045F02CEC0BF00601426BB5EC32F0A8ECEE
:100FB0005AF00CC244F112007CECC0F00BE0760554
:100FC0000AE0080E765D07E0030E765D04E0040E8D
:100FD000765D01E0000C010CB9ECB6F055ECC1F007
:100FE00003E00C0E076E41D0208E18980901EE6BBD
:100FF000FE0EDB501BE00101855118E03350080B59
:1010000015E02B50100B12E118885DECBCF085C187
:1010100048F1B4ECC4F00101395108E065ECBDF0D1
:101020000EECC3F003E1FA0EDDECB6F077EC13F052
:10103000F5EC08F0E66AB2EC19F0E5522A84006893
:101040000DEC22F0B9DF000903E1006818EC22F092
:1010500009EC1CF001019D6F1FA202D0D56B01D0DD
:10106000D46B49EC2AF076EC5BF0B5EFB6F06C0E81
:1010700000ECB8F0258E2B9AADEF0CF07BECC6F0AF
:10108000179E2582238AB4ECBDF0BAECBBF00101B7
:10109000AC5105E0E451040B02E1010EAC6FA0EC91
:1010A00011F0FF080FE0BBEC11F0006E01013951A7
:1010B00005E0180E005C02E133ECC4F00101B59BC1
:1010C000B5996AD102017F5113E1230E155C41E00D
:1010D0000101E651800B0CE12C50040B09E12C506E
:1010E000080B06E11950100B03E1E851400B31E009
:1010F000010EDF6E0101E6AF04D0E69F9FECBCF06D
:101100001ED02CA402D02C941AD019A802D0199861
:1011100016D02CA60FD007AE02D070EC13F02C9690
:101120000901410EE66F460EE76FFDEC07F035EC66
:1011300005F005D0E8AD03D0E89D92EC46F0238A97
:10114000DF5004E021960101B59B258A5BEC0CF091
:1011500023D11AAC03D0F2EC07F01ED1BAECBCF0EC
:101160003EE01950040B3BE1048019AC13D00D0E86
:10117000155C03E11750010B03E1200E155C02E141
:1011800004901ED039EC09F0010EE66E52EC09F025
:10119000E55216D02390230E155C04E10701FA0EE8
:1011A000036F0BD007010351496E4A6AFA0E4918C2
:1011B00004E14A5002E1015103E01D82B0EC35F038
:1011C00004A00DD0249223BC24820101B597209461
:1011D00019AC02D00B0E01D00C0E076E58D01DAC0E
:1011E00005D039EC0AF0800E076ED6D01BECBDF0AE
:1011F00006E001014CECBAF00101E897CDD02FAA2E
:1012000003D046EC46F0C8D030A403D0C7EC48F079
:10121000C3D030AC03D043EC47F0BED023AE03D0F4
:10122000DAEC45F0B9D02450010B0EE0200E155C2D
:101230000BE0220E155C08E0410EE66E460E31EC26
:10124000B7F0D6EC45F0A8D032A003D0D3EC46F0EE
:10125000A3D0BCECC0F01DE064DE00090DE0020E7E
:1012600081ECBCF06BECB7F026E0CFECB7F023E1FB
:10127000030E0C5C0AE21FD025ECBEF006E017500E
:10128000100B07E00B0E155C04E1E6EC06F0010E16
:10129000A6D020A81FD0209844DE000915E0020E39
:1012A00081ECBCF06BECB7F006E0CFECB7F003E1FB
:1012B000030E0C5C09E2DDEC0CF0E66A0C50E66E05
:1012C00036EC6AF0E5524CD025940101B59B0AEC4E
:1012D0005CF062D02C50400B03E12C50800B54E0AA
:1012E000D9ECC4F023E0050E0C5C20E2040E0101F1
:1012F0002B03F350640F0C24FF0F026E4CECC2F072
:1013000001012B51005C03E02C50400B0DE002C0AA
:1013100044F195ECBCF0000903E12C50800B04E192
:101320000201010E296F38D0A2DE36D0230E155CE3
:1013300019E101014451ADECB8F0400E4403F35003
:10134000016E00680BEC34F0096A0101B66B06010E
:10135000030E426F95ECBCF01E0EE66E45EC22F0DB
:10136000E5521AD01750100B0CE02C50400B03E044
:10137000100E155C09E02C50800B03E0080E155C84
:1013800003E0ADEC0CF008D01F50100B07E0290E65
:10139000155C04E056EC0EF0000E21D00490380EDF
:1013A0001514080802E197D919D0380E1514100841
:1013B00002E16FDA13D0380E1514180802E19DDB34
:1013C0000DD0380E1514200803E11EEC8EF006D067
:1013D000380E1514280802E144EC8FF0000EE55297
:1013E000B5EFB6F017AE08D025ECBEF001E046DE52
:1013F0000101E3AB179EE39B12001AB202D0DDECB1
:10140000BBF0CDECBDF071EF29F0C0EC10F0E66A56
:101410001FEC26F0E5526DEF10F00101D551D45DBF
:1014200003E1B6ECBCF006E08AECB8F004E2030E8F
:10143000D55D01E2010C1F0E6FECB7F0410EE66EB8
:101440004E0E6BECBDF0000C0101DD9DD0BDDD8DBD
:10145000DC95CFB5DC85DD95D0B5DD8592ECC5F0AA
:10146000070BF36EF46EF9ECB7F0DC15F310DC6FDC
:10147000F4500A6ED451D55D03E11A82C6DF1A9288
:1014800012000701BAAD08D0BA9D83EC6AF01FB80C
:101490000CD0E66A4E0E07D0BA9B3492BA8D1FB8B4
:1014A00004D0E66ACB0E31ECB7F0B0EC07F0B4EF45
:1014B00007F02B9A28920201245102E135ECB9F091
:1014C0002BC100F0090E026E0101E3B10206100EFD
:1014D000155C24E11A88002A0250D880005405E2E5
:1014E000100E005C02E2100E006E0050180801E2BF
:1014F000006A100E005C3AE3100E005C016E090EEB
:10150000015C07E20150BAECC2F003E1002A012AB3
:10151000F6D7005018082AE2006A28D01A8A000676
:1015200000AE02D0180E006E100E005C06E20250F3
:10153000D880005402E20250006E0250D88000545D
:1015400015E2190E005C12E2100E005C016EFF0E37
:10155000015C07E00150BAECC2F003E100060106AD
:10156000F6D7100E005C02E20250006E00C02BF1B4
:1015700069EC13F047ECBBF0248C04900101D2BB62
:1015800004800201A751080802E2A76B09D004A059
:1015900006D0020E685D04E0A72B178E01D0A76B62
:1015A00025ECBAF002E2DEEC8FF02EEF1DF027EC16
:1015B000C6F0FE0EDB5002E0000E06D02850400BB5
:1015C00002E0030E01D0020EDF6E2850400B02E055
:1015D000060E01D0050EDF5C21E22850400B02E030
:1015E000030E01D0020EDF5C06E1FE0EDB5003E0CD
:1015F000520E82ECB7F0DF509BECB7F057ECBFF027
:101600000BE30050390808E3300E005C02E1540E91
:10161000006E005082ECB7F0DF2AD7D7E552B5EF65
:10162000B6F00101D4511CE10A01DA77BAEC0DF0F1
:101630000901410EE66F500EE76F0A01DAB7048028
:10164000FDEC07F00A01DAA703D00701BA8B02D03C
:101650000701BA9BBA9DB0EC07F034849DEFBBF054
:1016600006EF0AF0147C0101D4510BE0030ED45DA7
:1016700008E08D51100B16E0020ED45D02E0D40597
:1016800011E10901570EE66F440EE76F0A01D46BB2
:1016900014AC1AD00901530EE66F480EE76F0A0129
:1016A000030E11D009014C0EE66F4F0EE76F0A01D1
:1016B000010ED46F14AC08D00901480EE66F490E34
:1016C000E76F0A01020ED46F14AC0480FDEC07F042
:1016D000BEEF6AF01200E6ECC0F017A086D01550FD
:1016E0000D0A01E17BD0060A01E175D0020A63E030
:1016F000010A01E07AD0C0EC10F0D4C100F000047F
:1017000001E1002A020E005C02E1006A11D00050E3
:1017100005E1010196AD05D0040E09D0030E005C71
:1017200002E1020E04D0040E005C02E1020E006E23
:1017300004900101CFB10480000405E10450010BC5
:1017400002E0020E006E020E005C05E10450010B87
:1017500002E1010E006E0050E66E9DECBFF0D4C1B8
:10176000DFFF00C0D4F11F50020B06E0C4ECC0F054
:1017700003E1DFCFD4F11BD000C0D4F14AECB9F0C3
:101780001EAC03D00201098502D0020106810501C9
:101790004787010136AD05D0EAECC0F031ECB7F077
:1017A00006D0D40503E0020ED45D01E11A880201DF
:1017B000780E2C6F1AD019AA02D0258E16D03CECC8
:1017C000D7F0010136BD03D086EC5AF00ED0E66AA0
:1017D000EEDEE5520AD020ECC3F007D002012D5115
:1017E00003E0010E2D6F01D0208417A84FD01550B3
:1017F0000D0A2DE0060A24E0030A0CE0010A46E186
:1018000019BA27D00201010E686F1A880601509795
:1018100050953CD02C7E2CAE0BD035ECB9F0B6EC0C
:1018200087F0060102891A880201C80EDF6F2ED0E8
:1018300044C100F09CEC87F0CFEC87F01A8A26D0E8
:10184000258420ECC3F00101FA0EAC6F1FD019AA59
:1018500002D0258E1BD00301656B676B686B010E90
:10186000E66EECEC87F0E55233A610D000C249F0EA
:1018700001C24AF0020E0F0B04E0C0ECBBF0E80618
:10188000FCE149500201005F4A50015BE552B5EFAF
:10189000B6F017A0CFD01550130A01E1A0D0010A6D
:1018A00001E182D0020A68E0040A01E0C3D019AA6B
:1018B00002D0258EBFD025ECBAF05BE3395124E08D
:1018C0003050020B29E02B50100B26E123865DECF3
:1018D000BCF0320E006E690E02010B5D02E21E0EBC
:1018E000006E00500BECBAF03A0EE66EB10EE66EEA
:1018F000010E1DECB7F0320EDDECB6F0348EE66A68
:10190000ECEC87F0E55296D03A5106E02B50080BEC
:1019100003E02B50100B03E0C6EC20F08BD0020E3E
:101920003A5D21E133B606D0258E740E006E23ECAD
:1019300022F080D0FCEC5FF0E66AECEC87F0E55238
:1019400020AE78D05DECBCF01E0E006E5A0E020187
:101950000B5D02E2140E006E00500BECBAF0228810
:101960005AECADF067D03A0504E1D20E55ECBBF06D
:1019700061D006EC0AF05ED00201685104E001017A
:10198000269F97DD57D00101E88D00680DEC22F00D
:10199000EF0E02ECBDF01F9663EC46F0010136AD90
:1019A00049D06BEC46F046D0127601013B9B12A663
:1019B00003D050ECBEF004800901520EE66F490ED0
:1019C000E76FFDEC07F0A6EC39F01EAC03D0020186
:1019D000098702D0020106810501478D2BD011AE87
:1019E00004D0119EA4ECBFF009D011BC0AD0118C18
:1019F0000901410EE66F540EE76F0480FDEC07F01D
:101A00000BD011AC09D0118EA4ECBFF00480FDEC1A
:101A100007F00201780E2C6F5CEC1CF00201068DC1
:101A2000050147890201068F0501478B64EC1CF014
:101A300066ECB2F017A860D01550130A37E0070A19
:101A400031E0040A1AE0020A01E012001F721F507E
:101A5000020B05E0C4ECC0F002E11F921200090184
:101A6000530EE66F500EE76F1FB20480FDEC07F0D7
:101A70003DEC0CF00201068312002C7C2CAC06D04D
:101A8000B6EC87F0060101891A88120071EC29F082
:101A900044C1E6FFA9EC31F0E552CFEC87F029888C
:101AA0001A8A12002CC100F0BBEF6DF0F2EC06F0C8
:101AB000000909E0120EE66E950EE66E010EA7EC27
:101AC000B8F0E55212000101D27D09014E0EE66F19
:101AD000520EE76F0101D2BD0480FDEC07F08FECE0
:101AE00045F00101D251400B07E00201685104E1C9
:101AF0009CECBEF0CDEC45F0120017A036D015508E
:101B00001A0A0AE0010A31E1410EE66EC60E31EC16
:101B1000B7F0D1EC45F029D08AECB8F01EE0C0EC6B
:101B200010F01F50020B05E0C4ECC0F002E13DECE8
:101B30000CF00101030ED46F4AECB9F01EAC03D0D7
:101B40000201098502D00201068105014787540E72
:101B5000E66E440E31ECB7F008D00201685103E1A3
:101B6000C9EC46F002D006EC0AF017A866D0155072
:101B70001A0A2AE0010A01E012000101D45102E12F
:101B800011EF8BF0D40503E0020ED45D1BE10701D9
:101B9000BAA113D0147814A807D0D90E55ECBBF015
:101BA0004E0EE66EC10E06D0520E00ECB8F04E0E90
:101BB000E66E410E31ECB7F003D0149806EC0AF053
:101BC000FEEF46F006EF0AF00101D45106E0CFEC3B
:101BD000B7F003E121ECBAF02EE00101D4510FE19E
:101BE00036AD06D00601EA6BCCEC48F06FEFC4F0DE
:101BF0000601EA5101E00480FDEC07F01AD0CFECB9
:101C0000B7F003E121ECBAF014E00601EC5103E176
:101C1000010EEC6F01D0EC6B0901540EE66F440E1F
:101C2000E76F0601EC5101E00480FDEC07F0CCEC1D
:101C300048F0BAEF48F006EC0AF0120017A0D5D031
:101C40001550230A01E1B6D0010A2DE0020A01E095
:101C5000CCD024A011D00A01DA8FD6CA81F2D7CA1B
:101C60004AF2970E55ECBBF04D0EE66ECE0E31ECFF
:101C7000B7F091EC6AF0B9D06BECB7F003E0CFECC1
:101C8000B7F007E01A9407AE02D069EC13F0258C88
:101C900005D04E0EE66ECD0E31ECB7F02C862186C7
:101CA000E9EC38F0A2D024A011D0540EE66EC30E99
:101CB00031ECB7F00A01190ED76F030ED46F3484DC
:101CC0003388010EE66EC0EC17F072D06BECB7F003
:101CD00003E0CFECB7F022E01F88006A18EC22F096
:101CE0001350010B16E021ECBAF013E10201FA0ED9
:101CF0001A6F0701329CBA51200B01E0328CBA8B6B
:101D0000BA9DD90E55ECBBF0E66A130E22ECB7F083
:101D100002D095ECBFF0B0EC07F067D0010156514E
:101D2000800B18E0D40503E0020ED45D13E12772A6
:101D300027A206D0A4EC38F0530EE66ECB0E05D0E9
:101D4000E5EC37F0470EE66E4D0E31ECB7F09FEC48
:101D5000BCF04BD002013D5103E001013B9502D0A4
:101D600001013B750901530EE66F520EE76F010149
:101D70003BA505D00901430EE66F410EE76F010157
:101D80003BB50480FDEC07F09FECBCF001013BA5E6
:101D900006D0320EE66EB10EE66E010E05D02B0EA9
:101DA000E66EB10EE66E010E9BECC5F0E552E55213
:101DB000E5521BD001013BAB04D03B9BA8EC5AF091
:101DC00012D0060150A507D0218450955087420EAD
:101DD000E66ED60E06D0219450855097460EE66EDC
:101DE0004F0E31ECB7F0238A258217A84CD015503E
:101DF000230A2DE0010A1EE0020A01E0120001019F
:101E0000D07B0201078D09014E0EE66F420EE76F8F
:101E10000101D0BB0480FDEC07F0DDEC45F00101D1
:101E2000D051200B30E0020168512DE19CECBEF056
:101E300042EF46F01A88198821869FECBCF031ECFD
:101E4000C0F0E552EEECB8F01EE0FCEF5FF0010EE2
